S00A000047572E737265637C
S214400000A55AA55A0100000000000000001040005C
S21440100000F0422021144400155345001753450074
S214401010195345001B5345001D5345000000000072
S2144010200000000000000000000000001F534500C4
S21440103053534500000000005553450057534500A4
S21444010047573334342056302E322E352032303250
S214440110332E31312E362031323A30300A0D00003B
S20C4401803412AA5500000000E9
S214440200A55AA55A01000000000000000010440052
S2144402100000000000104400000000000000000041
S2144402200000000000000000000000000000000085
S2144402300000000000000000000000000000000075
S2144402400000000000000000000000000000000065
S2144402500000000000000000000000000000000055
S21444100000F0422021144400155345001753450070
S214441010195345001B5345001D534500000000006E
S2144410200000000000000000000000001F534500C0
S21444103053534500000000005553450057534500A0
S2144410405953450059534500595345005953450093
S2144410505953450059534500595345005953450083
S2144410605953450059534500595345005953450073
S2144410705953450059534500595345005953450063
S214441400595345005953450000BF00BF00BF00BFB5
S214441410FFF7FABF000000000000000000000000D4
S21444142072B64FF000004FF000014FF000024FF04C
S21444143000034FF000044FF000054FF000064FF055
S21444144000074F4801684FF0807201EA0201002904
S2144414501CD14C4801684FF0807241EA0201016099
S214441460494801684FF0010241EA020101604748D9
S21444147045F6F02101604AF20F5101604048016888
S2144414804FF0807201EA02010029F7D040484149F2
S2144414900160414801684FF00000814200D003E0FB
S2144414A03E4880F3088803E03D4880F3088822E0FD
S2144414B03C484CF2205101604DF6281101603A48F0
S2144414C03A4901600AE03A484CF2205101604DF630
S2144414D028110160374835490160FFE7364800283F
S2144414E009D03649364A521A013A04DD0020002310
S2144414F009C1083AFCDA3348002810D03249086853
S2144415004FF0010240EA020008603049304A521A5D
S214441510013A04DD0020002309C1083AFCDA2D48CC
S214441520002810D02C4908684FF0010240EA020017
S21444153008602A492A4A521A013A04DD0020002348
S21444154009C1083AFCDA274800684FF05A31884205
S214441550F9D0114801684FF00000814200D001E004
S21444156013F0FCFE13F026FF62B613F021FF00F0E2
S2144415703BF800BFFEE700BFAFF30080AFF3008048
S21444158010C32D4030C32D4004C32D4000C02D4011
S21444159008ED00E0001043200400264000F04220FE
S2144415A0000043201000274000002740400000FF72
S2144415B010C0464000C046400100000000004020E5
S2144415C0004044200100000094EF00E000000020AA
S2144415D0000001200100000090EF00E00000000041
S2144415E000800000E42440202DE9F04F87B05B4C97
S2144415F001F084FC5A4815F0FFFB5A494E2000255A
S21444160025F0AAFD58481CF087FD58481CF0A8FD54
S21444161001F0E7FB4CF24453E05800F029F901F09E
S21444162023FE00F04DFA00F029FA00F0A7F95049DD
S21444163000201FF0EDFE4F4900201FF0FFFE002162
S21444164008461FF0A5FF002144F6206208461FF016
S2144416505BFF2846013501F081FF062DF9D101F0E4
S214441660BDFB4CF23853444D4FF47A7054F8038023
S214441670E75805F1040BE25854F803900592E258F3
S2144416800292E2580392E2580492E25854F803A0B5
S214441690E6582C46019201F068FB08F0D1F9374829
S2144416A001F094FC00F0B4F82A6806F57A739A427E
S2144416B002D32E6808F0B3F922680AF1C8039A42A6
S2144416C003D3D4F800A008F0A3F9019B226864333E
S2144416D09A4203D32368019308F087F9049B22684F
S2144416E032339A4201D323680493039B226814330B
S2144416F09A4203D32368039303F0B2FB029B226807
S2144417000A339A4203D32368029308F032F92268D4
S21444171009F105039A4203D3D4F8009008F0A7F8D9
S214441720059B226802339A4203D32368059300F04C
S21444173070F822687B1C9A4200D32768DBF80020A6
S21444174008F101039A4203D3DBF8008008F03CF921
S21444175008F07CF90DF08AF8A6E700BF5C48412003
S214441760508C4600E803402094994600C4944600B2
S2144417707417402068174020940D4220B4824600D7
S214441780024B586800F00300704700BF0000264034
S214441790024600F03F00931010B583EA5203540803
S2144417A0534084EA121483EA121384EAD2049B0157
S2144417B084EA521403F0400314F0010F43EA000392
S2144417C00CBF80240024234319B99A4218BFFF2033
S2144417D010BD01290CBF1846FF20F9E73C2A0CD05F
S2144417E07D2A0AD0FE2A08D0BF2A06D092B20144E7
S2144417F0814204D1D043C0B270470022F7E710F8C4
S214441800013B1A4492B2FF2A84BFFF3A92B2EFE7F2
S21444181070470BF0B7B8704710B5104C002001F075
S21444182007FA2080012001F003FA0D4B2288188025
S2144418300C4B1A800AF010FF0AF032FF0AF054FFED
S2144418400AF076FF0AF098FF0AF0BAFF0AF0DCFFC7
S2144418500AF0FEFFBDE810400BF01EB856184020B4
S214441860541840200018402070477047704770470F
S214441870002110B50446084618F078FC01210020E3
S21444188018F074FC0221002018F070FC032100209C
S21444189018F06CFC002018F065FB0E49002018F088
S2144418A077FA0D4BA2B20020197818F0AFFB0B491B
S2144418B0002018F021FF0A49002018F01DFF0949AE
S2144418C0002018F019FF08490020BDE8104018F021
S2144418D013BF00BF0C9146004491460094924600C4
S2144418E0749246005492460034924600F8B50D462B
S2144418F006461F4928461F4F0EF006FA044670B1A6
S2144419004CF24453F85806F54553123307EB830715
S2144419107D60032E2BD8DFE806F01A212427002109
S21444192028460EF0E7F980B94CF24453F8580DF0C7
S214441930E1FF29460EF036F80DF086FB00220E4BEA
S2144419400DF004FD0DF0B0FEDDE72046DBE782B285
S21444195000210020BDE8F84019F018B982B20121F0
S214441960F7E782B20221F4E782B20321F1E7F8BD39
S2144419700000C8425C4841200000594008B503486E
S2144419801DF0BCFD024B187008BD00BF8C9C460081
S214441990AC474020F7B50123104C114D6370A21C90
S2144419A0EB68A91C0F480235009335F8023C1DF03D
S2144419B047FC00222073A01C6178134615F8017B6F
S2144419C0013310F8016BDBB2B7421CBF0122002181
S2144419D00A2BF3D102B1617003B0F0BDAC4740208E
S2144419E0A01F4020A09C46004B7C062B0AD1012217
S2144419F0054B1A74CA7B1A2A04D1032203F1110137
S214441A001DF05EBF704700BFA01F40204B7C062BD6
S214441A100AD10122054B1A74CA7B2A2A04D103220E
S214441A2003F111011DF04CBF704700BFA01F4020BA
S214441A301FB500231A210446039301238DF807306B
S214441A401EF084F80B4B03930B4B1A7C002AFCD0F5
S214441A501B7C63B102A920461DF07CFF8DF807006D
S214441A60039B5A1E039213B19DF80730F1E704B066
S214441A7010BD00BF006A1800A01F402008B5A12072
S214441A801CF090FB00220A49A1201CF08AFB094B5B
S214441A90094902220120C3F8F413C3F8982DC3F869
S214441AA0F813C3F8902D0549BDE808401DF07AB8F0
S214441AB09BEF45000000294004002800009C460097
S214441AC008B5A2201CF06EFB00220B49A2201CF095
S214441AD068FB0A4B0A4A01210020C3F8E023C3F8F6
S214441AE0AC1DC3F8E42302220649C3F8A42DBDE87E
S214441AF008401CF097BD00BFA1EF450000002940F8
S214441B0002002800249C460010B5082217490120EC
S214441B104FF480341DF002F90123082214490020B2
S214441B201CF06CFE002108461CF0B6FF022801D1CA
S214441B30013CF7D14FF48034002101201DF0F8F821
S214441B40022801D1013CF7D1094A0823A2F1080032
S214441B5012F8011B013B10F8014BA14204BF0131AE
S214441B6002F8011C13F0FF03F2D110BDB41F40204D
S214441B70BC1F402082B00190019B5A1E0192002B4C
S214441B80FAD102B07047044B4FF400224FF4FA7077
S214441B90C3F8C022FFF7EEBF00002940044B4FF4C1
S214441BA020124FF4FA70C3F8C022FFF7E3BF00BF19
S214441BB0000029402DE9F04104460D461046002910
S214441BC03ED1DFF8908050260B46C1B2564308F10A
S214441BD010072846BA19B04419F0E8FF1C484FF4D9
S214441BE0FB534FF4FB62D8F81410083603FB040387
S214441BF03744D3F8FC3802FB043203F17A0602F584
S214441C00107C02F5427240F82C1098F8581040F8B0
S214441C102210FB2212FB046200EB4212A94211D8A6
S214441C204FF4FB520133642102FB0404B3FBF1F28C
S214441C3001FB1233C4F8FC3804F521540123236015
S214441C40BDE8F08117F8016B013502F8016BE5E752
S214441C505C484120AC4740202DE9F04104460D46FF
S214441C60104600293ED1DFF8908050260B46C1B27C
S214441C70564308F521670120BA19B04419F096FF77
S214441C801C484FF4FB534FF4FB62D8F8141A08363A
S214441C9003FB04033744D3F8FC3802FB043203F155
S214441CA07A0602F5107C02F5427240F82C1098F839
S214441CB0581A40F82210FB2212FB046200EB421230
S214441CC0A94211D84FF4FB520133642102FB0404A9
S214441CD0B3FBF1F201FB1233C4F8FC3804F521548B
S214441CE001232360BDE8F08117F8016B013502F843
S214441CF0016BE5E75C484120AC4740202DE9F041C4
S214441D0004460D46104600293ED1DFF89080502602
S214441D100B46C1B2564308F546770220BA19B0447A
S214441D2019F044FF1C484FF4FB534FF4FB62D8F8B9
S214441D301C13083603FB04033744D3F8FC3802FB71
S214441D40043203F17A0602F5107C02F5427240F83A
S214441D502C1098F8601340F82210FB2212FB046201
S214441D6000EB4212A94211D84FF4FB5201336421CE
S214441D7002FB0404B3FBF1F201FB1233C4F8FC3853
S214441D8004F5215401232360BDE8F08117F8016B64
S214441D90013502F8016BE5E75C484120A458402031
S214441DA02DE9F04104460D46104600293ED1DFF8A1
S214441DB0908050260B46C1B2564308F61857032067
S214441DC0BA19B04419F0F2FE1C484FF4FB534FF4D2
S214441DD0FB62D8F81C1D083603FB04033744D3F8CB
S214441DE0FC3802FB043203F17A0602F5107C02F555
S214441DF0427240F82C1098F8601D40F82210FB22DE
S214441E0012FB046200EB4212A94211D84FF4FB5273
S214441E100133642102FB0404B3FBF1F201FB1233E9
S214441E20C4F8FC3804F5215401232360BDE8F0814E
S214441E3017F8016B013502F8016BE5E75C48412071
S214441E40A45840202DE9F04104460D46104600298A
S214441E503ED1DFF8908050260B46C1B2564308F573
S214441E60C4670420BA19B04419F0A0FE1C484FF4C5
S214441E70FB534FF4FB62D8F82416083603FB0403DE
S214441E803744D3F8FC3802FB043203F17A0602F5F1
S214441E90107C02F5427240F82C1098F8681640F808
S214441EA02210FB2212FB046200EB4212A94211D814
S214441EB04FF4FB520133642102FB0404B3FBF1F2FA
S214441EC001FB1233C4F8FC3804F521540123236083
S214441ED0BDE8F08117F8016B013502F8016BE5E7C0
S214441EE05C4841209C6940202DE9F04104460D465B
S214441EF0104600293ED1DFF8908050260B46C1B2EA
S214441F005643A8F1D8070520BA19B04419F04EFE36
S214441F101C484FF4FB534FF4FB6258F8D41C083665
S214441F2003FB04033744D3F8FC3802FB043203F1C2
S214441F307A0602F5107C02F5427240F82C1018F826
S214441F40901C40F82210FB2212FB046200EB421263
S214441F50A94211D84FF4FB520133642102FB040416
S214441F60B3FBF1F201FB1233C4F8FC3804F52154F8
S214441F7001232360BDE8F08117F8016B013502F8B0
S214441F80016BE5E75C484120947A40204FF4FB52CD
S214441F90054B02FB0033D3F8F808D3F8FC38C31AD1
S214441FA058425841704700BF5C4841202DE9F74FDE
S214441FB0D14D0021D14E4FF4FB692C4641F698781A
S214441FC037464FF0640A0846FFF7E0FF58BBD6F89A
S214441FD0F83809FB013202F5427257F822C008FB72
S214441FE0014200924FF4FB524A4302EB43123A44F6
S214441FF0019200F1010EC0B2844500F2A88009FBAC
S2144420000132013385F820C002F5107257F82220B9
S2144420106A624FF0010285F82120B3FBFAF20AFB0C
S2144420201233C6F8F8380131454406F5FB560629FE
S214442030C9D194F82130012B19D1002384F82130DA
S214442040636AB3F5407F00F0CF8000F29F80B3F51B
S214442050BA7F00F0D28000F28B80422B00F0D98009
S2144420607FD8402B00F0C380412B00F0C38041F65C
S214442070B973E25C012A0FD10022E25441F6BC73E4
S214442080E358932B00F0D68000F2C680912B00F0E4
S214442090CB80922B00F0CB8043F65173E25C012A4E
S2144420A014D10022E25443F65473E358962B00F0BE
S2144420B0E98000F2CA80822B00F0E18000F2BD8005
S2144420C0722B00F0E580732B00F0E58045F6E9635B
S2144420D0E25C012A14D10022E25445F6EC63E3584C
S2144420E09B2B00F0F98000F2E4808D2B00F00881F1
S2144420F000F2D780722B00F0F880732B00F0F88043
S21444210047F68163E25C012A0BD10022E25447F68B
S2144421108463E358722B00F0F980732B01D102F0EC
S214442120C5FD49F61963E25C012A40F0F7800022B7
S214442130E25449F61C63E358722B00F0EA80732B92
S21444214040F0EC8003B0BDE8F04F02F0DFBD019AEA
S21444215002EB000B009A9BF840BF02F800B07046B2
S21444216047E740F25512934281D101F011FD7EE7D4
S214442170B3F5BE7F44D040F22122934243D0B3F518
S214442180BC7F7FF474AF01F04DFD70E740F285529A
S214442190934226D00DD8B3F5AE6F19D0B3F5B06FD1
S2144421A019D040F2013293427FF461AF01F0FAFD58
S2144421B05DE740F29552934210D040F277729342D4
S2144421C024D0B3F5B26F7FF452AF01F0B9FE4EE7B8
S2144421D001F0F4FD4BE701F041FE48E701F0C2FE92
S2144421E045E701F085FE42E701F0BCFD3FE701F01C
S2144421F058FC3CE701F068FC39E701F0F1FC36E7AF
S21444220001F032FD33E701F04DFD30E701F0C2FE48
S2144422102DE701F077FC2AE740F2511293427FF40F
S2144422203BAF01F01FFF37E701F0C6FE34E701F08D
S214442230E9FE31E701F0F8FE2EE78C2B25D0922BF1
S2144422407FF444AF02F070F840E7AA2B26D007D8B4
S2144422509A2B0ED0A02B7FF439AF02F085F935E7E0
S214442260C82B09D0B3F5F36F7FF430AF02F046FACB
S2144422702CE702F039F929E702F002FA26E701F0E2
S214442280C1FF23E702F0D8F820E701F0E5FF1DE799
S21444229001F03EFF1AE701F083FF17E702F0B0F9BA
S2144422A014E7932B2FD0972B7FF42AAF02F016FB1C
S2144422B026E7C92B13D007D8A12B13D0AA2B7FF41B
S2144422C01FAF02F0DBFB1BE740F2997293427FF4A8
S2144422D017AF02F0B9FC13E702F058FB10E702F020
S2144422E00DFC0DE702F092FB0AE702F01BFA07E743
S2144422F002F060FA04E700BF408740205C48412073
S21444230002F03AFCFCE602F087FAF9E602F0B0FC8A
S21444231007E703B0BDE8F04F02F0DABC03B0BDE80F
S214442320F08FEC4BEC4A5969586C0A40EB49DFF89D
S214442330CCC32DE9F0475A610022E94E4FF000081D
S2144423405A654FF0000983F86F201A67E54DDFF8A9
S214442350B0E3DFF8B0A3C3E90212197C21F0070109
S2144423601974596A31405962196C01F00041196474
S214442370DD4908405864986C00F0604040F4C8203A
S214442380986493F8580020F00F0083F85800D74814
S2144423909C6DC3E91302D64820409865D86D3040FA
S2144423A0D865186E00F000401866B3F8640000EA7A
S2144423B00C00A3F86400B3F8680000EA0C00A3F825
S2144423C06800586F9C6F00F07F40D3F8987083F88D
S2144423D08C205867C74804409C67D3F8804004F074
S2144423E07F44C3F88040D3F8844004F07F44C3E974
S2144423F02142D3F890402C40C3F89040D3F8944000
S21444240004F07C44C3F89440BB4C2740C3F898700F
S214442410D3F89C7007F04047C3F89C70D3F8A0707C
S2144424200F40C3E92872D3F8A8700740C3F8A870D1
S214442430D3F8AC7007F04047C3F8AC70B3F8B0704C
S21444244062F30D07A3F8B070D3F8B47007F04047B2
S214442450C3E92D7293F8BC7027F0030783F8BC7069
S214442460D3F8C070C3F8D4A007F00047C3F8C070D0
S214442470D3F8C4702740C3F8C470D3F8C87007F0C4
S2144424807047C3F8C870D3F8CC7007F07F47C3F8DA
S214442490CC70B3F8D07007EA0E07A3F8D070D3F820
S2144424A0D87007F04047C3F8D870D3F8DC7007F00C
S2144424B07847C3E9377293F8E47062F3000783F809
S2144424C0E470D3F8E870074047F48037C3F8E87000
S2144424D0C7F30F4727F4FE77A3F8EA70D3F8EC70F7
S2144424E00F40C3F8EC70D3F8087107F04047C3F8C0
S2144424F00871D3F80C710F40C3E94372D3F81471D2
S2144425000740C3E94022C3E93E89C3F81471D3F8AF
S2144425101871A3F8282107F0404783F85421A3F8FC
S2144425206C21C3F838A1C3E9467293F8207127F0AA
S214442530030783F82071D3F8247107F06047C3F883
S2144425402471D3F82C7107F07047C3F82C71D3F874
S214442550307107F07F47C3F83071B3F8347107EA37
S2144425600E0ED3F83C712740A3F834E1C3F83C710F
S214442570D3F8407107F07847C3F84071B3F8447114
S21444258007F47847A3F84471D3F8487107F07E47B8
S21444259047F48037C3F84871D3F84C713940C3F8D0
S2144425A04C11D3F8501101F06041C3F85011D3F8E0
S2144425B068113140C3E95689C3F86811D3F87011DD
S2144425C0A3F874213140C3F8782183F88021C3F8F6
S2144425D07011D3F87C1183F8E82101F07F41C3F8E9
S2144425E0A021A3F8A421C3F87C11D3F88411C3F81E
S2144425F0A8212940A3F8AC21C3F8B02183F8B4211C
S214442600C3F8B82183F8BC21C3F8C02183F8C42199
S214442610C3E9611293F88C1121F00F0183F88C11F1
S214442620D3F8C81101F07C41C3F8C811D3F8CC11D3
S2144426302140C3E97822C3E96422C3E96622C3F889
S214442640CC1193F8D41183F8982221F00701C3F8EB
S214442650282283F82C2283F8D411D3F8D411C3F853
S214442660302221F0FF4183F83422C3F8382221F483
S214442670FF0183F83C22C3F8402221F4FF4183F84B
S2144426804422C3F8482221F0780183F85622C3E94D
S2144426907512D3F84C122140C3F84C12D3F850129A
S2144426A001F07E41C3F8501293F89C1221F01F01AA
S2144426B041F0010183F89C12B3F8A01262F30901B9
S2144426C0A3F8A01293F8A41221F00F0183F8A412E1
S2144426D01AE000BFC083402000F807F80000E281FB
S2144426E00000F0FF0000FEFF000080FF0080204E48
S2144426F00F0000F00000FCFF0000C0FF00C0FFFF1A
S21444270000F0FFFF0000C04B93F8A81262F30201EA
S21444271083F8A812D3F80412314093F8AC62C3F895
S2144427200412C1F30F4162F3030621F47F6183F878
S214442730AC62A3F80612D3F80C127B4E01F00041AB
S21444274083F80822C3F81422C3F80C12B3F8101204
S214442750A3F8E42201EA0C0CD3F8181201F07F41E6
S214442760A3F810C2C3F81812D3F81C120140C3F8D9
S2144427701C12D3F824120C40D3F8C8122940C3F8CC
S2144427802442C3F8C812D3F8B01201F07E41C3F80D
S214442790B012D3F8B41201F00041C3F8B41293F85F
S2144427A0B81221F00F0183F8B812B3F8E01201F41E
S2144427B00041A3F8E012D3F8BC1201F07841C3F804
S2144427C0BC12D3F8C01201F07F41C3F8C012B3F86C
S2144427D0C4123140A3F8C412D3F8E01221F0FF41EA
S2144427E021F4FF01C3E9B489C3F8E012C3F8E82230
S2144427F093F8EC12D3F80C4362F30001C3F8202399
S21444280004F0784483F8EC12D3F8F012C3F80C437F
S21444281001F07F41D3F81043C3F8F01204F07F442C
S214442820D3F8F412C3F810430140C3F8F412D3F8B3
S214442830F81201F04041C3F8F812D3F8FC1201F044
S2144428407841C3F8FC12D3F8001301F07841C3E989
S214442850C01293F8081362F3000183F80813D3F800
S21444286030132940C3F83013D3F8181301F07E41CF
S214442870C3F81813D3F81C130D40B3F8141331409F
S214442880C3F81C53A3F8141393F8241362F30001FB
S21444289083F82413D3F8281301F07F41C3F8281390
S2144428A0D3F82C13C3F85C230840D3F84813C3F872
S2144428B06C2301F04041C3F82C03C3F84813D3F803
S2144428C04C1301F07841C3F84C13D3F8501301F07D
S2144428D07841C3E9D41293F8581362F3000183F89D
S2144428E0581393F8601362F3000183F86013D3F827
S2144428F0641301F07F41C3F8641393F86A1321F01C
S214442900030183F86A1393F8701362F3000193F893
S214442910762322F0030283F87013C3E9CE8983F842
S2144429207623BDE8F08700BF00E0FFFF41F69873CA
S2144429300849002258430B182830DA64084483F8C0
S21444294048202023013B00F8012B13F0FF03F9D164
S214442950704700BF4087402041F6987310B55843EF
S2144429600B4C41F692732218D35A28225A4300231A
S21444297011185030104421441A46204481F87030CF
S2144429804B67013300F8012BDBB2202BF9D110BD85
S214442990408740202DE9F8439946234B0546884610
S2144429A003EB00139B6A402B31D820494FF4FB536A
S2144429B003FB001342F644015B5843B341F6987652
S2144429C01B4C00274FF0280C06FB00F3E11801F5DA
S2144429D0FC511031F8B248451BD328467543FFF7DF
S2144429E0A5FF41F69071601928260122435A06FB3A
S2144429F0035513442C4484F87120C4F8748084F836
S214442A007090C824B3FBF4F204FB12334352BDE87F
S214442A10F883088812F807E00CFB0030204438445A
S214442A20013780F850E0D5E7A01F40205C4841209D
S214442A304087402041F6987241F692732DE9F3415F
S214442A4002FB00F14E4D04466A18D05A282202FB77
S214442A5000122A4492F87020082A31D8494B08229A
S214442A6003EB04139A62282341F6947603FB00F2A0
S214442A7041F6987320466343D118EF1850332944DF
S214442A801344414A2B4402EB041200934B6FB95D46
S214442A9019F014F8012C80462FD143F62C711C20D3
S214442AA06B5C0133B3FBF0F200FB12336B54B8F1AA
S214442AB0000F2BD0B8F1020F40D002B0BDE8F08131
S214442AC0102A04D82F4B102203EB0413CAE7182A03
S214442AD005D82C49182301EB04118B62C3E7202A3E
S214442AE004D82849202301EB0411F6E7402ABAD833
S214442AF02449402301EB0411EFE7BB5D0E2101336B
S214442B00B3FBF1F201FB1233BB55D0E72046FFF787
S214442B1023FF41F6987041F69271604328242E189C
S214442B20735A04FB03040133C8202544B3FBF0F274
S214442B3000FB123385F871807352BEE72046FFF7D8
S214442B400BFF41F6987041F69271002244432820C8
S214442B502E19735A00FB03440133C820254485F8D4
S214442B607120B3FBF0F200FB1233064A7352D2E9EB
S214442B702231013341F10001C2E922319DE700BF11
S214442B8040874020A01F4020C41F4020F8B50024A2
S214442B900A4D41F698760A4F06FB04F22821E0B225
S214442BA0D35B01FB03232B4493F87130012B01D1F3
S214442BB0FFF740FF0134062CEED1F8BD4087402095
S214442BC0D2A6402008B50B21034824F00DFA034B47
S214442BD083F8280908BD00BF02172940947A40208C
S214442BE001290A4628BF0122072819D8DFE800F041
S214442BF004070B0D1012141600210A4801E00A219E
S214442C00094824F0B8B90C21F7E702210748F8E749
S214442C100D21F2E70E21F0E70F21EEE70021F5E75C
S214442C20704700BF02172940101729400017294053
S214442C3007281AD8DFE800F004070B0E1013151700
S214442C4008210B4801E00B210A4824F0CDB90121A4
S214442C500948FAE70B21F4E704210848F5E705217B
S214442C60FBE70821F9E70A21F7E7FF20704700BF92
S214442C7006172940021729401217294004172940ED
S214442C8001284FF002010CBF0022012210B5044671
S214442C90034824F070F9034A4CF24053D45010BD14
S214442CA0081729405C48412005281DD8DFE800F075
S214442CB003080C1014180D4A4CF27453D05A70473B
S214442CC00A4A4CF27653F9E7084A4CF27853F5E749
S214442CD0064A4CF27A53F1E7044A4CF27C53EDE749
S214442CE0024A4CF27E53E9E7FF2070475C48412095
S214442CF008B50621002012F0BEFE024A4CF2745378
S214442D00D05208BD5C48412010B50221012012F083
S214442D10B2FE064C4CF276532B21E052012012F0C0
S214442D20AAFE4CF27E53E05210BD00BF5C484120E0
S214442D3010B50321022012F09EFE094C4CF2785343
S214442D400421E052022012F096FE4CF27A530521FA
S214442D50E052022012F08FFE4CF27C53E05210BD3B
S214442D605C484120002112F073BD084A4CF23853A7
S214442D7082B00749D35800930B68009A9B1A019374
S214442D80019B8342F8D902B0704700BF5C4841209B
S214442D90940D422038B50F4D0F4C95F890305BB9E2
S214442DA001234CF23C5285F89030A3580133A3508B
S214442DB0BDE8384006F008BE0AF010FB4CF23C5220
S214442DC0002385F89030A3580133A3504CF2385270
S214442DD0EBE700BFA01F40205C4841200020FFF7DF
S214442DE04FBF10B58D20244C1BF0DCF9002223493C
S214442DF08D201BF0D6F98F201BF0D4F900222049F1
S214442E008F201BF0CEF997201BF0CCF900221D49E9
S214442E1097201BF0C6F99A201BF0C4F900221A49E1
S214442E209A201BF0BEF9194900201DF003FD1849ED
S214442E3002201DF0FFFC17490A201DF0FBFC164932
S214442E400D201DF0F7FC2146012200201DF074FFE2
S214442E5004F59671012202201DF06EFF04F26C51B7
S214442E6001220A201DF068FF04F28C5101220D2035
S214442E70BDE810401DF060BF684B4120411246003B
S214442E80471246004D124600531246008C9D46009B
S214442E90609D4600349D4600089D460010B48AB99D
S214442EA00949D1F86C3891F8B848CA18013301F684
S214442EB0B801DBB282F8584610BC012241F84C3CBB
S214442EC01EF08AB810BC70475C48412010B48AB9DA
S214442ED00949D1F8743891F8D848CA18013301F62C
S214442EE0D801DBB282F8584710BC012241F8643C52
S214442EF01EF072B810BC70475C484120194B012143
S214442F0042F644000022195044F2A470195046F286
S214442F100470195048F2646019504AF2C45019506B
S214442F204CF22450195042F648015A5044F2A871C3
S214442F305A5046F208715A5048F268615A504AF25A
S214442F40C8515A504CF22851C3E9C1225A504CF247
S214442F5048524CF2503199504CF244524FF4486126
S214442F60995070475C48412010B5064B4FF4FB54CB
S214442F7004FB003042F64803C15042F64C03C250AC
S214442F8010BD00BF5C484120094BD3E9C1218A42A9
S214442F900BD01A4492F8042202700020D3F804237B
S214442FA00132D2B2C3F8042370470120704700BFF1
S214442FB05C48412007B501220DF107018DF8070052
S214442FC000201DF00DFD03B05DF804FB0FB470B592
S214442FD0C2B0002446AA02AE52F8041B3046019200
S214442FE00EF0B2FD30460BF073FEC5B2E3B29D421E
S214442FF004D842B0BDE8704004B07047305D013438
S214443000FFF7D8FFF2E708B58E201BF0CBF89620E2
S2144430101BF0C8F80748FFF7D9FF074900201CF003
S21444302089FB012005491CF085FB0548BDE808409E
S214443030FFF7CCBF08814600DC9C4600B09C4600A7
S214443040108146000B2938B5044614D142F6440391
S2144430500E4D00220E48EA50FFF7B8FF42F64803EA
S214443060EB581BB142F64C02A85898472046BDE898
S214443070384019F099BA074B1A6832B1002206480C
S2144430801A60BDE83840FFF7A1BF38BD5C48412010
S214443090168146009C704120328146000B2938B583
S2144430A005460E4C13D144F2A47300220C48E25059
S2144430B0FFF78CFF44F2A873E3581BB144F2AC729A
S2144430C0A05898472846BDE8384019F06DBA44F2EF
S2144430D0A073E2580AB10022E25038BD5C48412051
S2144430E0518146000B2938B5044614D146F2047380
S2144430F00E4D00220E48EA50FFF768FF46F208736A
S214443100EB581BB146F20C72A85898472046BDE8C7
S214443110384019F049BA074B1A6832B100220648BB
S2144431201A60BDE83840FFF751BF38BD5C484120BF
S2144431306D8146005CAF4120898146000B2938B535
S21444314004464FF4FB55134815D105FB040542F6D7
S214443150440300221048EA50FFF738FF42F648037B
S214443160EB581BB142F64C02A85898472046BDE897
S214443170384019F019BA05FB040404F521542368B1
S21444318033B1002305482360BDE83840FFF71EBF2F
S21444319038BD00BF5C484120A7814600C381460035
S2144431A00B2938B504464FF4FB55134815D105FB97
S2144431B0040542F6440300221048EA50FFF706FF8F
S2144431C042F64803EB581BB142F64C02A8589847BF
S2144431D02046BDE8384019F0E7B905FB040404F579
S2144431E02154236833B1002305482360BDE83840A2
S2144431F0FFF7ECBE38BD00BF5C484120E281460084
S214443200FE8146000B2938B504464FF4FB55134857
S21444321015D105FB040542F6440300221048EA5043
S214443220FFF7D4FE42F64803EB581BB142F64C0275
S214443230A85898472046BDE8384019F0B5B905FB6C
S214443240040404F52154236833B10023054823605D
S214443250BDE83840FFF7BABE38BD00BF5C484120E1
S2144432601D8246003982460038B50A243C4D29461C
S214443270002013F011F838B1013C14F0FF04F6D1E5
S21444328021463848FFF7A2FE0A24374D2946012036
S21444329013F002F838B1013C14F0FF04F6D10121D2
S2144432A03048FFF793FE0A24304D2946022012F098
S2144432B0F3FF38B1013C14F0FF04F6D1022129484B
S2144432C0FFF784FE00222A49B4200A241AF069FF34
S2144432D000222849B5201AF064FF00222649B62069
S2144432E01AF05FFFB4201AF05DFFB5201AF05AFFBB
S2144432F0B6201AF057FF002012F064FC38B1013CA7
S21444330014F0FF04F7D121461C48FFF75FFE0A2459
S214443310012012F057FC38B1013C14F0FF04F7D1F9
S21444332001211648FFF752FE0A24022012F04AFCF6
S21444333038B1013C14F0FF04F7D102210F48FFF7DF
S21444334045FE0121002012F0BFFC0121084612F080
S214443350BBFC01210220BDE8384012F0B5BC00BFDA
S21444336078904600748246001C904600C08F460003
S214443370756845007B68450081684500588246006C
S21444338038B51C4C0546206804302044FFF7FCFD45
S214443390012801D1012038BD2368E21810790A2893
S2144433A010D00D280ED0082815D123B1013B124861
S2144433B02360FFF70BFE2368AB42EBD32544002083
S2144433C0E87006E00D48FFF701FE2368002023441A
S2144433D018712060DFE7A0F120035E2BEBD8FFF7DF
S2144433E0E9FD2368E11801330A792360303A81F80D
S2144433F00421E0E75C4841208982460098824600E2
S21444340010B58020FFF7BCFF90B90A4C23797BB1F6
S2144434100949201D0BF052FC20B90848BDE810406D
S214443420FFF7D4BD211D0648BDE81040FFF7CEBDCA
S21444343010BD00BF5C4841208D8246009382460002
S2144434409B8246002DE9F04F082389B0002492461B
S2144434503B4A054689464FF064081068EDB2516809
S21444346002AF012622468DF810408DF81C40DFF846
S214443470E8B0CDE905346B4403C35146484623F0CF
S2144434807AFD04AA214640F255532846CDF80480D6
S21444349000978DF81C608DF81040059418F072FF64
S2144434A0284B04AA2146284602934FF607738DF804
S2144434B01060ADF80C300623CDE9007805935B46E2
S2144434C018F060FF204A0623214602924FF6FF7208
S2144434D0059328465B46ADF80C2004AA8DF8106088
S2144434E0CDE9007818F04EFF184A0623214602928A
S2144434F0284604AA05935B46ADF80C408DF8106048
S214443500CDE9007818F03EFF114B124A2146284672
S2144435108DF81060CDE90232082304AA05935B4671
S214443520CDE9007818F02EFF0A20FFF71EFC32463D
S2144435305146484623F01FFD09B0BDE8F08F00BF52
S214443540D47646001000500010019FFF1002C000C1
S2144435507102030405060708F100DA182DE9F04164
S2144435600446002855D16D201AF01CFE2246C04958
S2144435706D201AF016FE6E201AF014FE2246BD493F
S2144435806E201AF00EFE01220821BB4823F0F3FCFD
S21444359001220521B84823F0EEFCB84AB849204633
S2144435A018F082F90121204619F040F922460E21EE
S2144435B0204618F097FF204619F016F92346B14ADC
S2144435C00E21204618F0AEFA2346AF4A0E21204676
S2144435D018F0ECFAFEF7A5FE2046FFF7A7F9AB4B2A
S2144435E0012242F644015A5003F521531A6041F62B
S2144435F098700023A64A4443A648A35004441A4657
S214443600013384F871202834C82BF9D10020BDE852
S214443610F081012846D0022840F0898074209E4FCD
S2144436201AF0C0FD00229D4974201AF0BAFD752098
S2144436301AF0B8FD00229A4975201AF0B2FD01220C
S2144436400421984823F097FC01220621964823F04B
S21444365092FC0025954A20469549DFF8B88218F032
S21444366023F9204619F0C0F805F10E0658F835300F
S214443670904A0220F6B223F060430135314618F0F2
S21444368051FA3A46002331460220503718F08EFA53
S2144436900B2DE9D17D4B012246F204715A5003F5B5
S2144436A0CE43A3E77120844F1AF07CFD0022834961
S2144436B071201AF076FD72201AF074FD00228049BB
S2144436C072201AF06EFD22460721774823F053FCF9
S2144436D022460221734823F04EFC0025794A2046B0
S2144436E07949DFF8348218F0DFF8204619F07CF880
S2144436F005F11C0658F83530744A0120F6B223F01A
S21444370060430135314618F00DFA3A4600233146F7
S2144437100120503718F04AFA042DE9D144F2A47136
S2144437205A4B01225A5044F2A0715A505FE703287C
S21444373059D0042800F0F48005287FF458AF7B2045
S214443740634D1AF02FFD002262497B201AF029FDB2
S2144437507C201AF027FD00225F497C201AF021FDC8
S21444376001220E21504823F006FC01225B481146F4
S21444377023F001FC5A4A5B49204618F095F8204647
S21444378019F032F8012255492046FFF75BFE564AA7
S2144437905449204618F088F8204619F025F82B6836
S2144437A0524A0E2123F06043204618F0BBF900230A
S2144437B04F4A0E21204618F0F9F9AB684B4A0F21C0
S2144437C023F06043204618F0ADF90023494A0F2100
S2144437D0204618F0EBF94CF224512C4B01225A5057
S2144437E04CF22051A1E77720434F1AF0DBFC00222D
S2144437F0424977201AF0D5FC78201AF0D3FC0022F0
S2144438003F4978201AF0CDFC012200213D4823F0A0
S214443810B2FB01223B4800251146DFF8008123F025
S214443820AAFB394A3949204618F03EF8204618F093
S214443830DBFF05F10E0658F83530354A0320F6B25C
S21444384023F060430135314618F06CF93A460023BC
S21444385031460320503718F0A9F90A2DE9D148F229
S21444386064610A4B01225A5048F260615DE700BF2A
S214443870A5DF4500ABDF4500081729406C94460099
S21444388078414020342040201C4C40205C48412055
S214443890D0A64020408740201C604020EDDF4500F5
S2144438A0F3DF45000E1729400C172940BC93460009
S2144438B028384020542040207C5A4020CFDF450002
S2144438C0D5DF450014944600D03C40204420402098
S2144438D0F07946002FE0450035E0450010172940B2
S2144438E0DC764600302A4020B492460084204020AD
S2144438F01C7E40206C7E40201C6A40200BE0450025
S21444390011E0450006172940649346008033402062
S21444391064204020607A4600B87A4600107A460012
S2144439207920294D1AF03EFC0022284979201AF0C5
S21444393038FC7A201AF036FC002225497A201AF000
S21444394030FC01220A21234823F015FB01220921D9
S214443950204823F010FB204A2049204617F0A4FFB5
S214443960204618F041FF09221A492046FFF76AFD0F
S2144439701B4A1A49204617F097FF204618F034FF92
S2144439802B68184A0E2123F06043204618F0CAF8E4
S2144439900023154A0E21204618F008F9AB68114A50
S2144439A00F2123F06043204618F0BCF800230F4A4A
S2144439B00F21204618F0FAF84AF2C4510C4B012263
S2144439C05A504AF2C051B0E6007A46001DE045001F
S2144439D023E0450008172940DC764600D82E4020D0
S2144439E00C934600742040201C7440206C74402085
S2144439F05C4841200000000041F69872084B02FBE8
S214443A00003310B503EB8104E278A07800EB022083
S214443A10627802EB002213F8210000EB022010BD6E
S214443A204087402010B5094B41F6987404FB00309B
S214443A30130A00EB810181F8282081F82930130C01
S214443A40120E81F82A3081F82B2010BD4087402082
S214443A5013B502AB044603E9060041F69871094AD9
S214443A609DF8043001FB0022009903F03F0321F047
S214443A706041FEF78FFF204602B0BDE81040FEF7D7
S214443A8055BF00BF68874020FDF7F0BE70477047BB
S214443A907047704770477047704770477047704725
S214443AA07047074B074A196858799160197941EA73
S214443AB0002191819979DB799173D373704700BF64
S214443AC040874020C08340200C4A0D4810B55178AA
S214443AD0137801F00104C1F3410143EA042343EAA5
S214443AE041239178D27843EAC12343EAC2434269E8
S214443AF002F078421343436110BD00BF4087402024
S214443B00C0834020074B08491B7803F003021B0977
S214443B1003F0040313430A7C22F0070213430B7496
S214443B20704700BF40874020C08340200549064B6D
S214443B300A7E1B7822F01F0203F01F0313430B7602
S214443B40704700BFC0834020408740200549064B4D
S214443B500A7F1B7822F01F0203F01F0313430B77E0
S214443B60704700BFC0834020408740200649074B2B
S214443B7091F820201B7822F00F0203F00F03134322
S214443B8081F82030704700BFC083402040874020E3
S214443B90114B124810B55A78997802F003041B78F2
S214443BA043EA0423C2F3810443EA8423C2F30114A0
S214443BB0920943EA043343EA823301F00302C1F331
S214443BC0810143EA0243426A120D43EA81431205E5
S214443BD01343436210BD00BF40874020C08340204B
S214443BE00E4B0F4A5878197841EA002158791185C6
S214443BF0997801F00F0182F82A10D97882F82B10B0
S214443C00197941EA002191859979DB7901F00F0110
S214443C1082F82F3082F82E10704700BF408740202D
S214443C20C08340200E4B0F4A5878197841EA002149
S214443C3058791186997801F00F0182F83210D978B4
S214443C4082F83310197941EA002191869979DB7913
S214443C5001F00F0182F8373082F83610704700BF03
S214443C6040874020C08340200C4B0D4A5878197832
S214443C7041EA002158791187997801F00F0182F8BA
S214443C803A10197941EA002191879979DB7901F054
S214443C900F0182F83F3082F83E107047408740203C
S214443CA0C08340202D492E4A10B50B78487803F03F
S214443CB07F0343EAC013887843EAC033C87843EAAC
S214443CC0C053106C00F00040034348791364C0F3BB
S214443CD040040B79897982F8443000F001031B02D2
S214443CE043EA4423C0F3800443EA8423C0F3C00475
S214443CF043EAC423C0F3001443EA0433C0F3401435
S214443D0043EA4433C0F38014C00943EA843343EAA5
S214443D10C03301F0010043EA0043C1F3400043EAE4
S214443D204043C1F3800043EA8043C1F3C00043EA02
S214443D30C043C1F3001043EA0053C1F34010C1F33B
S214443D40801143EA405343EA8153516C21F4FF0106
S214443D5021F4FE410B43536410BD00BF408740200E
S214443D60C08340200D4A0E4810B55178137801F0B0
S214443D700F04C1F3001143EA042343EA0133917864
S214443D8043EA4133D17843EA4153816C01F06041C0
S214443D900B4383645368C36410BD00BF4087402010
S214443DA0C0834020034A044B1168526819655A651B
S214443DB0704700BF40874020C0834020244A25499E
S214443DC070B55578137805F003069078D47843EAAE
S214443DD00623C5F3810643EA8623C5F30116AD09D7
S214443DE043EA063343EA8533C0F3011543EA054301
S214443DF0850900F00F0043EA854304F0030543EACF
S214443E000553C4F3810543EA8553C4F30115A40955
S214443E1043EA056343EA84638C6D04F070442343A9
S214443E2054798B651379D27981F85C30230104F098
S214443E30030403F4706343EA0233CA6D43EA005052
S214443E40054B40EA046013401843C86570BD00BF84
S214443E5040874020C0834020FF0000FC70B5224DC0
S214443E60224A2C78E878C4F3401604F00F032979E4
S214443E7043EA0613C4F38016E40943EA461343EAC6
S214443E8084136C7843EAC413AC7843EAC43300F032
S214443E90030443EAC453C0F3810443EA4463C0F3CF
S214443EA00114800943EAC46343EA4073106E00F089
S214443EB00040034301F0030013668B0803F0040339
S214443EC00343880800F0080003438808C90900F043
S214443ED01000034343EA411392F8641021F03F0173
S214443EE00B4382F8643070BD40874020C083402036
S214443EF0114A124810B55178137801F0030443EA86
S214443F000423C1F3810443EA8423C1F301148909D9
S214443F1043EA043343EA8133A0F868305388A0F870
S214443F206A309388A0F86C30937980F86E30D379F1
S214443F3080F86F3010BD00BF40874020C0834020CB
S214443F40064B074A1968587911671979DB7941EAAB
S214443F50002182F87630A2F87410704740874020DB
S214443F60C0834020084A09491378907881F878300D
S214443F7053781843D378064A9B0443EA0023886F51
S214443F80024013438B67704740874020C0834020DD
S214443F90FF0000FC08B5054B18880BF0AFFC04493D
S214443FA00BF000FD034BD86708BD00BF4087402098
S214443FB0CDCCCC3DC0834020104B41F69871104A7E
S214443FC0595C82F8801041F69B71585C41F69A71B0
S214443FD0595C41EA0021A2F8811041F69D71585C73
S214443FE041F69C71595C41EA0021A2F8841041F6DE
S214443FF09F715B5C82F88630704700BF40874020E4
S214444000C0834020064A41F69871064B5158C3F87F
S214444010881041F69F71525C83F88C20704700BF2D
S21444402040874020C08340200C4A41F69F730C4989
S21444403010B541F69974D05C41F69873D35C125D22
S21444404002F0010243EA0223D1F89020520C43EADC
S214444050402352041343C1F8903010BD408740209B
S214444060C0834020284941F69973284A70B5C85CF5
S21444407041F69A73CD5C41F69B7300F00306CC5C24
S21444408041F69873CB5C43EA0623C0F3810643EAC1
S2144440908623C0F30116800943EA063343EA803395
S2144440A005F00300C5F3810543EA004304F003002A
S2144440B043EA854343EA0053C4F38100A40943EA30
S2144440C08053D2F8940043EA046300F07C400343F0
S2144440D041F69F70C2F8943041F69C73CB5C82F8EC
S2144440E0983041F69D73CB5C095C1B0203F47C5309
S2144440F043EA8133D2F8981021F47F1121F47C519D
S2144441000B43C2F8983070BD40874020C08340209F
S214444110214843F63073214930B5C35A5BBAA1F8F7
S2144441209C3043F63373C25C43F63273C2F30115D4
S214444130C45C930943EA850304F00F05240943EA63
S214444140051343F63675455DED0843EA0523C2F389
S214444150800543EA4533B1F89E5005F440452B4369
S214444160A1F89E3043F63473C55C43F63573C35C9E
S21444417043EA0523A1F8A030C2F3C003520143EA40
S214444180440302F060021A4391F8A23023F07F03FE
S2144441901A4381F8A22030BD40874020C083402087
S2144441A0164A43F63073164910B5D35A5BBAA1F88B
S2144441B0A43043F63273D05C43F63373D35C43EA9D
S2144441C00023A1F8A63043F63673D05C43F6347326
S2144441D0D45C43F63573D35C43EA042200F001030F
S2144441E0C0F3400043EA4203D1F8A820920C43EAC5
S2144441F0404392041343C1F8A83010BD4087402082
S214444200C0834020124A43F63071124B515A49BA81
S214444210A3F8AC1043F63271505C43F63371515CEC
S21444422041EA0021B3F8AE0061F30D0043F636715F
S214444230A3F8AE0043F63770515C125C42EA0122A2
S214444240B3F8B01062F30D01A3F8B010704700BF86
S21444425040874020C083402030B543F63073304C0E
S2144442603049E35A5BBAA1F8B43043F63673E05C9F
S21444427043F63773E25C43F63273E55C00F00303BF
S21444428043EA8503C0F3800543EA8523C2F38005E9
S21444429043EAC523850943EA0533B1F8B65005F425
S2144442A040452B43C2F3C005A1F8B63043F63373FA
S2144442B0E35C81F8B830C0F3C0031B0243EA4523ED
S2144442C002F0030543EA852343F63475655D43EA05
S2144442D00533C0F30015C0F3401043EA0553C2F358
S2144442E0001543EA45539509120943EA8553D1F824
S2144442F0B85002F0020225F47F05024325F47F45B8
S2144443002B43C1F8B83043F63573E35C81F8BB30D1
S21444431091F8BC3023F003031A4381F8BC2030BD27
S21444432040874020C0834020F0B543F63273404F68
S214444330404DFE5C43F63473F95C43F63373C6F380
S214444340801CF85C43F63573FC5C43F63673FA5CC3
S214444350F30943EA4C0343F6317C42EA042217F855
S2144443600CC043EA8C03C6F3401C43EA8C23C6F3D2
S214444370001C43EACC23C1F3400C43EA0C3343F617
S214444380307C17F80C7043EA4733C6F3C00743EA59
S2144443904753C6F3800743EA8753C0F3001743EAFC
S2144443A0C753470943EA0763C4F30117A40943EA1A
S2144443B0C763C6F3400706F0010643EA477343EA79
S2144443C08673D5F8C06006F00046334301F0010614
S2144443D0C5F8C030C2F30903C0F3C00243EA8623DB
S2144443E043EAC223C0F3800243EA0233C0F34002E6
S2144443F000F0010043EA4233C1F3C00243EA80338B
S21444440043EAC433C1F3001443EA44438C09C1F37A
S214444410800143EA844343EA025343EA4151D5F8D0
S214444420C4309B0D9B051943C5F8C410F0BD00BFAE
S21444443040874020C0834020284843F6307343F6E4
S21444444036722749F0B5C35A43F63275845C43F650
S21444445035725BBA455D825CA709A1F8C83043F65D
S214444460337347EA820743F63772C65C43F63473BF
S214444470825CC35CB009B1F8CAC042EA042240EA8E
S2144444808500C6F3810543EA0623C6F3011640EACF
S2144444908520144DC3F309030CEA050C43EA86232E
S2144444A040EA0C0043EA0733A1F8CA00C4F381008B
S2144444B0C4F3011443EA8053D1F8CC0000F07F40A3
S2144444C00343C1F8CC30C2F30903B1F8D02043EA21
S2144444D0842315402B43A1F8D030F0BD40874020BC
S2144444E0C083402000F0FFFF1D4943F630731D484B
S2144444F0F0B5CB5A43F632745BBA0E5DA0F8D430AE
S21444450043F63373CA5C43F63573CD5CC2F3810419
S21444451043F634732F09CB5C44EA870443F6367774
S21444452043EA0223C95D41EA052144EA8111A0F821
S214444530D610C3F30901C2F3001343EA41039109B9
S214444540C2F3401243EAC62343EAC16343EA4273D2
S214444550D0F8D82002F040421343C0F8D830F0BD1B
S21444456040874020C083402070B5234943F63674C4
S21444457043F6357543F630730C5D4E5DCB5AA5094C
S2144445801E485BBA45EA860543F63776A0F8DC3023
S21444459043F633738E5DCA5C43F6347346EA0424AA
S2144445A043F63276CB5C8E5D910943EA022341EAB8
S2144445B08601C2F38006C3F3090341EA8621B0F8B4
S2144445C0DE6006F478463143A0F8DE10C2F3C0013C
S2144445D043EA8123C2F30011520943EAC52343EA5E
S2144445E0415343EA8453C0F8E03090F8E43062F331
S2144445F0000380F8E43070BD40874020C0834020EC
S2144446001D4A43F630731D4870B5D35A5BBAA0F8BA
S214444610E83043F63273D45C43F63473D55C43F6E1
S2144446203373D15C2B09C5F3C00543EA011143F645
S2144446303673D65C43F63573D35CDB0043EA5612D6
S214444640C4F3400343EA450304F00105A40843EADF
S214444650850343EAC403B0F8EA4004F47E442343A3
S214444660A0F8EA3041EA0233D0F8EC20D20DD20565
S2144446701343C0F8EC3070BD40874020C0834020D0
S2144446801B4943F631731B4830B5CB5C80F8F03099
S21444469043F63273CA5C43F63573CD5C43F63473E3
S2144446A0CC5C43F63073C95C93091B0243EA81230E
S2144446B0C2F3401143EA8143C2F38001C2F3C0020D
S2144446C043EAC143D0F8F01043EA02532A0905F0FE
S2144446D00F0543EA4253084A43EA45630A401343F4
S2144446E0C0F8F030230943EA041480F8F44030BD9F
S2144446F040874020C0834020FF0000E0074943F63F
S2144447003073074ACB581BBAC2F8003143F63473A9
S214444710CB581BBAC2F80431704700BF40874020CC
S214444720C0834020214845F6C863214930B5C35A62
S2144447305BBAA1F8083145F6CB63C25C45F6CA635A
S214444740C2F30115C45C930943EA850304F00F05DC
S214444750240943EA051345F6CE65455DED0843EA6C
S2144447600523C2F3800543EA4533B1F80A5105F4FC
S21444477040452B43A1F80A3145F6CC63C55C45F663
S214444780CD63C35C43EA0523A1F80C31C2F3C003EE
S214444790520143EA440302F060021A4391F80E3190
S2144447A023F07F031A4381F80E2130BD4087402012
S2144447B0C0834020164A45F6C863164910B5D35AF6
S2144447C05BBAA1F8103145F6CA63D05C45F6CB63B4
S2144447D0D35C43EA0023A1F8123145F6CE63D05C9D
S2144447E045F6CC63D45C45F6CD63D35C43EA0422F9
S2144447F000F00103C0F3400043EA4203D1F8142119
S214444800920C43EA404392041343C1F8143110BD5A
S21444481040874020C0834020F0B545F6CA632D4FFC
S2144448202D4CFD5C45F6CC63F95C45F6CB63C5F38D
S214444830801CFE5C45F6CD63F85C45F6CE63FA5CB8
S214444840EB0943EA4C0345F6C96C42EA002217F8E2
S2144448500CC0C2F3090243EA8C03C5F3401C43EA86
S2144448608C23C5F3001C43EACC23C1F3400C43EA33
S2144448700C3345F6C86C17F80C7043EA4733C6F356
S2144448800017760943EA475343EA8653C0F30116B2
S214444890800943EA4663C5F3400605F0010543EA4A
S2144448A0C66343EA0573D4F8245105F060452B43A8
S2144448B0C4F8243101F0010342EA832242EAC020CC
S2144448C0C1F30012890940EA423040EA8131A4F833
S2144448D02811F0BD40874020C0834020284845F634
S2144448E0C86345F6CE622749F0B5C35A45F6CA654D
S2144448F0845C45F6CD625BBA455D825CA709A1F847
S2144449002C3145F6CB6347EA820745F6CF62C65C50
S21444491045F6CC63825CC35CB009B1F82EC142EA6A
S214444920042240EA8500C6F3810543EA0623C6F31B
S214444930011640EA8520144DC3F309030CEA050C1E
S21444494043EA862340EA0C0043EA0733A1F82E01E3
S214444950C4F38100C4F3011443EA8053D1F8300110
S21444496000F07F400343C1F83031C2F30903B1F885
S214444970342143EA842315402B43A1F83431F0BD57
S21444498040874020C083402000F0FFFF1D4945F685
S214444990C8631D48F0B5CB5A45F6CA645BBA0E5D8B
S2144449A0A0F8383145F6CB63CA5C45F6CD63CD5C9A
S2144449B0C2F3810445F6CC632F09CB5C44EA8704F2
S2144449C045F6CE6743EA0223C95D41EA052144EA37
S2144449D08111A0F83A11C3F30901C2F3001343EA64
S2144449E041039109C2F3401243EAC62343EAC14352
S2144449F043EA4253D0F83C21920D92051343C0F843
S214444A003C31F0BD40874020C0834020184845F6DE
S214444A10C863184930B5C35A5BBAA1F8403145F665
S214444A20CC63C55C45F6CA63C45C45F6CB63C35CDD
S214444A3043EA042245F6CD63E409C35CB1F8420177
S214444A4043EA0523ED09C3F3090343EA85230A4DE4
S214444A5028400343A1F84231C2F30903B1F8442184
S214444A6043EA84232A401343A1F8443130BD00BFAF
S214444A7040874020C083402000F8FFFF1D4A45F68B
S214444A80C8631D4870B5D35A5BBAA0F8483145F69A
S214444A90CA63D45C45F6CC63D55C45F6CB63D15C3F
S214444AA02B09C5F3C00543EA011145F6CE63D65C2F
S214444AB045F6CD63D35CDB0043EA5612C4F34003A9
S214444AC043EA450304F00105A40843EA850343EAA0
S214444AD0C403B0F84A4104F47E442343A0F84A3160
S214444AE041EA0233D0F84C21D20DD2051343C0F824
S214444AF04C3170BD40874020C08340201B4945F65A
S214444B00C9631B4830B5CB5C80F8503145F6CA6360
S214444B10CA5C45F6CD63CD5C45F6CC63CC5C45F6C5
S214444B20C863C95C93091B0243EA8123C2F380012C
S214444B3043EA8143C2F3C001C2F3401243EAC1438D
S214444B40D0F8501143EA02532A0905F00F0543EA08
S214444B504253084A43EA45630A401343C0F8503177
S214444B60230943EA041480F8544130BD408740206A
S214444B70C0834020FF0000E030B545F6C863304CA3
S214444B803049E35A5BBAA1F8183145F6CE63E05C87
S214444B9045F6CF63E25C45F6CA63E55C00F0030382
S214444BA043EA8503C0F3800543EA8523C2F38005C0
S214444BB043EAC523850943EA0533B1F81A5105F497
S214444BC040452B43C2F3C005A1F81A3145F6CB63E2
S214444BD0E35C81F81C31C0F3C0031B0243EA45235F
S214444BE002F0030543EA852345F6CC65655D43EA52
S214444BF00533C0F30015C0F3401043EA0553C2F32F
S214444C00001543EA45539509120943EA8553D1F8FA
S214444C101C5102F0020225F47F05024325F47F4529
S214444C202B43C1F81C3145F6CD63E35C81F81F3154
S214444C3091F8203123F003031A4381F8202130BD34
S214444C4040874020C0834020074945F6C863074A4A
S214444C50CB581BBAC2F8603145F6CC63CB581BBA66
S214444C60C2F86431704700BF40874020C08340206C
S214444C700C4947F664630C48CA5C47F66563CB5CEC
S214444C8043EA022247F66263CB5C03F00F0343EA2F
S214444C900213D0F86821120D12051343C0F8683188
S214444CA0704700BF40874020C0834020064A47F6EE
S214444CB06263D15C47F66363D35C044A43EA0123E8
S214444CC0A2F86C31704700BF40874020C083402024
S214444CD00C4949F6FC530C48CA5C49F6FD53CB5C78
S214444CE043EA022249F6FA53CB5C03F00F0343EA45
S214444CF00213D0F87021120D12051343C0F8703118
S214444D00704700BF40874020C0834020064A49F68B
S214444D10FA53D15C49F6FB53D35C044A43EA012375
S214444D20A2F87431704700BF40874020C0834020BB
S214444D3010B51B4C20890AF0E1FD1A490AF032FEF0
S214444D40194BA27B1860194B60891A600AF0D6FD8D
S214444D5017490AF027FE17490AF01AFD0AF074F9B3
S214444D600DA3D3E900230AF00FF80AF0BDFC124B5A
S214444D70124A1860E37BA08903F00F0313600AF01D
S214444D80BDFD0F490AF00EFE0AF0D2FF0D4B186027
S214444D9010BD00BFAFF30080C3F5285C8FC2D53F7B
S214444DA0C0834020CDCCCC3D981F4020801F40205F
S214444DB00AD7A33C00C023448C1F40207C1F4020BD
S214444DC0ACC52737841F4020104A1149137D03F091
S214444DD003000860C3F383000E499B0908600E492C
S214444DE00B60537D0D49C3F3410003F00103086093
S214444DF00B490B6053690B49C3F3C7230B60D38A33
S214444E00094AC3F3C7031360704700BFC0834020FA
S214444E106C1F4020681F4020641F40205C1F4020B9
S214444E20601F4020501F4020581F4020074B084A10
S214444E301B7CC3F300011170C3F34001054AC3F35E
S214444E4080031170044A1370704700BFC08340202B
S214444E504E1F40204D1F40204C1F4020FFF7E6BF0A
S214444E6008B5FFF7E3FFBDE80840FCF7FDBC174A6A
S214444E70174992F8243003F003000860C3F3810016
S214444E8014490860C3F3011013499B090860134989
S214444E900B6092F82530124903F003000860C3F310
S214444EA0810010490860C3F301100F499B0908604C
S214444EB00E490B6092F826300D4A03F00301C3F303
S214444EC0810311600B4A1360704700BFC0834020C3
S214444ED0781A4020741A4020701A40206C1A4020D9
S214444EE0681A4020641A4020601A40205C1A402009
S214444EF0581A4020541A402010B5194C208D0AF0F8
S214444F00FDFC18490AF04EFD17490AF041FC174BC0
S214444F10174A186094F82A30A08D03F00F011B0935
S214444F201160144A136094F82B30134A323B1360D2
S214444F300AF0E4FC11490AF035FD11490AF028FC50
S214444F40104B114A186094F82E3003F00F011B09D9
S214444F5011600E4A136094F82F200D4B1A6010BD52
S214444F60C08340200AD7A33B0AD72343481F402088
S214444F70441F4020401F40203C1F40200AD7A33AED
S214444F80F8D32342381F4020341F4020301F40208F
S214444F902C1F402010B5194C208E0AF0AFFC18493F
S214444FA00AF000FD17490AF0F3FB174B174A18603E
S214444FB094F83230A08E03F00F011B091160144A96
S214444FC0136094F83320134B1A600AF097FC124986
S214444FD00AF0E8FC11490AF0DBFB114B114A186051
S214444FE094F8363003F00F011B0911600E4A136023
S214444FF094F837200D4B1A6010BD00BFC083402084
S2144450000AD7A33B0AD72343281F4020241F402007
S214445010201F40201C1F40200AD7A33AF8D323421F
S214445020181F4020141F4020101F40200C1F4020F3
S21444503010B5174C208F0AF061FC16490AF0B2FCF2
S21444504015490AF0A5FB154B154A186094F83A30F2
S214445050A08F03F00F011B091160124A13600AF077
S2144450604DFC11490AF09EFC10490AF091FB104B86
S214445070104A186094F83E3003F00F011B09116083
S2144450800D4A136094F83F200C4B1A6010BD00BFC5
S214445090C08340200AD7A33B0AD72343081F402097
S2144450A0041F4020001F40200AD7A33AF8D32342C7
S2144450B0FC1E4020F81E4020F41E4020F01E4020D7
S2144450C010B53E4C3E4A94F84030B4F8400003F0E5
S2144450D00101C0F3C7101160C3F34001394A11609F
S2144450E0C3F38201384AC3F341131160374A13604D
S2144450F00AF004FC36490AF055FC0AF019FE354B12
S2144451001860206CC0F3C7300AF0F8FB30490AF048
S21444511049FC0AF00DFE304B1860B4F84200C0F368
S214445120C7100AF0EBFB2D490AF032FB0AF000FEEA
S2144451302B4B94F8442018602A4B1A6094F8453058
S214445140294A03F001011160C3F34001274A116064
S214445150C3F38001264A1160C3F3C001254A116097
S214445160C3F30011244A1160C3F34011234A11606B
S214445170C3F38011224ADB091160224A136094F873
S2144451804630214A03F001011160C3F340011F4A2F
S2144451901160C3F380011E4A1160C3F3C0011D4A67
S2144451A01160C3F300111C4A1160C3F340111B4A3B
S2144451B0C3F3801311601A4A136010BDC0834020A5
S2144451C0EC1E4020E81E4020E41E4020E01E402006
S2144451D00AD7233CDC1E4020D81E40200000204234
S2144451E0D41E4020D01E4020CC1E4020C81E402046
S2144451F0C41E4020C01E4020BC1E4020B81E402076
S214445200B41E4020B01E4020AC1E4020A81E4020A5
S214445210A41E4020A01E40209C1E4020981E4020D5
S214445220941E402038B5264D264B95F8484004F049
S2144452300102C4F302101A60C4F34002224B1A60FF
S214445240C4F38002214B1A60C4F3C002204BE40925
S2144452501A600AF04FFB1F4B1F4A18601F4BA86C7E
S2144452601C6095F84930C0F3473003F00F01C3F390
S2144452700013323811601A4A13600AF03FFB194B88
S2144452801860B5F84A00C0F3471032380AF036FBC7
S214445290154B1860B5F84C00A0F500400AF02EFBFC
S2144452A0124B1860B5F84E000AF028FB10490AF075
S2144452B079FB10490AF06CFA0F4B186038BD00BFF2
S2144452C0C0834020901E40208C1E4020881E4020D4
S2144452D0841E4020801E4020781E40207C1E402095
S2144452E0741E4020701E40206C1E4020681E4020C5
S2144452F00AD7233C00004843641E40207047304B86
S214445300304A10B593F85940C4F381011170C4F380
S21444531001112D4A1170C4F301012C4AA4091170DD
S21444532093F858202A49C2F381100870C2F301103A
S21444533028490870C2F381002749C2F30102087065
S21444534026490A7093F85D202549C2F38100C2F3CA
S2144453500102087023490A7093F85E202249C2F37A
S21444536003120A7093F85F202049C2F301020A70C0
S21444537093F85A201E4902F003000860C2F38100E5
S2144453801C490860C2F301101B49920908601B4976
S2144453900A6093F85B201A4902F00300C2F38102C4
S2144453A00860184993F85C000A700AF0A7FA164990
S2144453B00AF0F8FA154B1860154B1C6010BD00BF78
S2144453C0C0834020601E40205F1E40205E1E40205A
S2144453D05D1E40205C1E40205B1E40205A1E40201E
S2144453E0591E4020581E40206C184020201E402045
S2144453F0501E40204C1E4020481E4020441E402044
S214445400401E402065184020CDCCCC3D381E402060
S214445410541E4020264A274992F8603003F007007D
S2144454200860C3F3C00024490860C3F3001023494E
S2144454300870C3F340102249C3F38013087021490F
S2144454400B70B2F860302049C3F3C7130B60136E79
S2144454501E49C3F3C7330B60B2F862301C49C3F32A
S214445460C1130B6092F863301A49C3F341000860D5
S214445470C3F3C1001849C3F34113086017490B60CE
S21444548092F86430164A03F003011160C3F38001B6
S214445490144A1160C3F3C001134A1160C3F30011E8
S2144454A0124AC3F340131160114A1360704700BF99
S2144454B0C08340201C1E4020181E4020161E40203C
S2144454C0151E4020141E4020101E40200C1E402056
S2144454D0081E4020041E4020001E4020FC1D402084
S2144454E0F81D4020F41D4020F01D4020EC1D4020B7
S2144454F0E81D402010B5194C194A94F8683094F8C1
S2144455006A00C3F38101C3F301131170154A137083
S21444551094F86930144AC3F301011170C3F381014E
S214445520124AC3F381131170114A13700AF0E2F958
S214445530104B186094F86B000AF0DCF90E4B94F8A4
S2144455406C2018600D4B1A7094F86D200C4B1A7032
S21444555094F86E200B4B1A7010BD00BFC0834020D9
S214445560DE1D4020CD1D4020DD1D4020CC1D4020AA
S214445570DC1D4020D81D4020D41D4020D01D402096
S214445580CF1D4020CE1D402010B50C4CB4F8720000
S2144455900AF0B4F90A490AF005FA0A4B1860B4F856
S2144455A070000AF0ABF906490AF0FCF9064BB4F869
S2144455B074201860054B1A8010BD00BFC08340207D
S2144455C0CDCCCC3DC81D4020C41D4020C21D40202B
S2144455D0054A0649B2F87A3092F87820C3F387032E
S2144455E00B70034B1A707047C0834020C11D402087
S2144455F0C01D402010B5124C124B94F88020B4F8CD
S21444560081001A600AF07AF90F490AF0CBF90F497B
S2144456100AF0BEF80E4B1860B4F884000AF06EF92F
S2144456200C490AF0BFF90C4B0C4A186094F88630C3
S21444563003F00F011B091160094A136010BD00BF37
S214445640C0834020BC1D4020ACC52737ACC5A73E10
S214445650B81D4020CDCCCC3DB41D4020B01D4020CC
S214445660AC1D402010B5114CB4F888000AF046F939
S2144456700F490AF097F90F490AF08AF80E4B18605A
S214445680B4F88A000AF03AF909490AF08BF909494C
S2144456900AF07EF8094B0A4A186094F88C3003F0F6
S2144456A00F011B091160074A136010BDC0834020D8
S2144456B00AD7A33C00C02344A81D4020A41D402074
S2144456C0A01D40209C1D4020114A124992F890305B
S2144456D003F003000860C3F381000F490860C3F376
S2144456E001100E499B0908600D490B6092F89130F1
S2144456F00C4903F00100C3F3430308600A490B60F6
S214445700D2F89030094AC3F343331360704700BF5E
S214445710C0834020981D4020941D4020901D40206A
S2144457208C1D4020881D4020841D4020801D402024
S2144457301B4B1C4A1B685BBB92F894301A4903F017
S21444574003000860C3F3810018490860C3F30110DE
S21444575017499B09086017490B6092F8953016491B
S21444576003F003000860C3F3810014490860C3F3E0
S214445770011013499B09086012490B6092F8963051
S214445780114903F00300C3F3810308600F490B601B
S214445790D2F898300E4AC3F383331360704700BF81
S2144457A0541C4020C08340207C1D4020781D40204F
S2144457B0741D4020701D40206C1D4020681D4020F4
S2144457C0641D4020601D40205C1D4020581D402024
S2144457D0541D402010B50E4C0E4B94F89F0094F880
S2144457E09C2000F01F001A6000EB80000AF086F848
S2144457F0094B1860B4F8A0000AF080F807490AF08C
S214445800D1F8074909F0C4FF064B186010BD00BF25
S214445810C0834020501D4020381D4020CDCC4C3DF8
S21444582000C0CC44341D402010B50C4CB4F8A6003F
S2144458300AF064F80A490AF0B5F80A4909F0A8FFDC
S214445840094B1860D4F8A800C0F34F00A0F5FF40F9
S2144458507F380AF053F8054B186010BDC0834020CB
S2144458600AD7A33C00C02344241D40201C1D4020CE
S21444587010B50D4CB4F8AE00C0F30D000AF03EF877
S2144458804FF07A510AF08EF8084B1860B4F8B0001E
S214445890C0F30D000AF032F84FF07A510AF082F85D
S2144458A0034B186010BD00BFC0834020141D402029
S2144458B0101D402070470B4A0B49B2F8C40008B587
S2144458C0B2F8C030C0F30900C3F387030B700AF084
S2144458D015F806490AF066F8054909F059FF054BDC
S2144458E0186008BDC08340200C1D4020CDCCCC3D64
S2144458F09A994C42081D402010B5174CB4F8CA007B
S214445900C0F3090009F0FAFF14490AF04BF8144BA7
S2144459101860B4F8CC00C0F3090009F0EFFF0F4953
S2144459200AF040F80F4B1860D4F8CC00C0F30930A6
S21444593009F0E4FF09490AF035F80B4B1860B4F84F
S214445940D000C0F3090009F0D9FF04490AF02AF848
S214445950064B186010BD00BFC0834020CDCCCC3D64
S214445960041D4020001D4020FC1C4020F81C402004
S21444597038B5144DB5F8D600800909F0BFFF124972
S2144459800AF010F8114909F003FFB5F8D840104B57
S214445990C4F349041860204609F0B0FF0D490AF0E4
S2144459A001F80D4B1860D5F8D800C0F3CF2009F0A5
S2144459B0A5FF0A4909F0F6FF094B1860094B1C601D
S2144459C038BD00BFC0834020CDCC4C3D6666724196
S2144459D0F41C40209A99193EF01C40200AD7233CD8
S2144459E0EC1C4020781C402010B5164CB4F8DE0061
S2144459F0C0F3090009F082FF134909F0D3FF134BA3
S214445A001860B4F8E000C0F3090009F077FF0E49C7
S214445A1009F0C8FF0E4B1860D4F8E000C0F3C92064
S214445A2009F06CFF084909F0BDFF0A4B1860B4F84A
S214445A30E200800909F062FF034909F0B3FF064B10
S214445A40186010BDC08340209A99193EE81C402037
S214445A50E41C4020E01C4020DC1C402010B5134CC5
S214445A60B4F8EA00C0F3C50009F048FF104909F04D
S214445A7099FF104909F08CFE0F4B1860B4F8EC00FF
S214445A80C0F30B0009F03AFF0C4909F08BFF0C4BAE
S214445A901860D4F8EC00C0F30A3009F02FFF04492C
S214445AA009F080FF074B186010BD00BFC08340203C
S214445AB0CDCCCC3DCDCC4C40D81C40200AD7233C42
S214445AC0D41C4020D01C40207047704710B50E4C64
S214445AD00E4B94F80B0194F8082100F01F001A604E
S214445AE000EB800009F00AFF094B1860B4F80C017B
S214445AF009F004FF074909F055FF074909F048FE35
S214445B00064B186010BD00BFC0834020CC1C40200C
S214445B10C81C4020CDCC4C3D00C0CC44C41C4020C6
S214445B2010B50C4CB4F8120109F0E8FE0A4909F025
S214445B3039FF0A4909F02CFE094B1860D4F81401C1
S214445B40C0F34F00A0F5FF407F3809F0D7FE054B61
S214445B50186010BDC08340200AD7A33C00C023442D
S214445B60C01C4020BC1C402070470B4A0B49B2F86E
S214445B70280108B5B2F82431C0F30900C3F38703FB
S214445B800B7009F0BBFE064909F00CFF054909F005
S214445B90FFFD054B186008BDC0834020981C40207C
S214445BA0CDCCCC3D9A994C42941C402010B5174C11
S214445BB0B4F82E01C0F3090009F0A0FE144909F018
S214445BC0F1FE144B1860B4F83001C0F3090009F034
S214445BD095FE0F4909F0E6FE0F4B1860D4F83001E5
S214445BE0C0F3093009F08AFE094909F0DBFE0B4B85
S214445BF01860B4F83401C0F3090009F07FFE044984
S214445C0009F0D0FE064B186010BD00BFC08340208C
S214445C10CDCCCC3D901C40208C1C4020881C402081
S214445C20841C402010B5134CB4F83A01800909F09E
S214445C3065FE114909F0B6FE104909F0A9FD104B5E
S214445C401860B4F83C01C0F3490009F057FE0D490A
S214445C5009F0A8FE0AF06CF80B4B1860D4F83C0127
S214445C60C0F3C72009F04AFE084909F09BFE084BDA
S214445C70186010BDC0834020CDCC4C3D6666724152
S214445C80B81C40209A99193EB01C40200AD7233CA1
S214445C90B41C402010B50C4CB4F84201C0F30900C3
S214445CA009F02CFE094909F07DFE094B1860B4F84A
S214445CB04401C0F3090009F021FE044909F072FECC
S214445CC0044B186010BD00BFC08340209A99193E0B
S214445CD0AC1C4020A81C402008B5FFF729F8FFF765
S214445CE073F8FFF7C4F8FFF7EBF9FFF79BFAFFF7F3
S214445CF006FBFFF78FFBFFF7FDFBFFF745FCFFF7BF
S214445D0067FCFFF7F9F8FFF745F9FFF791F9FFF756
S214445D1071FCFFF7A7FCFFF7D7FCFFF709FDFFF779
S214445D20EBFDFFF725FEFFF75FFEFFF73FFFFFF7AC
S214445D3079FFBDE80840FFF7ADBF10B5124CB4F884
S214445D404A01C0F3C50009F0D9FD104909F02AFEFE
S214445D500F4909F01DFD0F4B1860B4F84C01C0F311
S214445D600B0009F0CBFD0C4909F01CFE0B4B1860E8
S214445D70D4F84C01C0F30A3009F0C0FD034909F0D9
S214445D8011FE074B186010BDC0834020CDCCCC3DDF
S214445D90CDCC4C40A41C40200AD7233CA01C402019
S214445DA09C1C402008B5FFF759FEBDE80840FFF7A5
S214445DB0C4BF7047704708B5084BD3F86801C0F3B2
S214445DC00F1009F09BFD064909F0ECFD054909F062
S214445DD0DFFC09F0ADFF044B186008BDC0834020CB
S214445DE0CDCC4C3D00C0CC44C01B402008B5084B2D
S214445DF0B3F86C0109F082FD064909F0D3FD064963
S214445E0009F0C6FC09F094FF044B186008BD00BFB7
S214445E10C08340200AD7A33C00C02344C41B402070
S214445E2008B5094BD3F87001C0F30F1009F066FDAE
S214445E30064909F0B7FD064909F0AAFC09F078FFBF
S214445E40044B186008BD00BFC0834020CDCC4C3DF9
S214445E5000C0CC44B41B402008B5084BB3F87401CA
S214445E6009F04CFD064909F09DFD064909F090FCF1
S214445E7009F05EFF044B186008BD00BFC083402095
S214445E800AD7A33C00C02344B41B402008B5FFF700
S214445E90A1FCFFF7C9FCFFF7EBFCFFF70CFDFFF78F
S214445EA015FEFFF73DFEFFF760FEFFF784FFFFF7A2
S214445EB09DFFFFF7B5FFBDE80840FFF7CDBF1A4B7F
S214445EC0186810B5C830194C09F014FD184909F083
S214445ED01DFE09F0B9F80EF0BFF809F0E5FB154BC6
S214445EE01549A4F87801186809F054FC134909F0D8
S214445EF00DFE09F0A9F80EF0AFF809F0D5FB104BEB
S214445F00A4F87A011B68A4F87C310E4B186809F093
S214445F109BF80EF0A1F809F0C7FB0B4B84F87E0102
S214445F201B6884F87F3110BD801C4020C08340200D
S214445F30CDCCCC3D7C1C402000C023440AD7A33C97
S214445F40781C4020741C4020701C4020224B234A5E
S214445F501B78234982F88431224B09681B6809025E
S214445F609B0201F4407103F480630B431E490968A5
S214445F70C90201F4C0510B431C490968490301F4A2
S214445F80C0410B431A490968C90301F4C0310B43A5
S214445F90D2F8841121F4FF3121F480710B43154962
S214445FA0C2F88431144B09681B6801F00701A2F853
S214445FB08A31124B1B68A2F88831114B1B78DB00E0
S214445FC003F008030B4392F88C1121F00F010B43A6
S214445FD082F88C31704700BFCE1D4020C0834020DD
S214445FE0601C40205C1C4020581C4020541C402010
S214445FF0501C40201C1E40204C1C4020481C402066
S214446000161E4020184B1949186810B509F07EFD35
S214446010174C09F019F80EF01FF809F045FB154B1C
S2144460201249A4F89001186809F070FD09F00CF8BC
S2144460300EF012F809F038FB0F4B0C49A4F8920105
S214446040186809F063FD08F0FFFF0EF005F809F044
S2144460502BFB0A4BA4F894011B7884F89731084B21
S2144460601B7884F8963110BDC41D4020CDCCCC3D61
S214446070C0834020C81D4020381E4020C11D4020FB
S214446080C01D4020174B184A1B7812785B0002F05C
S214446090010203F002031343144A1278920002F0FA
S2144460A004021343124A1278D20002F00802134341
S2144460B0104A1278120102F0100213430E4A127864
S2144460C0520102F0200213430C4A1278920102F065
S2144460D0400213430A4A127843EAC213094A82F832
S2144460E0E8317047251C4020261C4020241C4020B4
S2144460F0231C4020221C4020211C4020201C4020E1
S21444610078174020C083402038B51A4B1A4C19687B
S2144461101A4B186809F03EFB194B0546194918688E
S21444612009F038FB184909F0F1FC08F08DFF0DF032
S21444613093FF09F0B9FA154B1549A4F8EC01186811
S21444614009F028FB134909F0E1FC08F07DFF0DF047
S21444615083FF09F0A9FA1049A4F8EE01284609F08D
S214446160D5FC08F071FF0DF077FF09F09DFAA4F80E
S214446170F00138BD9C174020C0834020981F402023
S214446180A0174020000048430AD7233C98174020D5
S21444619000C023440AD7A33CCDCCCC3D1C4B1D4960
S2144461A0186810B509F0B2FC1B4C08F04DFF0DF012
S2144461B053FF09F079FA194BA4F89801186808F0C7
S2144461C043FF0DF049FF09F06FFA154B1549A4F843
S2144461D09A01186809F0DEFA134909F097FC08F0AA
S2144461E033FF0DF039FF09F05FFA104B1049A4F85D
S2144461F09C01186809F0CEFA0E4909F087FC08F0AD
S21444620023FF0DF029FF09F04FFAA4F89E0110BDB4
S214446210901F4020CDCCCC3DC0834020B4194020B4
S214446220A018402000C023440AD7A33C581B402053
S214446230000048430AD7233C114B1249186810B54E
S21444624009F064FC104C08F0FFFE0DF005FF09F061
S2144462502BFA0E4B0E491B78A4F8A001A4F8A231E1
S2144462600C4B186809F096FA0B4909F04FFC08F0F5
S214446270EBFE0DF0F1FE09F017FAA4F8A40110BDE8
S21444628004194020CDCCCC3DC08340200E1940207C
S21444629000C02344881840200AD7A33C184B194909
S2144462A0186810B509F076FA174909F02FFC174C10
S2144462B008F0CAFE0DF0D0FE09F0F6F9144B154965
S2144462C0A4F8A801186809F065FA134909F01EFCF9
S2144462D008F0BAFE0DF0C0FE09F0E6F90F4BA4F83C
S2144462E0AA011B6884F8AC310D4B1A680D4B1B6829
S2144462F003F00F0343EA021384F8AD3110BD00BF28
S214446300241D402000C023440AD7A33CC083402019
S214446310341D402000C0CC44CDCC4C3D281C4020ED
S214446320D81B4020DC1B4020164B1749186810B574
S21444633009F030FA154909F0E9FB154C08F084FEDB
S2144463400DF08AFE09F0B0F9124B1349A4F8B001D7
S214446350186809F01FFA114909F0D8FB08F074FED2
S2144463600DF07AFE09F0A0F90D4BA4F8B2011A68B4
S2144463700C4B1B6803F00F0343EA021384F8B43152
S21444638010BD00BFC01C402000C023440AD7A33C15
S214446390C0834020C41C402000C0CC44CDCC4C3DDF
S2144463A0C81B4020CC1B4020174B186810B500F281
S2144463B08F20164C09F09EFA154909F0A7FB08F001
S2144463C043FE0DF049FE09F06FF9124BA4F8B801EC
S2144463D0186800F2666009F08DFA0F4909F096FBDA
S2144463E008F032FE0DF038FE09F05EF90B4BA4F8C7
S2144463F0BA011A680A4B1B6803F00F0343EA0213F8
S21444640084F8BC3110BD00BFC41B4020C08340206C
S2144464100AD7A33CC01B4020CDCC4C3DB81B4020E3
S214446420BC1B4020174B186810B500F28F20164C42
S21444643009F060FA154909F069FB08F005FE0DF00D
S2144464400BFE09F031F9124BA4F8C001186800F2AB
S214446450666009F04FFA0F4909F058FB08F0F4FD5E
S2144464600DF0FAFD09F020F90B4BA4F8C2011A68A6
S2144464700A4B1B6803F00F0343EA021384F8C43143
S21444648010BD00BFB41B4020C08340200AD7A33CA5
S214446490B01B4020CDCC4C3DA81B4020AC1B40201C
S2144464A00A4A0B4B126883F8E0210A4A126883F8BA
S2144464B0E121094A126883F8E221084A126883F8FF
S2144464C0E321074A1268C3F8E4217047A41B40201E
S2144464D0C0834020A01B40209C1B4020981B40208B
S2144464E0941B40204D4B4E4A1B68012B5BD14D4BB1
S2144464F04D491B6809689B0001F0030103F00C0337
S2144465000B434A490968090101F030010B434849E5
S21444651009688901C9B20B4346490968090201F46E
S21444652040710B4344490968890201F440610B43B6
S21444653042490968090301F440510B43404909683C
S214446540890389B20B433F490968090401F4403181
S2144465500B433D490968890401F440210B43D2F8B2
S214446560C811090D09050B43C2F8C831374B1B78CF
S21444657003F00301364B1B7803F003031B0143EA85
S21444658081133449097801F0030143EA0123B2F840
S214446590CA1121F47C710B43A2F8CA312E4B1B88D6
S2144465A082F8CC317047002B33D12C4B2C491B68D6
S2144465B009689B0001F0030103F00C030B432949CF
S2144465C00968090101F030010B432749096889012C
S2144465D0C9B20B4325490968090201F440710B43CB
S2144465E023490968890201F440610B43214909683B
S2144465F0090301F440510B431F490968890389B2D2
S2144466000B431E490968090401F440310B431C49F5
S214446610A0E7023B012BA9D8C7E700BF541C402083
S214446620C0834020741A4020781A4020701A4020B4
S2144466306C1A4020681A4020641A4020601A402091
S2144466405C1A4020581A4020541A4020271B4020E9
S214446650261B4020281B4020241B4020781D402019
S2144466607C1D4020741D4020701D40206C1D402021
S214446670681D4020641D4020601D40205C1D402055
S214446680581D4020124B13491B7803F00302124B4B
S2144466901B7803F0030343EA8203104A127802F09D
S2144466A0030243EA02130E4A127802F0030243EA54
S2144466B082130C4A127802F0030243EA0223B1F82A
S2144466C0D02102F47C421343A1F8D031704700BF76
S2144466D0671B4020C0834020681B4020661B402028
S2144466E0651B4020641B4020094B0A491A680A4B24
S2144466F002F001021B6803F0030343EA820391F8A5
S214446700DC2122F00702134381F8DC31704700BFD6
S2144467105C1B4020C0834020601B402038B5344B6F
S214446720344D1868C83009F0E5F8334909F0EEF9F5
S21444673008F08AFC0DF090FC304B1C68304B64002B
S2144467401B6804F0020403F001031C432D4B1B6832
S2144467509B0003F004031C432B4B1B68DB0003F035
S21444676008031C43294B1B681B01DBB21C43284B04
S2144467701B681B0203F440731C43264B1B689B0296
S21444678003F4E0531C43244B1B685B0303F4C043ED
S2144467901C4308F089FF214B214903EAC0331C43BC
S2144467A0D5F8D43103F000431C431E4BC5F8D441FE
S2144467B0186808F0EFFF104909F0A8F908F044FCFF
S2144467C00DF04AFC08F070FF174B1549A5F8D801A0
S2144467D0186808F0DFFF084909F098F908F034FC17
S2144467E00DF03AFC08F060FFA5F8DA0138BD00BFAA
S2144467F0301B4020C08340200AD7233C4C1B4020FB
S214446800501B4020481B4020441B4020401B402037
S2144468103C1B4020381B4020341B40200080FF7F18
S214446820000048432C1B4020581B4020274B284937
S214446830186810B508F0AEFF264909F067F9264CEB
S21444684008F002FC0DF008FC08F02EFF234B244908
S214446850A4F84802186808F09DFF224909F056F942
S21444686008F0F2FB0DF0F8FB08F01EFF1E4BA4F8F0
S2144468704A021B68A4F84C321C4B1A681C4B02F0A4
S21444688003021B6803F0010343EA4203194A1268F1
S21444689002F0030243EAC203174A126802F00102F6
S2144468A043EA4213154A126802F00F0243EA82137F
S2144468B0134A126802F00F0243EA8223B4F84E22C7
S2144468C002F440421343A4F84E3210BD641E4020E6
S2144468D0000048430AD7233CC0834020241D402060
S2144468E000C023440AD7A33C181B4020581C402011
S2144468F0101B4020501C4020041B4020001B4020FE
S214446900FC1A4020244B4FF08E41244A1B681268E0
S2144469101B0102F00F02DBB21343214A1268120233
S21444692002F4706213431F4A1268120302F4805240
S21444693013431D4A1268520302F4C04213431B4ACF
S2144469401268D20302F4C0321343194A126852043E
S21444695010B502F0FF72174C1343D4F8502202F0DD
S2144469607E421343C4F85032134B186808F012FFA3
S21444697008F06AFB0DF070FB08F096FE0F4BA4F887
S21444698054021A680E4B1B6803F00F0343EA0213C3
S21444699084F8563210BD00BFF41A4020F81A40203E
S2144469A0F01A4020EC1A4020541C4020E41A4020A0
S2144469B0101E4020C0834020681E4020DC1A402021
S2144469C0E01A4020114B10B5186808F03DFB104CF7
S2144469D00DF042FB08F068FE0E4B84F858021B6824
S2144469E084F859320C4B1B68A4F85A320B4B1B687C
S2144469F0A4F85C320A4B1A680A4B1B6803F00F0370
S214446A0043EA021384F85E3210BD00BF741C402073
S214446A10C0834020701C4020481C40204C1C402012
S214446A20C41A4020C81A40201C4A936CC3F3473308
S214446A3082F89032B2F84A30C3F3471382F8913260
S214446A40B2F84230C3F3C71382F8923292F85C30FD
S214446A5082F89332124B1968124B01F007011B68F7
S214446A6003F0010343EA41030F49097801F00101A9
S214446A7043EA01130D49096801F00F0143EA411343
S214446A800B49096801F00F0143EA4123B2F8941216
S214446A9001F460410B43A2F894327047C08340200F
S214446AA01C1E4020E81D4020161E4020C01A4020D0
S214446AB0BC1A4020FFF7B8BF174B184A1B78127809
S214446AC05B0002F0010203F002031343144A1278F7
S214446AD0920002F004021343124A1278D20002F0E3
S214446AE008021343104A1278120102F010021343AC
S214446AF00E4A1278520102F0200213430C4A1278CE
S214446B00920102F0400213430A4A127843EAC2133F
S214446B10094A82F898327047251C4020261C40209B
S214446B20241C4020231C4020221C4020211C4020A2
S214446B30201C402078174020C0834020174B1868FC
S214446B4010B500F28F20164C08F0D4FE154908F014
S214446B50DDFF08F079FA0DF07FFA08F0A5FD124B38
S214446B60A4F82802186800F2666008F0C3FE0F49CD
S214446B7008F0CCFF08F068FA0DF06EFA08F094FDC1
S214446B800B4BA4F82A021A680A4B1B6803F00F033F
S214446B9043EA021384F82C3210BD00BFB81A4020D2
S214446BA0C08340200AD7A33CB41A4020CDCC4C3DE9
S214446BB0AC1A4020B01A4020174B186810B500F2A3
S214446BC08F20164C08F096FE154908F09FFF08F0F3
S214446BD03BFA0DF041FA08F067FD124BA4F8300278
S214446BE0186800F2666008F085FE0F4908F08EFFCC
S214446BF008F02AFA0DF030FA08F056FD0B4BA4F8CC
S214446C0032021A680A4B1B6803F00F0343EA021366
S214446C1084F8343210BD00BFA81A4020C0834020F8
S214446C200AD7A33CA41A4020CDCC4C3D9C1A402005
S214446C30A01A4020174B186810B500F28F20164C47
S214446C4008F058FE154908F061FF08F0FDF90DF00C
S214446C5003FA08F029FD124BA4F83802186800F22B
S214446C60666008F047FE0F4908F050FF08F0ECF95C
S214446C700DF0F2F908F018FD0B4BA4F83A021A6826
S214446C800A4B1B6803F00F0343EA021384F83C32B2
S214446C9010BD00BF981A4020C08340200AD7A33CAA
S214446CA0941A4020CDCC4C3D8C1A4020901A40205B
S214446CB0174B186810B500F28F20164C08F01AFED1
S214446CC0154908F023FF08F0BFF90DF0C5F908F0A0
S214446CD0EBFC124BA4F84002186800F2666008F019
S214446CE009FE0F4908F012FF08F0AEF90DF0B4F9AA
S214446CF008F0DAFC0B4BA4F842021A680A4B1B68ED
S214446D0003F00F0343EA021384F8443210BD00BF75
S214446D10881A4020C08340200AD7A33C841A4020C7
S214446D20CDCC4C3D7C1A4020801A40204C4B4FF032
S214446D3084412DE9F04FDFF864A187B01B788AF8C8
S214446D40BC32484B1B788AF8BD32474B186808F06B
S214446D5021FD4FF0834108F025FE08F075F90DF04B
S214446D607BF9424B8046894618684FF0844108F0C8
S214446D7011FD4FF0834108F015FE08F065F90DF05B
S214446D806BF93B4B06460F4693F800B0394B3A49ED
S214446D900BF0010B186808F0FDFC384908F0B6FE05
S214446DA008F052F90DF058F9354B364A1B78CDE9C0
S214446DB0000110683449059308F0ECFC334908F0A8
S214446DC0A5FE08F041F90DF047F9314A1478314AE6
S214446DD004F001041578240305F00105CDE9020109
S214446DE04946404608F060FCC0F30900AD02394607
S214446DF00543BAF8BE0200F4784005433046AAF884
S214446E00BE524FEA8B2508F04FFCC0F3090BDDE970
S214446E10000108F049FC204A059B45EA0B0B02EAB0
S214446E20C02203F001034BEA020BDAF8C0224BEA15
S214446E30C35302F07F421343DDE90201CAF8C0326D
S214446E4008F032FCC0F30B000443BAF8C40200F462
S214446E5060400443AAF8C44207B0BDE8F08F00BFC0
S214446E605919402058194020541940204C194020A4
S214446E70481940204419402033336F410AD7233CF5
S214446E80401940203C194020CDCCCC42CDCC4C3D82
S214446E90381940205019402000F87F00C083402015
S214446EA0124B1A8DC3F86022114A1168114A01F038
S214446EB00F01126802F00F0242EA011293F82B10F7
S214446EC042EA0122A3F864229A8DC3F868220A4A49
S214446ED011680A4A126802F00F0242EA011283F865
S214446EE06C22074A126883F86D227047C08340209C
S214446EF0401F4020441F4020301F4020341F402065
S214446F002C1F4020114B1A8EC3F87022104A116869
S214446F10104A126802F00F0242EA011283F8742201
S214446F200D4A126883F875229A8EC3F878220B4A63
S214446F3011680B4A126802F00F0242EA011283F803
S214446F407C22084A126883F87D227047C08340201A
S214446F50201F4020241F40201C1F4020101F40207C
S214446F60141F40200C1F40200F4B1A8FC3F880225A
S214446F700E4A11680E4A126802F00F0242EA0112E3
S214446F8083F884229A8FC3F888220A4A11680A4AE8
S214446F90126802F00F0242EA011283F88C22074A72
S214446FA0126883F88D227047C0834020001F40201B
S214446FB0041F4020F41E4020F81E4020F01E4020AF
S214446FC0334B3449F0B51E78334B06F0030691F83C
S214446FD05C201D78314B42EA062205F003051C6806
S214446FE02F4B42EA8522240318682E4BA4B2000491
S214446FF01B78224300F4702003F003072A4B104307
S2144470001B7803F0030343EA8703284F3F7807F0CF
S214447010030743EA0713264F3F7807F0030743EA7C
S2144470208713244F3F7807F0030743EA0723224F8A
S2144470303F7807F0030743EA8723204F3F7807F05B
S214447040030743EA07331E4F3F68BF03BFB23B43C1
S2144470501C4F43EA06433F7843EA864307F0030758
S21444706043EA065343EA865343EA066343EA87639E
S214447070D1F8047207F070473B43C1F80432D1F8A4
S21444708008321B0D1B051843C1F80802F0BD00BFAB
S214447090581E4020C0834020591E40200C1A4020D1
S2144470A0081A40205B1E40205A1E40205C1E40208A
S2144470B05D1E40205E1E4020601E40205F1E402015
S2144470C0541E402065184020204B214A70B51C6849
S2144470D0204BB2F8605004F00F04186892F8603001
S2144470E005F4FF4592F8641000F00F0003F07F03A8
S2144470F02B43156E05F4FF052B43B2F86250C5F3D7
S214447100C11543EAC55392F86350C5F3410643EAB2
S2144471104663C5F3C106C5F3411543EAC66343EA6D
S2144471204573D2F80C5205F000452B43C2F80C3296
S21444713001F03F03B2F8101243EA841301F44041CD
S21444714043EA80230B43A2F8103270BDE41D40206E
S214447150C0834020E01D40201D4B1E4A1B68126819
S2144471609B001D4902F0030203F00C0313431B4A21
S2144471701268120102F030021343194A126892014F
S214447180D2B21343174A1268120202F440721343EF
S214447190154A1268920202F440621343134A126874
S2144471A0120302F440521343114A1268920302F443
S2144471B0703213430F4A1268920402F47012134357
S2144471C0D1F82422920D92051343C1F82432704715
S2144471D0F8194020FC194020C0834020F419402070
S2144471E0F0194020EC194020E8194020E4194020CA
S2144471F0E0194020DC1940201A4B1B49186810B58A
S21444720008F084FC194C07F01FFF0CF025FF08F02B
S2144472104BFA174B1449A4F81402186808F076FC85
S21444722007F012FF0CF018FF08F03EFA114BA4F8D2
S2144472301602188808F062FB0B4908F067FC07F052
S21444724003FF0CF009FF08F02FFA0B4BA4F81802C2
S2144472501A680A4B1B6803F00F0343EA021384F8C8
S2144472601A3210BDC41D4020CDCCCC3DC083402036
S214447270C81D4020C21D4020281E40202C1E4020F1
S214447280124A92F8783010B582F81C32104BD2F875
S2144472901C421878B2F87A30C3F38701936FC3F36D
S2144472A009231B0243EA81430A49097801F00F0186
S2144472B043EA8163084921400B43C2F81C3292F8E2
S2144472C0203260F3030382F8203210BDC08340208E
S2144472D0D6194020D7194020FF0000C0094B0A4960
S2144472E01A680A4B02F007021B6803F0030343EADA
S2144472F0820391F89C2222F01F02134381F89C32A9
S214447300704700BF581C4020C08340204C1B402080
S214447310064B10B5064C186808F00AFDB4F8A032BF
S21444732060F30903A4F8A03210BD00BF741C4020CB
S214447330C0834020094B0A4A1B7812789B000949AF
S21444734002F0030203F00C03134391F8A42222F044
S2144473500F02134381F8A432704700BFD21940206D
S214447360D3194020C0834020044B054993F8A822F3
S214447370097861F3020283F8A8227047C08340204C
S214447380D1194020044B054993F8AC22097861F39F
S214447390030283F8AC227047C0834020D0194020B3
S2144473A0F8B53D4B3D4D1B783D4985F8B0323D4BD5
S2144473B0186808F0ABFB07F047FE0CF04DFE08F0EB
S2144473C073F9394A394B03EA40231068D5F8B0229A
S2144473D0000200F480700343354810400343C5F868
S2144473E0B032344B1B7885F8B432334B1C68334B7D
S2144473F004F003041F68324B07F001071E68314B44
S21444740044EA870406F00106186808F073FA4FF059
S214447410814108F0C7FA08F08BFC2B4A2B4B44EA10
S214447420C606D5F8B41203EA00231068284A800535
S21444743095F8B84200F4800024F00F040343106823
S214447440244A2643C005126800F4000085F8B86252
S2144474501206034302F0407213431F4A1268920610
S21444746002F0406213431D4A1268120702F080522B
S21444747013431B4A1268520702F000521343194A38
S2144474801268920702F080421343174A0A40134395
S214447490C5F8B432F8BD00BF78194020C0834020F8
S2144474A0CDCCCC3DA8194020AC19402000FEFF01AD
S2144474B0FF0000FE7919402084194020801940209E
S2144474C07C194020A4194020A019402000FF3F000A
S2144474D09C194020581C4020941940209019402064
S2144474E08C19402088194020FF000080084A094B28
S2144474F01278094983F8C822084A0978127883F82A
S214447500C92293F8CA2261F3000283F8CA2270475C
S214447510C2194020C0834020C0194020C1194020D1
S214447520114B12491B6810B5114C84F8E832114BC4
S2144475301B6884F8E932104B186808F02BF90F4999
S21444754008F0E4FA07F080FD0CF086FD08F0ACF88D
S2144475500B4A94F8EC321278A4F8EA0262F3000379
S21444756084F8EC3210BD00BFBC19402000C0234450
S214447570C0834020B8194020B41940200AD7A33C01
S214447580B0194020F8B5204B204D186808F0B2F9E1
S2144475904FF0814108F006FA08F0CAFB1C4B04463B
S2144475A01F681C4BC4F30D0407F001071E681A4BF2
S2144475B044EA8734186844EAC63408F09BF94FF026
S2144475C0814108F0EFF908F0B3FB144AC0F30D0309
S2144475D0A5F8E4421068124A800300F4804003434E
S2144475E01068104AC003126800F4FF00D205034333
S2144475F002F0FF421343D5F8E02202F00042134360
S214447600C5F8E032F8BD00BF64194020C08340206E
S214447610601940205C19402074194020701940209D
S2144476206C194020681940200D4B0E4A1B780E49B1
S21444763082F8F4320D4B09781B7801F0010182F888
S214447640F5320B4B1B785B0003F002030B4392F8B6
S214447650F61221F003010B4382F8F632704700BF5E
S21444766037194020C0834020351940203619402021
S214447670341940200C4B0D4A1B680D4982F8F032F1
S2144476800C4B09781B6801F0030182F8F1320A4B6F
S2144476901B789B0003F00C030B430849097843EA24
S2144476A0011382F8F232704730194020C0834020DC
S2144476B02B1940202C1940202A19402029194020F3
S2144476C0F8B5254B254C1B78254F84F8F832254BC6
S2144476D01B7884F8F932244B1878323008F00EF9C7
S2144476E0014608F057F808F023FB204984F8FA02CC
S2144476F00E781F493F780D781E4907F001071E4B48
S21444770008781E491A78303009781D4B49001B7892
S21444771001F03E01394394F8FB7227F03F073943A2
S21444772084F8FB1203F03F0102F01F0306F00F0239
S21444773043EA411343EAC22305F03F0243EAC23315
S21444774000F03F0243EA4253D4F8FC2202F0784267
S2144477501343C4F8FC32F8BD28194020C0834020A7
S2144477602519402027194020261940202119402059
S214447770201940201F194020231940202419402056
S2144477802219402038B50C4B0C4C5D68284607F04F
S2144477905BFC0CF061FC07F087FF0949C4F8DC0287
S2144477A0284608F0B3F907F04FFC0CF055FC07F0F8
S2144477B07BFFC4F8D80238BD20464020C083402012
S2144477C0000008422DE9F74F374D384E686808F0F8
S2144477D0AFFA86F80003A86808F0AAFA344986F88F
S2144477E00103686907F0D6FF324908F08FF908F0BC
S2144477F09FFA8346A86908F09BFA2D490446E8692F
S21444780007F0C8FF2B4908F081F9CBF3090B08F0C1
S2144478108FFA8246286A08F08BFA25498146686AB8
S21444782007F0B8FF234908F071F908F081FA80465A
S214447830A86A08F07DFA1E4900F00107E86807F0D8
S214447840A9FF1C4908F062F908F072FAC0F309036C
S2144478502869019308F06CFA019B00F0010043EAA2
S2144478608023B6F8020300F4784003431248A6F88F
S2144478700233A30200EACA2A03F480634FEA49505B
S21444788043EA0B0300F4001043EA0A03034343EAC3
S2144478908853C6F8043396F8083367F3000386F82B
S2144478A0083303B0BDE8F08F20464020C083402014
S2144478B066667241CDCC4C3D00F81F00084A094B21
S2144478C01278094983F83023084A0978127883F8ED
S2144478D0312393F8322361F3000283F8322370474E
S2144478E01E194020C08340201C1940201D194020EA
S2144478F0114B124A1B68124910B5124C127884F880
S2144479002033114B1B6884F8213394F8243362F3F4
S214447910000384F824330D4B186807F03BFF0C49EA
S21444792008F0F4F807F090FB0CF096FB07F0BCFE6A
S214447930A4F8220310BD00BF181940200E19402099
S21444794000C02344C083402014194020101940200E
S2144479500AD7A33C284B294910B5294C1B7884F8F0
S2144479601833284B186808F0D1F807F06DFB0CF074
S21444797073FB07F099FE244A244B03EA402310681D
S214447980D4F81823000200F48070034320481040C3
S214447990204A03431268C4F8183312021E4B02F4FA
S2144479A080721B7884F81C331C4B1B685B0203F400
S2144479B0C06313431A4A1268D20202F4C0521343F5
S2144479C0184A1268520302F400521343164A1268C5
S2144479D0920302F480421343144A1268D20302F418
S2144479E0C0321343D4F81C2322F4FF3222F48072AC
S2144479F01343C4F81C3310BD0C194020CDCCCC3DE9
S214447A00C0834020041940200819402000FEFF018E
S214447A10FF0000FE001940200D194020FC184020AD
S214447A20F8184020F4184020F0184020EC18402065
S214447A303A4B4FF084412DE9F047394E1B7886F88F
S214447A400C33384B1B7886F80D33374B186807F0E1
S214447A50A1FE4FF0834107F0A5FF08F069F9334BC8
S214447A600446334993F800A0324B0AF0010A1868DA
S214447A7007F090FE304908F049F808F059F92F4BC2
S214447A8081462F4993F800802E4B08F00108186869
S214447A9007F080FE2C4908F039F808F049F92B4BDA
S214447AA005464FF084411F78294BC5F30B0507F074
S214447AB00107186807F06EFE4FF0834107F072FF27
S214447AC008F036F9234BC0F3090245EA073518781F
S214447AD0C4F3090300F0010043EA8A2342EA802201
S214447AE0B6F80E0300F4784002431B4800EAC9295E
S214447AF0A6F80E23D6F8102343EA090302F07F4281
S214447B0043EAC8531343C6F81033B6F8143303F4A1
S214447B1060431D43A6F81453BDE8F087E918402097
S214447B20C0834020E8184020DC184020D818402065
S214447B3033336F41D41840200AD7233CD018402012
S214447B40CDCCCC42CC184020CDCC4C3DC81840209F
S214447B50E4184020E018402000F87F002DE9F74F55
S214447B60374D384E686808F0E3F886F85003A8683E
S214447B7008F0DEF8344986F85103686907F00AFECF
S214447B80324907F0C3FF08F0D3F88346A86908F0E3
S214447B90CFF82D490446E86907F0FCFD2B4907F069
S214447BA0B5FFCBF3090B08F0C3F88246286A08F001
S214447BB0BFF825498146686A07F0ECFD234907F07B
S214447BC0A5FF08F0B5F88046A86A08F0B1F81E4943
S214447BD000F00107E86807F0DDFD1C4907F096FF52
S214447BE008F0A6F8C0F309032869019308F0A0F842
S214447BF0019B00F0010043EA8023B6F8520300F4E8
S214447C00784003431248A6F85233A30200EACA2A2D
S214447C1003F480634FEA495043EA0B0300F4001030
S214447C2043EA0A03034343EA8853C6F8543396F8B0
S214447C30583367F3000386F8583303B0BDE8F08F33
S214447C4020464020C083402066667241CDCC4C3DE1
S214447C5000F81F000D4B0E4A1B780E4982F82C3351
S214447C600D4B09781B7801F0010182F82D330B4B3C
S214447C701B785B0003F002030B4392F82E1321F0AB
S214447C8003010B4382F82E33704700BFC7184020C9
S214447C90C0834020C5184020C6184020C418402041
S214447CA00C4B0D4A1B680D4982F828330C4B097857
S214447CB01B6801F0030182F829330A4B1B789B00AA
S214447CC003F00C030B430849097843EA011382F88E
S214447CD02A337047C0184020C0834020B81840203C
S214447CE0BC184020B7184020B6184020F8B5254B9D
S214447CF0254C1B78254F84F84833254B1B7884F84D
S214447D004933244B1878323007F0F8FD014607F023
S214447D1041FD08F00DF8204984F84A030E781F49BF
S214447D203F780D781E4907F001071E4B08781E4918
S214447D301A78303009781D4B49001B7801F03E0113
S214447D40394394F84B7327F03F07394384F84B1371
S214447D5003F03F0102F01F0306F00F0243EA41130B
S214447D6043EAC22305F03F0243EAC23300F03F022F
S214447D7043EA4253D4F84C2302F078421343C4F8FF
S214447D804C33F8BDB5184020C0834020B21840207C
S214447D90B4184020B3184020AE184020AD184020F8
S214447DA0AC184020B0184020B1184020AF184020EE
S214447DB008B5FFF785FCBDE80840FFF797BF38B520
S214447DC00C4B0D4C5D68284607F03EF90CF044F920
S214447DD007F06AFC0949C4F84403284607F096FEAF
S214447DE007F032F90CF038F907F05EFCC4F84003AB
S214447DF038BD00BF20464020C083402000000842D3
S214447E0008B5FEF75CF8FEF7A1F8FEF7FBF8FEF7B8
S214447E1039F9FEF779F9FEF741FAFEF785FAFEF7E7
S214447E20C3FAFEF7FFFAFEF73BFBFEF75BFBFEF7F3
S214447E3029FCFEF759FCFEF771FCFEF7F7FCFEF74B
S214447E4061FDFEF7BFFDFEF737FEFEF777FEFEF751
S214447E50B3FEFEF7EFFEFEF72BFFFFF721F8FFF722
S214447E6051F8FFF781F8FFF7ABF8FFF72DF9FFF766
S214447E70C3F9FFF705FAFFF76FF9FFF72FFAFFF795
S214447E8047FAFFF757FAFFF76FFAFFF77BFAFEF762
S214447E904DFFFFF777FCFFF7CBFDBDE80840FFF743
S214447EA08EBF114B11491B6810B5114C84F85C33D6
S214447EB0104B1B6884F85D330F4B186807F06AFC58
S214447EC00E4907F023FE07F0BFF80CF0C5F807F09C
S214447ED0EBFB0B4A94F860331278A4F85E0362F323
S214447EE0000384F8603310BDA818402000C0234423
S214447EF0C0834020A4184020A01840200AD7A33CA2
S214447F009D1840200D4B0E4A1B780E4982F8683364
S214447F100D4B09781B7801F0010182F869330B4B4D
S214447F201B785B0003F002030B4392F86A1321F0BC
S214447F3003010B4382F86A33704700BF9C18402005
S214447F40C08340209A1840209B184020991840200F
S214447F500C4B0D4A1B780D4982F864330C4B097858
S214447F601B7801F0030182F865330A4B1B789B00AB
S214447F7003F00C030B430849097843EA011382F8DB
S214447F806633704798184020C08340209618402097
S214447F90971840209518402094184020114B1249B9
S214447FA01B6810B5114C84F86C33114B1B6884F86D
S214447FB06D33104B186807F0EDFB0F4907F0A6FD2C
S214447FC007F042F80CF048F807F06EFB0B4A94F8BA
S214447FD070331278A4F86E0362F3000384F87033A7
S214447FE010BD00BF9018402000C02344C0834020EA
S214447FF08C184020881840200AD7A33C8418402078
S2144480000D4B0E4A1B780E4982F874330D4B097893
S2144480101B7801F0010182F875330B4B1B785B002B
S21444802003F002030B4392F8761321F003010B434B
S21444803082F87633704700BF83184020C0834020C0
S2144480408118402082184020801840200C4B0D4A4E
S2144480501B680D4982F878330C4B09781B6801F08D
S214448060030182F879330A4B1B789B0003F00C0318
S2144480700B430849097843EA011382F87A33704778
S2144480807C184020C0834020751840207818402033
S214448090741840207318402008B5FFF727FAFFF7F6
S2144480A03FFAFFF77DF9FFF76DFAFFF78BFBFFF713
S2144480B0BBFAFFF7DFFAFFF701FCFFF719FCFFF7FF
S2144480C049FCFFF74BFDFFF7C5FDFFF7E9FDFFF75A
S2144480D0E8FEFFF717FFFFF73BFFFFF75FFFFFF7EB
S2144480E08FFFBDE80840FFF7B1BF074A0020074BA3
S2144480F0D2F87811D2F87C219962DA62044B93E87C
S2144481000600FBF7A5BC00BFC08340204087402044
S21444811034774600144A154892F8851192F884310B
S21444812010B4C1F3010480F8283001F01C03C1F3F5
S2144481304111234380F82930D2F88431C3F3C13443
S21444814092F88C31C3F3C003DB0143EA84030B4348
S21444815080F82A30D2F88831C3620020044B10BC21
S21444816093E80600FBF774BCC08340204087402059
S2144481703C7746000B4A00200B4BD2F8901199628C
S214448180B2F8941183F82C1092F8961192F897212D
S21444819083F82D1083F82E20044B93E80600FBF753
S2144481A057BC00BFC08340204087402044774600E9
S2144481B0084B002093F8E831C3F3000203F0FE03B3
S2144481C01343054A82F82830044B93E80600FBF72D
S2144481D03FBC00BFC0834020408740204C774600C9
S2144481E0064A0020064BD2F8EC11B2F8F021996208
S2144481F09A85044B93E80600FBF72ABCC0834020CC
S214448200408740207C77460008B50A4B50200A4AEF
S214448210D3F8A81193F8AC312832116008211371B1
S21444822003F0F4FE054B002093E80600BDE8084042
S214448230FBF70EBCC083402040874020547746005E
S214448240094B00200949D3F8B02193F8B4318A6227
S21444825003F0F002C3F30303134381F82F30044BB7
S21444826093E80600FBF7F4BBC083402040874020D9
S2144482705C774600094B00200949D3F8B82193F8A7
S214448280BC318A6203F0F002C3F30303134381F85C
S2144482902F30044B93E80600FBF7DABBC08340203C
S2144482A04087402064774600094B00200949D3F8AC
S2144482B0C02193F8C4318A6203F0F002C3F3030387
S2144482C0134381F82F30044B93E80600FBF7C0BBFA
S2144482D0C0834020408740206C7746000A4A0020EE
S2144482E00A4BD2F8E01192F8E421996283F82C20E4
S2144482F083F82D2083F82E2083F82F20044B93E810
S2144483000600FBF7A5BB00BFC08340204087402043
S21444831074774600254A264992F8C831C3F30100CB
S21444832003F0FC03034310B481F8283092F8C931B3
S214448330C3F3010003F0FC03034392F8CA0181F837
S2144483402930C0F3010400F00C0323438409C0F32E
S214448350011081F82A3092F8CB3103F003039B01D5
S21444836043EA8403034381F82B3092F8CC3181F8F6
S2144483702C3092F8CD3103F03800C3F302030343A4
S21444838081F82D3092F8CE31C3F38300D2F8CC3145
S214448390C3F3833343EA0013002081F82F30054BA0
S2144483A010BC93E80600FBF753BB00BFC0834020D5
S2144483B040874020847746000B490C4A91F8D031D8
S2144483C0C3F3010003F0FC030343002082F8283083
S2144483D091F8D131C3F3010382F82930044B93E872
S2144483E00600FBF735BB00BFC083402040874020D3
S2144483F08C774600084B002093F8DC3103F00402E7
S214448400C3F301031343054A82F82830044B93E828
S2144484100600FBF71DBB00BFC083402040874020BA
S214448420947746001049114A91F8D431C3F30000BA
S21444843003F0FE03034382F8283091F8D53103F065
S2144484407C00C3F301030343002082F82930D1F8AB
S214448450D431C3F3CF335385D1F8D831D362044BE8
S21444846093E80600FBF7F4BAC083402040874020D8
S2144484709C7746001B4938B51B4CD1F8483204F566
S214448480FE52B1F84C02136041F6C473E05291F8C0
S2144484904E32C3F34100C3F3C1050543C3F30000A2
S2144484A0C3F3401340EA850040EA430341F6C670EE
S2144484B0235491F84F32C3F38300B1F84E3241F659
S2144484C0C771C3F3831343EA00131320635408218C
S2144484D003F005FF054B012093E80600BDE838404D
S2144484E0FBF7B6BAC083402040874020C477460096
S2144484F02149224B91F8500203F5FE5210B500F084
S214448500F004C0F303002043107091F8510200F0C9
S2144485107004C0F30300204341F6C174185541F675
S214448520C274D1F85002C0F3C130185541F6C37432
S214448530B1F85202C0F34700185541F6C470B1F87A
S214448540544291F856121C5441F6C57000241C54EB
S21444855001F0F000C1F30301014341F6C77019541A
S2144485600821142003F0BBFE054B012093E80600C7
S214448570BDE81040FBF76CBAC083402040874020DB
S214448580CC774600154B164903F5FE5291F858022F
S21444859010B51070002441F6C1701C5441F6C270E8
S2144485A0B1F85A421C5241F6C470B1F85C4291F894
S2144485B05E121C5201F0F000C1F30301014341F680
S2144485C0C77019540821152003F089FE054B012075
S2144485D093E80600BDE81040FBF73ABA40874020CF
S2144485E0C0834020D477460010B512490020124C70
S2144485F001F5FE52D4F89032136041F6C473C85461
S21444860094F89532C3F34300B4F89432C3F3431357
S21444861043EA001341F6C7700B540821162003F0B2
S2144486205EFE064B012093E80600BDE81040FBF7CB
S2144486300FBA00BF40874020C0834020DC77460006
S214448640FFF7D2BF08B5FDF7ADFBF9F70EF9FEF715
S214448650EBF9BDE80840FFF7C7BF084B012093F885
S2144486609832C3F3000203F0FE031343044A137024
S214448670044B93E80600FBF7EBB900BFC0834020E9
S21444868000A74020E477460008B50E480E4B00F598
S214448690FE52D3F8281293F82C32116003F0F001FE
S2144486A0C3F303030B4341F6C771435408215020D8
S2144486B003F015FE054B012093E80600BDE808408C
S2144486C0FBF7C6B940874020C0834020A4774600C5
S2144486D008B50E480E4B00F5FE52D3F8301293F808
S2144486E03432116003F0F001C3F303030B4341F645
S2144486F0C77143540821512003F0F1FD054B012076
S21444870093E80600BDE80840FBF7A2B9408740203E
S214448710C0834020AC77460008B50E480E4B00F5A3
S214448720FE52D3F8381293F83C32116003F0F0014D
S214448730C3F303030B4341F6C77143540821602037
S21444874003F0CDFD054B012093E80600BDE8084044
S214448750FBF77EB940874020C0834020B47746006C
S21444876008B50E480E4B00F5FE52D3F8401293F867
S2144487704432116003F0F001C3F303030B4341F6A4
S214448780C77143540821612003F0A9FD054B01201D
S21444879093E80600BDE80840FBF75AB940874020F6
S2144487A0C0834020BC774600194B1A4A03F5FE5155
S2144487B0B2F86002088092F8641201F0F000C1F347
S2144487C00301014341F6C270195441F6C37192F84D
S2144487D06502585441F6C47092F86812195441F62A
S2144487E0C570195492F86C1201F0F000C1F30301FD
S2144487F0014341F6C6701954012092F86D1241F6B1
S214448800C7729954044B93E80600FBF721B900BF9E
S21444881040874020C0834020EC774600194B1A4AD4
S21444882003F5FE51B2F87002088092F8741201F013
S214448830F000C1F30301014341F6C270195441F6F6
S214448840C37192F87502585441F6C47092F878127F
S214448850195441F6C570195492F87C1201F0F00090
S214448860C1F30301014341F6C6701954012092F83E
S2144488707D1241F6C7729954044B93E80600FBF701
S214448880E7B800BF40874020C0834020F4774600C6
S214448890174B184A03F5FE51B2F88002088092F846
S2144488A0841201F0F000C1F30301014341F6C270A3
S2144488B0195441F6C370D2F888121954090A41F67D
S2144488C0C470195492F88C1201F0F000C1F30301FD
S2144488D0014341F6C6701954012092F88D1241F6B0
S2144488E0C7729954044B93E80600FBF7B1B800BF2F
S2144488F040874020C0834020FC77460028482949CA
S21444890090F8043201F5FE5270B5C3F3010403F047
S214448910FC032343137090F80532C3F3010403F0B9
S214448920FC03234341F6C1740B5541F6C27390F8D9
S21444893006422501A609C4F30114CD5490F8075203
S21444894005F00303C5F381051B0143EA860323436D
S21444895041F6C37443EA85130B5541F6C47390F845
S2144489600842CC5441F6C57490F8093290F80A028D
S2144489701D01C3F3031300F00F000D5543EA001323
S21444898041F6C7700B5408214FF4AE6003F0A7FCC1
S214448990054B012093E80600BDE87040FBF758B845
S2144489A0C083402040874020247846002D4991F8D3
S2144489B00C0238B5C0F3001500F008032A4C43EA0D
S2144489C04513C0F3020504F5FE522B43C0F340158D
S2144489D0C0F3801043EA851343EAC01341F6C170DE
S2144489E01370B1F80C32C3F3C713235441F6C27064
S2144489F0D1F80C32C3F3C733235491F80F02C0F3B3
S214448A00C103C0F34105C0F341101B0143EA85038B
S214448A10B1F80E52C5F3C1152B4343EA801341F611
S214448A20C370235441F6C47091F810329B0023540B
S214448A3091F81132C3F38300B1F8103241F6C7718E
S214448A40C3F3831343EA00134FF4B060635408211E
S214448A5003F045FC054B012093E80600BDE838408A
S214448A60FAF7F6BFC0834020408740202C78460063
S214448A701849194891F8243200F5FE5210B5C3F34C
S214448A80010403F0FC032343137091F8253203F0EA
S214448A903C04C3F30103234341F6C174035591F8E0
S214448AA02632C3F38304D1F8243241F6C771C3F3A4
S214448AB0833343EA04134354082140F2855003F0B9
S214448AC00EFC064B012093E80600BDE81040FAF77A
S214448AD0BFBF00BFC0834020408740203478460054
S214448AE01149124B01F5FE52D3F8140210B5B3F8EF
S214448AF01842106041F6C47093F81A320C5203F0D0
S214448B00F000C3F30303034341F6C7700B54082134
S214448B104FF4B26003F0E3FB054B012093E80600F4
S214448B20BDE81040FAF794BF40874020C0834020F9
S214448B30447846001749184891F81C3200F5FE520E
S214448B4010B5137041F6C174D1F81C32C3F309232F
S214448B50035541F6C274B1F81E32C3F3810303557C
S214448B6091F8203203F00F0491F81F3241F6C77192
S214448B70C3F3830343EA04134354082140F2955055
S214448B8003F0ADFB054B012093E80600BDE810401A
S214448B90FAF75EBFC0834020408740204C784600AA
S214448BA0084B0120084993F89C3203F01C02C3F397
S214448BB00103134341F6C3728B54044B93E80600F7
S214448BC0FAF746BFC08340204087402004784600DA
S214448BD0084B41F6C271B3F8A022074BC2F30120FA
S214448BE0585441F6C37101205A54044B93E8060086
S214448BF0FAF72EBFC0834020408740200C784600BA
S214448C00054B0120054A93F8A4321B011370044B0C
S214448C1093E80600FAF71CBFC083402000A7402014
S214448C2014784600074B41F6C1720749012093F871
S214448C30A83203F007039B008B54044B93E80600CA
S214448C40FAF706BFC0834020408740201C78460081
S214448C50074B41F6C1720749012093F8AC32C3F37F
S214448C6003038B54044B93E80600FAF7F1BE00BFA7
S214448C70C0834020408740203C7846000D4843F659
S214448C805872B0F8C81208B549BA0B4B99521A44F0
S214448C9090F8CA1243F65A70C90119540321322077
S214448CA003F0B4F9054B022093E80600BDE80840FB
S214448CB0FAF7CEBEC0834020408740205478460012
S214448CC0114B43F65870114AB3F8E81249BA10B536
S214448CD0115243F65A74B3F8EA1293F8EC3249BA8E
S214448CE003F00103115343F65C719B015354024451
S214448CF00521402003F013F8054B022093E80600B4
S214448D00BDE81040FAF7A4BEC08340204087402008
S214448D105C7846003048314A90F8B43290F8B01245
S214448D2070B543F6587590F8B742535543F65973A1
S214448D30D15443F65A71D0F8B032C3F34F235BBADA
S214448D405352C4F3801304F0100141EAC301C4F340
S214448D500103194390F8B13203F0010341EA431189
S214448D60C4F3810304F0200441EA831143F65C73A0
S214448D70D15490F8B812C1F3800601F00803C1F349
S214448D80010143EA06130B4390F8B612D0F8B40236
S214448D902343CC09C1F3801143EA841343F65D743C
S214448DA01355C0F30D2343F65E74C0F305409B0091
S214448DB01055642043EA410343F65F7153542A44F2
S214448DC0082103F023F9064B022093E80600BDE889
S214448DD07040FAF73DBE00BFC08340204087402025
S214448DE0647846001F4843F658721F4BB0F8E212A8
S214448DF0C1F3C71170B5995443F65974D0F8E012CC
S214448E001A44B0F8E052C1F3C731C5F305261955E4
S214448E1090F8E54204F08001C4F38014314343F6ED
S214448E205A76995543F65B715D54B0F8E45290F81F
S214448E30E112C5F3052001F04001014343F65C709E
S214448E4041EAC411195443F65D716A205D54062103
S214448E5003F0DCF8054B022093E80600BDE87040BA
S214448E60FAF7F6BDC0834020408740206C78460021
S214448E7038B52C4B43F658702B4AB3F8BC12B3F8AB
S214448E80C45249BA115293F8C212CC09C5F303210D
S214448E9041EA041193F8C542C4F3001441EA44116C
S214448EA093F8BF42C4F3800441EA841193F8C14264
S214448EB0C4F3800441EAC41143F65A74115543F688
S214448EC05B71B3F8BE42555443F65C71C4F309056E
S214448ED0C4F387045454B3F8C012D3F8C032C1F371
S214448EE00904C1F3051141EA851143F65D755155F0
S214448EF0C3F3CB21C3F3C34343EA041343F65E747C
S214448F00135543F65F73D15402440821702003F08E
S214448F107DF8064B022093E80600BDE83840FAF791
S214448F2097BD00BFC08340204087402074784600E9
S214448F30284A43F658702849B2F800335BBA30B42E
S214448F400B5243F65A73B2F80203B2F80453C0F312
S214448F500904C0F38700C854C5F3012092F80333CC
S214448F6003F00403034392F80503C0F3800043EA86
S214448F70C00392F80603C0F3401043EA001392F885
S214448F80080300F0010043EA401343F65B7043EAEB
S214448F90841343F65D740B5443F65C73D2F80403AF
S214448FA0CD54C0F3C923B2F80623C0F347309B011F
S214448FB00855900943EA923343F65E728B5443F65F
S214448FC05F73C8540220054B30BC93E80600FAF79A
S214448FD03FBD00BFC0834020408740207C78460089
S214448FE0104843F65871104A08B5B0F8F4325BBAE4
S214448FF0535290F8F63203F00100C3F3400343EAB9
S214449000400343F65A7013540A444FF44470032101
S21444901002F085FE054B022093E80600BDE80840B2
S214449020FAF716BDC0834020408740208478460027
S214449030134843F65872134BB0F8F01249BA10B5B9
S21444904099521A4490F8F21243F65A70C1F3010446
S2144490501C54C1F3031443F65B70C1F381011C54E2
S21444906043F65C70195405214FF4547002F057FED1
S214449070054B022093E80600BDE81040FAF7E8BC2A
S214449080C0834020408740208C784600254943F6DC
S2144490905872B1F8F80238B540BA234B91F8FB42FF
S2144490A098521A44D1F8FC0204F00105C4F344046F
S2144490B0C0F3C53040EAC51043F65A75585543F6D2
S2144490C05B75B1F8FC02C0F34510585543F65C7521
S2144490D091F8FC02C0F304005855B1F8FE02C0F300
S2144490E0022500F4FC6045EAC40443F65D755C550D
S2144490F091F8FD42C4F3C304204343F65E74185506
S21444910091F8FA0243F65F71585408214FF461709F
S21444911002F07CFF054B022093E80600BDE8384089
S214449120FAF796BCC0834020408740209478460097
S214449130094943F65870094AD1F8D8321BBA135035
S2144491400220D1F8DC3243F65C711BBA5350044B10
S21444915093E80600FAF77CBCC08340204087402052
S2144491609C7846000E4845F6F062B0F8301308B5D1
S21444917049BA0C4B99521A4490F8321345F6F260A9
S214449180C1F3000119540321332002F03FFF064B7C
S214449190032093E80600BDE80840FAF759BC00BF30
S2144491A0C083402040874020A4784600114B45F6B3
S2144491B0F060114AB3F8201349BA10B5115245F677
S2144491C0F264B3F8221393F8243349BA03F0010344
S2144491D0115345F6F4619B01535402440521402043
S2144491E002F0FAFD054B032093E80600BDE8104064
S2144491F0FAF72EBCC083402040874020AC78460017
S2144492002248234A90F8181338B590F81C3345F68C
S214449210F064135545F6F163D15445F6F261D0F83F
S2144492201833C3F34F235BBA535290F81D13C1F35C
S2144492304013C1F380151B0143EAC503C1F341053E
S2144492402B4390F8195305F0010543EA4513C1F33F
S214449250C10501F0010143EA851345F6F46553550B
S214449260D0F81C336520C3F3C13343EA811145F675
S214449270F563D1542244082102F0C8FE054B03206E
S21444928093E80600BDE83840FAF7E2BBC0834020C6
S21444929040874020B478460038B52C4B45F6F060FD
S2144492A02B4AB3F80C13B3F8145349BA115293F833
S2144492B01213CC09C5F3032141EA041193F815436C
S2144492C0C4F3001441EA441193F80F43C4F38004F2
S2144492D041EA841193F81143C4F3800441EAC4116B
S2144492E045F6F264115545F6F361B3F80E4355540A
S2144492F045F6F461C4F30905C4F387045454B3F83B
S2144493001013D3F81033C1F30904C1F3051141EA2D
S214449310851145F6F5655155C3F3CB21C3F3C343D5
S21444932043EA041345F6F664135545F6F763D154F9
S21444933002440821712002F069FE064B032093E89C
S2144493400600BDE83840FAF783BB00BFC083402020
S21444935040874020BC78460008B5FEF7C6FEFEF7B8
S214449360D9FEFEF707FFFEF723FFFEF74DFFFEF795
S21444937067FFFEF7B3FFFEF7CDFFFFF71DF8FFF7D5
S21444938039F8FFF74FF8FEF72BFFFFF773F8FFF7B0
S214449390AFF8FFF7F7F8FFF760F9FFF799F9FFF72B
S2144493A0BBF9FFF7DDF9FFF76FF9FFF7FDF9FFF7B4
S2144493B035FAFFF76DFAFFF7A1FAFFF7F7FAFFF76A
S2144493C08FFBFFF755FBFFF7B5FBFFF7E9FBFFF70E
S2144493D0FFFBFFF715FCFFF725FCFFF739FCFFF70B
S2144493E047FDBDE80840FFF757BF284A45F6F060FA
S2144493F02749B2F850335BBA30B40B5245F6F263A1
S214449400B2F85203B2F85453C0F30904C0F38700C9
S214449410C854C5F3012092F8533303F004030343BE
S21444942092F85503C0F3800043EAC00392F856030B
S214449430C0F3401043EA001392F8580300F00100CA
S21444944043EA401345F6F36043EA841345F6F5646D
S2144494500B5445F6F463D2F85403CD54C0F3C923F1
S214449460B2F85623C0F347309B010855900943EAA7
S214449470923345F6F6628B5445F6F763C854032098
S214449480044B30BC93E80600FAF7E2BAC0834020A7
S21444949040874020C4784600104845F6F061104A9C
S2144494A008B5B0F82C335BBA535290F82E3303F019
S2144494B00100C3F3400343EA400345F6F260135405
S2144494C00A444FF44470032102F086FC054B032003
S2144494D093E80600BDE80840FAF7BABAC0834020CD
S2144494E040874020CC784600134845F6F062134B3C
S2144494F0B0F8281349BA10B599521A4490F82A136A
S21444950045F6F260C1F301041C54C1F3031445F656
S214449510F360C1F381011C5445F6F46019540521E7
S2144495204FF4547002F058FC054B032093E80600B1
S214449530BDE81040FAF78CBAC083402040874020EC
S214449540D4784600254945F6F062B1F8480338B564
S21444955040BA234B91F84B4398521A44D1F84C03E3
S21444956004F00105C4F34404C0F3C53040EAC51012
S21444957045F6F265585545F6F365B1F84C03C0F325
S2144495804510585545F6F46591F84C03C0F304006D
S2144495905855B1F84E03C0F3022500F4FC6045EA82
S2144495A0C40445F6F5655C5591F84D43C4F3C304CD
S2144495B0204345F6F664185591F84A0345F6F76194
S2144495C05854082140F2853002F020FD054B032014
S2144495D093E80600BDE83840FAF73ABAC08340201C
S2144495E040874020DC78460008B5FFF74FFDBDE8CD
S2144495F00840FFF7A7BF08B5F8F739F9FEF7D8FBD8
S214449600BDE80840FFF7F0BF094945F6F060094A4F
S214449610D1F840331BBA13500320D1F8443345F6EF
S214449620F4611BBA5350044B93E80600FAF710BA99
S214449630C083402040874020E4784600114B47F6DC
S2144496408860114AB3F85C1349BA10B5115247F60C
S2144496508A64B3F85E1393F8603349BA03F001039F
S214449660115347F68C619B01535402440521402014
S21444967002F010FC054B042093E80600BDE81040B9
S214449680FAF7E6B9C083402040874020EC7846008D
S214449690104847F68861104A08B5B0F868335BBA94
S2144496A0535290F86A3303F00100C3F3400343EA8D
S2144496B0400347F68A6013540A444FF44470032127
S2144496C002F0E8FB054B042093E80600BDE808409A
S2144496D0FAF7BEB9C083402040874020F47846005D
S2144496E0134847F68862134BB0F8641349BA10B56A
S2144496F099521A4490F8661347F68A60C1F30104F7
S2144497001C54C1F3031447F68B60C1F381011C5407
S21444971047F68C60195405214FF4547002F0BAFB96
S214449720054B042093E80600BDE81040FAF790B9CC
S214449730C083402040874020FC78460008B50A4B4A
S21444974049F6226209494020B3F86E335BBA8B521D
S2144497500521074A02F0FCFB064B052093E8060069
S214449760BDE80840FAF774B9C083402040874020DB
S2144497706025412004794600134849F62062134B7D
S214449780B0F8781349BA10B599521A4490F87A1337
S21444979049F62260C1F301041C54C1F3810449F61E
S2144497A02360C1F303111C5449F62460195405215F
S2144497B04FF4547002F0CCFB054B052093E80600AA
S2144497C0BDE81040FAF744B9C083402040874020A3
S2144497D014794600104849F62061104A08B5B0F896
S2144497E074335BBA535290F8763303F00100C3F3F4
S2144497F0400343EA400349F6226013540A444FF4B4
S2144498004470032102F0A4FB054B052093E80600B0
S214449810BDE80840FAF71CB9C08340204087402082
S2144498200C79460008B5FFF729FAFFF749FAFFF71F
S21444983071FAFFF7D7FAFFF7D3FBFFF7F9FBFFF709
S21444984091FCFFF7B3FCFFF7DBFCFFF725FEFFF7C1
S2144498504BFEFFF7F3FEFFF71BFFFFF741FFFFF753
S2144498606DFFFFF7B7FFBDE80840FFF785BF08B5B3
S214449870FCF70CFBF7F7CFFFFEF70EFCBDE80840FD
S214449880FFF7D0BF7047704770477047064AB2F834
S2144498902432B2F8681003F44043C1F30D010B437D
S2144498A0A2F82432704700BFC0834020044BB3F86C
S2144498B01221A3F82822B3F80C21A3F82A227047D1
S2144498C0C0834020044BB3F8A620A3F83022B3F854
S2144498D0A020A3F832227047C083402070477047C8
S2144498E0054BB3F86C21A3F83822D3F86821C2F3A9
S2144498F00F12A3F83A227047C0834020054BB3F8B2
S2144499007421A3F84022D3F87021C2F30F12A3F8AF
S21444991042227047C0834020054BB3F86C21A3F81D
S214449920B821D3F86821C2F30F12A3F8BA217047BE
S214449930C0834020054BB3F87421A3F8C021D3F864
S2144499407021C2F30F12A3F8C2217047C08340208F
S21444995008B5FFF7E1FFFFF7EDFFFFF797FFFFF7C7
S214449960A5FFFFF7AFFFFFF7BBFFBDE80840FFF7D3
S214449970C5BF08B5FCF7B0F9F7F74EFFFEF740FA57
S214449980FFF7E6FFBDE80840FFF7E6BC70477047C0
S214449990704770470B4AD2F8C831D2F894101B0D62
S2144499A0C1F313011B050B43D2F89810C2F8C83113
S2144499B001F47F11D2F8CC3123F47F130B43C2F861
S2144499C0CC317047C083402008B5F9F7DFF8BDE8CE
S2144499D00840F8F7EBBA7047F7F71BBFFFF747BFE7
S2144499E0FFF7C7BFFBF73CBA7047074A1378632BA9
S2144499F096BF01330023DBB21370044A1368013365
S214449A001360FEF71FBE00BF58484120E0204020A8
S214449A1008B5FAF739F8BDE8084002F00BB808B5BF
S214449A20FFF7E9FD4CF24053044AD058B0FA80F0B0
S214449A30BDE808404009F9F723B900BF5C48412017
S214449A40014900201DF008BDB89D460000201DF0C9
S214449A5007BD0022114610461DF006BD704700BFE4
S214449A60044B1A78044B1B78134302BF034B022261
S214449A701A707047631840205F18402064184020CE
S214449A80064B01221A70064B1B78934204D1054AB2
S214449A9013707822044B1A80704700BF271B40205F
S214449AA05F184020261B4020241B4020074B0848B4
S214449AB00849094A10B51B78084C012B18BF0023E7
S214449AC0237003700B70137010BD00BF281B40201A
S214449AD06918402068184020671840206A184020BB
S214449AE0124B134870B51978124B012900781C782C
S214449AF0114B124D1A78124B1B780CD1012C0AD1FB
S214449B00012A08D1012B06D1012804D1002328704C
S214449B100C4A137070BD214300260A432E7013432B
S214449B2003430CBF01233346F2E700BF6C184020C2
S214449B30671840206A184020691840207118402051
S214449B406818402070184020044B01221A600022F6
S214449B50034B1A700322034B1A707047E8204020C8
S214449B606E1840206418402008B5FFF79FFFFFF7A3
S214449B70B7FF044B1B78012B03D1BDE80840FFF721
S214449B80E3BF08BD71184020054B1B78012B06D156
S214449B90044B1B78012B02BF034B00221A707047FC
S214449BA05F1840206D184020641840200D4B0E4A24
S214449BB01B7833B90D4B1B78012B02BF1388013336
S214449BC0138000230A490B700A490B801188B1F5AB
S214449BD0FA7F05D31380054A13700222064B1A7087
S214449BE0704700BF5E18402016184020271B4020B0
S214449BF0261B4020241B4020721840200F4B1B7805
S214449C00012B18D10E4B1B78012B14D10D4B1B780E
S214449C10012B10D10C4B1B78012B0CD10B4B1B7812
S214449C205A1E534253410A4A13700123094A137079
S214449C30094A137070470023F5E700BF6C184020AC
S214449C406A18402069184020681840206718402049
S214449C50711840207018402072184020FFF7A6BFA5
S214449C60064B1B78042B064B97BF002201221A7022
S214449C70032298BF034B1A70704700BF2818402031
S214449C80281B40207218402008B5FFF7B7FF0C4841
S214449C900278012A0ED1FFF789FF0A4B1B78012B65
S214449CA007D10278032A04D1074A00211160074AE3
S214449CB0137008BD022AF0D1FFF7D2FFEDE700BFCC
S214449CC07218402070184020E82040206418402035
S214449CD02DE9F04FC24CBBB04FF0000A4FF0000BDA
S214449CE0A046D4E91A23D4E90267CDE90E233046C8
S214449CF00022BC4B394605F085FC002840F0CA815A
S214449D00D4E91245D8E90C2320462946CDE9002358
S214449D1005F06EFC08B9DDE9004500224FF08043AB
S214449D20DDE90E0105F050FC0022002800F0B58164
S214449D3000232046294605F0DFF902460B46D8E9BB
S214449D408E45CDE9022322462B4605F01DF8804673
S214449D5089468FA3D3E9002305F05EFC002800F073
S214449D609E81204629468AA3D3E9002305F00EF8AF
S214449D70CDE90201DFF868820022DDE90234C8E951
S214449D808E34D8E94234CDE90034D8E90E45002370
S214449D902046294605F018FC002800F0928100224F
S214449DA00023D8E9140105F023FC50B100228E4B61
S214449DB03046394605F026FC18B100230024CDE988
S214449DC00034874C94F87832002B40F0C98140F236
S214449DD00113A4F87832DFF808820022834BD8E9CE
S214449DE044452046294605F017FC002840F0D78114
S214449DF000227F4B2046294605F0F0FB002840F021
S214449E00D18198F87A320BB1C8E94645744B20465E
S214449E102946D3E9468942464B4604F0B5FF0446F4
S214449E200D465DA3D3E9002305F0F6FB002840F079
S214449E30BC81204629465AA3D3E9002305F0CEFB2D
S214449E40002840F0B68122462B464046494604F058
S214449E509DFF02460B46CDE9282353A3D3E90023AE
S214449E6005F04AF9804689460AF03EF904460D460E
S214449E70404649460AF0AAF85E4B80468946204644
S214449E802946D3E9002305F037F904460D464046F3
S214449E90494647A3D3E9002305F02EF900220023C0
S214449EA005F02AF902460B462046294604F06EFF82
S214449EB041A3D3E9002305F01FF941A3D3E90023C6
S214449EC005F01AF900224C4B04460D4605F0A4FB57
S214449ED0002840F07281002200232046294605F0DF
S214449EE07DFB08B1002400253D4B93F87B220AB144
S214449EF0C3E94845D3E948892046294642464B4665
S214449F0004F042FF04460D462FA3D3E9002305F090
S214449F1083FB002840F05481204629462CA3D3E9ED
S214449F20002305F05BFB002840F04E8122462B467A
S214449F304046494604F02AFF02460B46284CCDE9E3
S214449F40362325A3D3E9002305F0D6F800222B4B6D
S214449F50CDE90401C4E9A8ABDDE9000105F034FB12
S214449F60031E4FF00002394618BF012330460C93B7
S214449F70234B05F03DFB051E4FF000024FF0804397
S214449F8018BF0125DDE902013CE000BFAFF30080C5
S214449F90FCA9F1D24D62703FFCA9F1D24D62603FFC
S214449FA0FCA9F1D24D6260BF399D52A246DF913F73
S214449FB0407EFCF8F14B7B40E3A59BC420B0D23FE7
S214449FC0578C22C76075B53FFCA9F1D24D62903FCD
S214449FD07B14AE47E17AC4BF9A9999999999E93F17
S214449FE0E00D422000004940000059400000244053
S214449FF0000024C0587B460000004E400000084045
S21444A0000000344005F0F4FA0C9B00280CBF2846A8
S21444A010681C184405F006F8D4E9AA2304F0B6FEF2
S21444A02000227B4B05F0EEFA0022D4E996890028FC
S21444A03000F0028100234046494605F0C5FA08B1BF
S21444A040C4E99CAB734E0023734C0022C6E9963495
S21444A0500023724CC6E99834D6E99C45704B20469A
S21444A060294605F0BBFA60B120462946DDE90423BB
S21444A070C6E99A2356A3D3E9002304F087FEC6E92B
S21444A0809C010023644CC6E9A8344FF0000ADFF86C
S21444A0908CB100E154465D463FE65F4B49E64EA32D
S21444A0A0D3E900234046494605F098FA00283FF491
S21444A0B061AE204629464AA3D3E9002304F064FE51
S21444A0C056E6DDE9000105F0C7FA03283FF679AE07
S21444A0D0DFE800F002191D1900220023D8E9140114
S21444A0E005F086FA00283FF46CAE00224A4B204620
S21444A0F0294605F069FA78BB0022494B2046294692
S21444A10005F062FA40BB00224FF080431AE000227A
S21444A1100023D8E9140105F06BFA00283FF451AE49
S21444A1200022404B3046394605F06CFA00283FF48E
S21444A13048AE0022384B2046294605F045FA40B939
S21444A1400022374B2046294605F03EFA00283FF4C5
S21444A15038AECDE9004534E600234FF080442EE681
S21444A16094F87932012BD4E900010BD100222E4B0E
S21444A17005F034FA18B1022384F879322BE6C4E9A0
S21444A180AAAB28E618A3D3E9002305F045FA08B19C
S21444A1900123F1E70022204BC4E9AA231BE600244E
S21444A1A0224D2EE60024224D2BE611A5D5E9004586
S21444A1B049E611A5D5E9004545E600241D4D93E63C
S21444A1C00FA5D5E90045B1E60FA5D5E90045ADE6AE
S21444A1D07B14AE47E17A743FFCA9F1D24D6280BF4E
S21444A1E0FCA9F1D24D62803F0000000000C06240EE
S21444A1F0FCA9F1D24D62603FFCA9F1D24D6260BF2A
S21444A200FCA9F1D24D62903F7B14AE47E17AC4BFBD
S21444A21000001040E00D42200000F03F00408F4018
S21444A2200000084000005940000049C00000244097
S21444A230000024C000004E40BF4B4046494605F04F
S21444A240C3F9002800F03987D4E99A23D4E91001E9
S21444A25005F0D8F9002800F02687D4E99867A8A323
S21444A260D3E900233046394604F046FF02460B46FF
S21444A2703046394604F088FD06460F46A2A3D3E985
S21444A280002305F0ABF9002840F00387C4E998673B
S21444A290AA4BD3E998ABA9490022A94BD1E94A0174
S21444A2A004F02AFF0022A74B04F026FF00220446AF
S21444A2B00D46A14BDDE9000105F086F90C9B00280C
S21444A2C04FF000022046294608BF1E469E4B18BF44
S21444A2D04FF0FF3605F0A0F9002840F0F48600223F
S21444A2E000232046294605F079F908B100240025C4
S21444A2F0304604F097FE22462B4604F0FDFE8F4B74
S21444A30004460D46D3E9906732463B4604F03CFD8E
S21444A31000228E4B8046894605F07EF900220028AE
S21444A32000F0D586894B3046394604F02FFD044666
S21444A3300D46824B002220462946C3E99045824B6F
S21444A34005F06AF9002840F0D28600220023204611
S21444A350294605F043F908B10024002500224FF0B1
S21444A3608043DDE90E0105F02FF9002800F0C3868E
S21444A37072490022764BD1E9140104F0BDFE06462C
S21444A3800F4663A3D3E9002305F046F9002840F0BE
S21444A390BA86002200233046394605F01FF908B134
S21444A3A000260027DFF89481C8E9B045DDE9043487
S21444A3B0D8E90401C8E9A434DDE92834C8E9A0672B
S21444A3C0C8E9AC34C8E9BC67D8E94C23C8E9AEABA5
S21444A3D004F0DCFC50A3D3E9002304F08DFE0446CD
S21444A3E00D464FA3D3E90023D8E94E0104F084FE7A
S21444A3F002460B462046294604F0C8FC4AA3D3E945
S21444A400002304F0A3FFD8E95023CDE92201D8E97C
S21444A410060104F0BBFC40A3D3E9002304F06CFE21
S21444A42004460D463EA3D3E90023D8E9520104F07E
S21444A43063FE02460B462046294604F0A7FC3AA390
S21444A440D3E9002304F082FFD8E95423CDE9100170
S21444A450D8E9080104F09AFC2FA3D3E9002304F0BA
S21444A4604BFE04460D462EA3D3E90023D8E95601F5
S21444A47004F042FE02460B462046294604F086FC7B
S21444A48029A3D3E9002304F061FFDDE91023CDE9D5
S21444A49012011046194604F02FFE04460D46DDE927
S21444A4A012231046194604F027FE02460B46204661
S21444A4B0294604F06BFC09F05DFE002200230446A6
S21444A4C00D4605F081F848B922462B46DDE92201BF
S21444A4D004F03CFF09F0F0FB04460D4620462946AE
S21444A4E0D8E94423CDE9242311A3D3E9002304F077
S21444A4F003FE02460B46DDE9240104F045FC29E050
S21444A5009A9999999999A93F7B14AE47E17A843FE1
S21444A510000000000088A340FCA9F1D24D62603FD1
S21444A520FEF2469F2892AF3F1F94D22C39CFB03FBD
S21444A530F8C1631ADCA54C400000F03FE00D422011
S21444A5400000B03F000054C000408F400000084068
S21444A55000005940D8E90A34CDE92A01CDE9263429
S21444A560DDE92601D8E95A2304F010FCB8A3D3E960
S21444A570002304F0C1FD04460D46B7A3D3E90023E7
S21444A580D8E95C0104F0B8FD02460B46204629464D
S21444A59004F0FCFBB2A3D3E9002304F0D7FE002268
S21444A5A00023CDE92C01DDE9000105F00DF806464F
S21444A5B0002840F0AD8500224FF08043DDE90001DD
S21444A5C005F002F858B9CA4B0022DDE9000104F050
S21444A5D0FBFF0C9B00280CBF1E464FF0FF360022A4
S21444A5E0C44BDDE9020104F087FD9FA3D3E90023B1
S21444A5F004F0ACFE9EA3D3E9002304F07DFD0022C4
S21444A600BD4B04F079FD9CA3D3E9002304F09EFEE1
S21444A61004460D46304604F005FD02460B462046E9
S21444A620294604F069FD02460B46CDE90823B34BA0
S21444A630D3E9924522462B4604F0A6FB06460F462F
S21444A6408FA3D3E9002304F0E7FF002800F06385D6
S21444A650204629468AA3D3E9002304F097FBCDE994
S21444A6600801A64CDDE90823DDE90801C4E9922384
S21444A670D4E95E2304F08AFB75A3D3E9002304F0EF
S21444A6803BFD06460F4680A3D3E90023D4E9600188
S21444A69004F032FD02460B463046394604F076FB5B
S21444A6A07BA3D3E9002304F051FE02460B46CDE9D2
S21444A6B00423D4E9622304F067FB00228D4B04F0A4
S21444A6C01BFDD4E9642304F05FFB02460B46CDE948
S21444A6D01423D4E9662304F057FB0022854B04F088
S21444A6E00BFDD4E9682304F04FFB02460B46CDE944
S21444A6F01623D4E96A2304F047FB00227D4B04F07A
S21444A700FBFCD4E96C2304F03FFB63A3D3E90023AA
S21444A710CDE92E01DDE9040104F0EEFC06460F46C1
S21444A7205FA3D3E90023DDE9140104F0E5FC3246D7
S21444A7303B4604F02BFB804689465BA3D3E90023C3
S21444A740DDE9160104F0D8FC02460B46404649466D
S21444A75004F01CFBDDE92E2304F018FB54A3D3E9D4
S21444A760002304F0C9FCD4E96E23CDE91801104651
S21444A770194604F00BFBDDE9182304F007FBD4E983
S21444A780322304F003FB4CA3D3E9002304F0B4FCC7
S21444A790804689464AA3D3E90023D4E9700104F0ED
S21444A7A0ABFC02460B464046494604F0EFFA804668
S21444A7B0894645A3D3E90023D4E9360104F09CFC3A
S21444A7C002460B464046494604F0DEFA40A3D3E927
S21444A7D0002304F0BBFD02460B46CDE91A23D4E918
S21444A7E0722304F0D3FA1AA3D3E9002304F084FCBA
S21444A7F08046894638A3D3E90023D4E9740104F09B
S21444A8007BFC02460B464046494604F0BFFA34A356
S21444A810D3E9002304F09AFDD4E90023CDE93001BE
S21444A820DDE9040104F0B0FA0022354B04460D4637
S21444A83004F0F2FE002840F08184204629462AA3EC
S21444A840D3E9002304F0CAFE5CE000BFAFF3008007
S21444A850FCA9F1D24D62603FFEF2469F2892AF3F7C
S21444A8601F94D22C39CFB03F000000000020AC40EB
S21444A8705C8FC2F528DC2740B46155D0CC38FB3F0A
S21444A8809A9999999999D93FB428207983A6BA3F39
S21444A89054434F56A8ACBB3F9A99999999996340AB
S21444A8A09A99999999996A40CDCCCCCCCCCC3540E0
S21444A8B0E3F36EFB79D0E33E277845D92444D93F69
S21444A8C0FB50D7647BD71C403043BB3975F10440FA
S21444A8D06D0D4BFEC9AF1840EBF33CDE4AA2813FF8
S21444A8E0E9C8B5C771D3893F0000000000409FC047
S21444A8F00000F03F00408F4000004E40E00D4220F4
S21444A90000409F40002840F02C840022C04B204644
S21444A910294604F081FE002800F014840022BC4B33
S21444A9202046294604F030FA80468946B94CDDE98B
S21444A9300401D4E9762304F027FA0022B64B04F047
S21444A940DBFBD4E9782304F01FFA02460B46CDE934
S21444A9501C23D4E97A2304F017FA0022AE4B04F001
S21444A960CBFBD4E97C2304F00FFA02460B46CDE930
S21444A9701E23D4E97E2304F007FA0022A64B04F0F3
S21444A980BBFBD4E9802304F0FFF987A3D3E9002373
S21444A990CDE93201DDE91C0104F0AEFB32463B460C
S21444A9A004F0F4F906460F4681A3D3E90023DDE913
S21444A9B01E0104F0A1FB02460B463046394604F01D
S21444A9C0E5F9DDE9322304F0E1F97BA3D3E900237A
S21444A9D004F092FBD4E9942304F0D6F902460B46DD
S21444A9E0CDE93823D4E9822304F0D0F974A3D3E91B
S21444A9F0002304F081FB06460F4673A3D3E90023E5
S21444AA00D4E9840104F078FB02460B4630463946C6
S21444AA1004F0BCF96EA3D3E9002304F097FCD4E910
S21444AA208623CDE90A011046194604F0AFF9DDE95C
S21444AA300A2304F0ABF9D4E93A2304F0A7F966A351
S21444AA40D3E9002304F058FB06460F4664A3D3E933
S21444AA500023D4E9880104F04FFB02460B463046F7
S21444AA60394604F093F906460F465FA3D3E900231C
S21444AA70D4E93E0104F040FB02460B4630463946D4
S21444AA8004F082F95AA3D3E9002304F05FFC0022C1
S21444AA90624BD4E91467CDE920013046394604F0C8
S21444AAA09DFD002840F0678300225C4B30463946C3
S21444AAB004F06AF950A3D3E9002304F01DFB0022F6
S21444AAC0574B04460D4604F09DFD08B10024544DF2
S21444AAD04BA3D3E90023DDE9200104F00DFB00225B
S21444AAE0504B83468A4604F079FD0690002840F091
S21444AAF06B8300224C4B5846514604F08DFD00288B
S21444AB0040F067830AF1004A404649463EA3D3E9EB
S21444AB10002304F0F1FADDE9302304F037F98046E7
S21444AB2089465A4653462046294604F0E5FA4246A4
S21444AB304B4604F02BF902460B46CDE90623002289
S21444AB403A4B04F069FD002840F048830022384B15
S21444AB50DDE9060104F042FD18B10023344CCDE98A
S21444AB6006342C4CD4E92023DDE90E01CDE9342308
S21444AB7000224FF0804304F027FD002205460028BB
S21444AB8000F02F83264BDDE9340104F01DFD002838
S21444AB9000F04F830022224BD4E9220104F014FD36
S21444ABA0002800F0468345E09A99999999996A4015
S21444ABB0CDCCCCCCCCCC3540E3F36EFB79D0E33E65
S21444ABC0FCA9F1D24D62603F5ED817C2038C9E3F0B
S21444ABD06F216A9B4B52A13F2ED7D19C0A49373FDF
S21444ABE07119ABB745FF1F40ECBC164D8E930F4012
S21444ABF01988C921F33610409A9999999999C93F69
S21444AC00CDCCCCCCCCCCEC3F3B08AA2A23DCA63F0C
S21444AC1000004940E00D422000408F4000001440B0
S21444AC200000F03F00003EC000003E40000054409C
S21444AC30000054C0304639460024A9A3D3E9002373
S21444AC4004F084FB0022AA4B04F0E6FC002800F043
S21444AC50F182A84DDFF8B082D8E91E23CDE90C2353
S21444AC60DDE90C010022A44B04F0AEFC002840F0C1
S21444AC70E38222462B46C8E9A623C8E9BE45DDE959
S21444AC8000343246C8E9B634DDE902013B4604F0F6
S21444AC907BF80022994BCDE90E013046394604F044
S21444ACA02BFA02460B460020954904F06DF8002224
S21444ACB0944B0C460546934E04F090FC00280BBF7C
S21444ACC0284600202146314687A3D3E9002304F0D2
S21444ACD013FA8D4B82468B4693F87C22D3E91601B1
S21444ACE00AB1C3E98A01D3E98A23CDE9022304F0F1
S21444ACF04BF8002280468946824B2846214604F07B
S21444AD006DFC002840F09B8204F1004442464B46CA
S21444AD105046594604F062FC002840F09382284688
S21444AD20214671A3D3E9002304F0E6F942464B4694
S21444AD3006460F4604F070FC08B946464F4632466F
S21444AD403B46DDE9020104F021F86F4B0A46CDE9A3
S21444AD5002010146C3E9A212C3E9BA1293F87D225E
S21444AD60D3E918010AB1C3E98C01D3E98C89424678
S21444AD704B4604F009F806460F4602460B46504634
S21444AD80594604F02BFC88B92846214656A3D3E9F5
S21444AD90002304F0B1F982468B4602460B46304601
S21444ADA0394604F01BFC08B9B246BB4652465B46DD
S21444ADB04046494603F0EAFF534C82468B460022FF
S21444ADC0002300264C4FC4E9B823D4E91C010022D2
S21444ADD0494BC4E9B2AB04F0F7FB68B932463B468C
S21444ADE0DDE90C0104F0F0FB30B932463B46D4E9C9
S21444ADF0280104F0E9FB08B1C4E9B867424C0022D4
S21444AE003D4BD4E92A0104F0DFFBA0B900223A4BBB
S21444AE10D4E92C0104F0D8FB68B90022364BD4E9B7
S21444AE202E0104F0D1FB30B90022334BD4E9300173
S21444AE3004F0CAFBA0B1DFF8D08000220023D8E992
S21444AE401A452046294604F0BFFB38B900224FF085
S21444AE5080432046294604F0B7FB08B1C8E9B867E2
S21444AE600022254BDDE9340104F0AEFB48B9264CFC
S21444AE700022214BD4E9220104F0A6FB002800F06E
S21444AE80E481214BC3E9B8671F4CDDE90023D4E9CC
S21444AE905889C4E94223404600221C4B494604F0E4
S21444AEA02BF906460F460022194BDDE92A0104F029
S21444AEB023F902460B463046394603F067FF0246FE
S21444AEC00B46DDE92C0103F05FFF07A3D3E900231B
S21444AED004F012F9DDE9242303F058FF1AE000BF1A
S21444AEE0CDCCCCCCCCCC0C40FCA9F1D24D62603F4E
S21444AEF00000E03F000054C00000F03F00001A404D
S21444AF000000794000806140E00D4220000014407B
S21444AF1000005940DDE92823C4E94401C4E9462336
S21444AF20DDE93623D4E94A01C4E9482300229E4B8E
S21444AF3004F0E2F8DDE90E2303F028FFD4E9042305
S21444AF40C4E94A01C4E94C23DDE92223DDE92A01A8
S21444AF50C4E94E23D4E90623C4E95023DDE910238B
S21444AF60C4E95223D4E90823C4E95423DDE912236F
S21444AF70C4E9562382A3D3E9002304F0BDF842462D
S21444AF804B4603F003FFDDE92623C4E95801C4E930
S21444AF905A23DDE92C23C4E95C23DDE90823C4E90C
S21444AFA05E23DDE90423C4E96023C4E96223DDE9C2
S21444AFB01423C4E96423C4E96623DDE91623C4E9FB
S21444AFC06823C4E96A23DDE92E23C4E96C23DDE95A
S21444AFD01823C4E96E23D4E93423C4E93223DDE9D3
S21444AFE01823C4E93423DDE91A23C4E97023D4E9D9
S21444AFF03823C4E93623DDE91A23C4E93823C4E9EF
S21444B0007223DDE93023C4E97423DDE90623C4E969
S21444B0109423DDE90423C4E97623DDE91C23C4E94B
S21444B0207823C4E97A23DDE91E23C4E98CABC4E95A
S21444B0307C23C4E97E23DDE93223C4E98023DDE9A9
S21444B0403823C4E98223DDE90A23C4E98423C4E916
S21444B0508623D4E93C23C4E93A23DDE90A23C4E938
S21444B0603C23DDE92023C4E98823D4E94023C4E90A
S21444B0703E23DDE92023C4E94023DDE90223C4E975
S21444B0808A230023A4F87A32A4F87C323BB0BDE885
S21444B090F08FC4E998ABC4E996ABC4E99AABC4E96B
S21444B0A09CABFFF7F5B80022404BC4E99823002236
S21444B0B03F4BC4E9A823FEF7E8BF4FF0000A4FF021
S21444B0C0000BFFF7E8B80024384DFFF711B9394BA9
S21444B0D04046494604F082FA00283FF42AA9002252
S21444B0E0354B3046394603F04FFEFFF720B900246F
S21444B0F02E4DFFF733B922462B465046594603F0A9
S21444B10045FEFFF73CB920A7D7E90067FFF74AB9E1
S21444B1100026FFF764BA1EA3D3E900233046394617
S21444B12004F05CFA00283FF49CAA204629461AA359
S21444B130D3E9002303F028FEFFF791BA00241F4DFD
S21444B140FFF7ECBB00221E4B2046294604F05AFA71
S21444B15058B900221B4B2046294603F017FEFFF73A
S21444B160E3BB0FA5D5E90045F3E74FF000084FF0E1
S21444B1700009FFF7DBBB00240025A9E4AFF30080F9
S21444B180FCA9F1D24D62603F000000000088A34055
S21444B1909A9999999999E9BF9A9999999999E93F68
S21444B1A00000000000409FC00000EE3F00408F407B
S21444B1B00000F03F000008C00000084000409F40E8
S21444B1C0000049C0000049404FF0000BDFF8ACA037
S21444B1D09AE4DDF818B0DFF8A8A095E40023244CE0
S21444B1E0BDE40023DDE9000104F0EEF90446E0B9CD
S21444B1F000224FF08043DDE9000104F0E5F9B0B9E0
S21444B2001C4B0022DDE9000104F0DEF900280C9B0B
S21444B21018BF4FF0FF33184603F004FFDDE906235A
S21444B22003F06AFF04460D4614E52846F4E7204634
S21444B230F2E7002400250DE5002200231BE5002547
S21444B2400D4C63E556465F4679E50022094BD4E942
S21444B250240104F0B9F900283FF416AE0022054B49
S21444B260D4E9260104F0B0F900287FF40AAE0BE6D0
S21444B270000054400000F03F008061C000003E40A3
S21444B28000003EC0034B40F20112A3F87A22A3F812
S21444B2907C227047E00D422038B5624B624C1868F9
S21444B2A003F0D2FE614B1D68C4E90001284603F052
S21444B2B0A9FE5F4BC4E91A01186803F0C5FE5D4B4E
S21444B2C0C4E91401186803F0BFFE5B4BC4E90401EB
S21444B2D0186803F0B9FE594BC4E90601186803F030
S21444B2E0B3FE574BC4E90801186803F0ADFE554B4E
S21444B2F0C4E90A01187803F085FE534BC4E92A01D1
S21444B300187803F07FFE514BC4E92C01187803F0FB
S21444B31079FE4F4BC4E92E01187803F073FE4D4B6B
S21444B320C4E93001187803F06DFE4B4BC4E91C01A8
S21444B330187803F067FE494BC4E91E01187803F0F9
S21444B34061FE474BC4E92001187803F05BFE454B89
S21444B350C4E92201187803F055FE434BC4E924019E
S21444B360187803F04FFE414BC4E92601187803F0E1
S21444B37049FE3F4BC4E92801186803F065FE3D4B7F
S21444B380C4E90201186803F03DFE3B4BC4E90C01D6
S21444B390186803F037FE394BC4E91201186803F005
S21444B3A031FE374BC4E90E01186803F04DFEC4E97C
S21444B3B01601002D2BD1334B186803F045FE324B53
S21444B3C0C4E90201186803F01DFE00222F4BC4E9AD
S21444B3D012232F4BC4E90C01186803F013FE2D4BBF
S21444B3E0C4E90E01186803F02FFE2B4BC4E916017E
S21444B3F0186803F029FEC4E91801284B1B7873B972
S21444B400274B186803F020FEC4E9100138BD023DFE
S21444B410012DF2D800220023C4E90C23EDE70020D6
S21444B4200021F1E7681E4020E00D4220541C4020D5
S21444B430741C4020181F4020381F4020FC1E40200B
S21444B440081F40207C1740207B1740207A17402056
S21444B450791740204E1F40204D1F4020241C40207A
S21444B460231C4020221C4020211C40204C1F4020EE
S21444B470981F4020801F4020501F4020681F4020B7
S21444B4808C1F4020B41D4020BC1D4020000044407A
S21444B4908C1D4020A81D4020A41D4020601840203C
S21444B4A0641E40202DE9F04F644C85B0644EDFF8AE
S21444B4B0F0A1DFF8F0B1D4E9000104F015F9614BCE
S21444B4C080461860D4E9060104F00EF93060D4E9E9
S21444B4D0040104F009F95C4B1860D4E9020104F055
S21444B4E003F95A4A5A4B074610601860D4E91201C9
S21444B4F004F0FAF8CBF80000CAF800008146D4E914
S21444B500160104F0D1F8534905460860D4E91801F9
S21444B51004F0CAF850490870D4E91E0104F0E4F86F
S21444B5204E490860D4E91C0104F0DEF84C49086032
S21444B530D4E91A0104F0D8F84A49086038464A491A
S21444B5400968039104F0EAFB404A414B02961646CA
S21444B5501C460399CDF804A060B111601960434FAE
S21444B5604846394604F0DAFBB8B1019BCBF8007084
S21444B5701F6019E001F1004A3846514604F0B0FB1A
S21444B58020B1C6F800A0C4F800A0E8E75146384603
S21444B59004F0A6FB0028E2D0F5E7354F4846394686
S21444B5A004F09EFB0028E0D1324B334F1B68002B3F
S21444B5B030D1324B25F002051968012D2ED1404674
S21444B5C004F0E8F8386039682D4A2E4B116019604B
S21444B5D02D490978012904BF002111602B4A1278AD
S21444B5E0012A04BF00221A60294B1B78012B04BF92
S21444B5F000233360274B1B78012B04BF00232360B2
S21444B600254B1B78012B02BF00233360236005B013
S21444B610BDE8F08F012B03D1204BCBE73960D2E74E
S21444B620022B02D1C7F80080CDE7032BCBD10023F1
S21444B630029A1360194B1B683B60C4E760104220B3
S21444B640581B4020881F4020B0174020B419402083
S21444B65010194020581C4020A4174020A017402012
S21444B6609C17402098174020A817402000004843C5
S21444B670000048C3541C4020901F4020B41D402066
S21444B680A819402004194020241C4020231C402094
S21444B690221C4020211C40204C1F4020981F402044
S21444B6A088184020A0184020294B1B68012B0FD037
S21444B6B0284B1B88012B0BD0274B1968012907D030
S21444B6C0264B1B68012B03D0254B1B78012B03D13B
S21444B6D0244B02221A600CE0234B1A68234B012A9F
S21444B6E01B680FD11F4A1068032827D1002B2AD184
S21444B6F013601F4B1B78013B012B27D8194B0322A1
S21444B7001A607047012B08D116490968032912D1DB
S21444B710002AEED1134B0122DCE72AB9114A1268FB
S21444B72012B9104B0322D5E7002BE2D10D4B1B6810
S21444B730012BDED1F5E7002AF0D0DAE7012BF3D16E
S21444B7400029E7D0D5E7012BD3D1F9E7704700BFEE
S21444B750601F402000184020881D4020701F402055
S21444B760A4174020541C4020981D40206C1F4020A5
S21444B7702218402008B5FEF719FA144B1B886BB9FB
S21444B780134B144A1B681268134307D1124A1360BA
S21444B790124A1360124A1360124A13600023124A74
S21444B7A001211360114A1360114A1360114A136051
S21444B7B0114A1360114A1360114A1360114A136008
S21444B7C0114A1160114A136008BD00BF001840209A
S21444B7D0601F4020881D40207C1D4020781D40204E
S21444B7E0741A4020781A40205C1C4020041B4020D9
S21444B7F0741D4020701D40206C1D4020681D402054
S21444B800641D4020601D40205C1D4020581D402083
S21444B81008B5FEF735F9044B1B68012B1EBF034BD6
S21444B82000221A6008BD00BF881D4020041B40202B
S21444B83008B5FEF725F9064B1B68012B1EBF054BC2
S21444B84000221A60044B1A68044B1A6008BD00BFF5
S21444B850601F40205C1C4020501F4020701C40202D
S21444B860F8B5134A0223134F1360134E134A3B6032
S21444B870136033600123124D124C2B602360FEF795
S21444B88095F9114B1B8893B9104B114A1B681268E3
S21444B8901343104A1268134309D10F4B1B7833B92C
S21444B8A003223B6033602B6023600C4B1A60F8BD68
S21444B8B0601B40207C1D4020781D4020581C4020A2
S21444B8C05C1C4020041B402000184020601F402081
S21444B8D0881D4020701F4020A4174020541C402040
S21444B8E008B5174B186804F023FA164B164A186026
S21444B8F001231360154A1360154A1360154A1168EC
S21444B900154A1160154A16491370164A1370164A9A
S21444B9101370164A1370164A1370164A1370002290
S21444B9200A7015490A7015490B7015490B7015496C
S21444B9300B7015490B70154B1A70154B1A7008BDD1
S21444B940581B4020A4194020A0194020901940209C
S21444B950F4184020581C4020FC184020C0194020B1
S21444B960C51840201C194020B01940200E1940200C
S21444B9703519402034194020C41840209D184020D2
S21444B980991840209A184020841840208018402057
S21444B9908118402000230A4A15211370094A13705F
S21444B9A0094A11700621094A1370094A1370094A54
S21444B9B01170094A13701822084B1A70704700BF5A
S21444B9C026194020251940202419402023194020B8
S21444B9D02219402021194020201940201F194020B8
S21444B9E008B5FFF77DFFFFF7D5FFFFF75DFEFFF7CE
S21444B9F053FCFEF76DF9FFF755FD0D4B1B681BB95D
S21444BA00BDE80840FFF704BF012B03D1BDE808405A
S21444BA10FFF70EBF022B03D1BDE80840FFF720BF57
S21444BA20032B03D1BDE80840FFF7A4BE08BD00BF02
S21444BA30541C4020F8B5174B174C1E68174D66B17A
S21444BA40012E19D000210020F5F750FF00210120D7
S21444BA50F5F74CFF00232B700CE02678002EF1D12E
S21444BA6000213046F5F742FF0D490120F5F73EFF29
S21444BA7001232E702370F8BD2F78002FE2D1084999
S21444BA803846F5F733FF00213046F5F72FFF2E7082
S21444BA902770F0E7541C4020E4174020E517402068
S21444BAA00000C8422C4B2D491A6810B542B90A68A2
S21444BAB0012A05D12A4802602A4802602A480260C0
S21444BAC02A4A502010602A4A2A4810602A4A126895
S21444BAD01A602A4B1B780B60294B1C6874B9294B97
S21444BAE00021186804F0F2F888B1274B07221A6040
S21444BAF00122264B1C60264B1A6008E0012C07D115
S21444BB000223214A1360214A1360214A136010BD60
S21444BB10022C0FD11B4B0021186804F0D7F80028DC
S21444BB20F5D0194B03221A600022184B1A60184BA2
S21444BB301C60ECE7032CEAD1124B0021186804F091
S21444BB40C5F80028E3D0104B04221A6001220F4B9C
S21444BB501A6002220E4BCFE7381B4020341B40208D
S21444BB60441B4020481B4020501B4020301B402094
S21444BB702C1B4020000048C2F8194020161E4020C6
S21444BB80581C4020741C4020401B40203C1B402036
S21444BB90601B40200000000038B5174B00211C688D
S21444BBA0204604F09DF808B104F10044134D2046A5
S21444BBB02C6003F049FA0CA3D3E9002303F0C6FB38
S21444BBC00BA3D3E9002303F097FA00220C4B03F0AF
S21444BBD093FA0C4B002203F0B9FB03F085FD0A4BA5
S21444BBE06860186038BD00BF5C8FC2F528DC27400B
S21444BBF0B4A766033D39FB3F681E4020F42040202E
S21444BC0000004E4000408F40741C4020074B1922D1
S21444BC101A600922064B1A600123064A1360064A34
S21444BC201360064B064A1A60704700BFA41B4020A8
S21444BC30A01B40209C1B4020981B4020941B402067
S21444BC40EFAB030008B5074B186803F053FE064BEA
S21444BC500649186004F04EF810B1054B01221A70DC
S21444BC6008BD00BF101E40204C1840200000F04184
S21444BC7050184020034B044A9B6FC3F309231370A8
S21444BC80704700BFC083402028184020084B1B78CC
S21444BC90013B022B0AD80023064A00211370064AA9
S21444BCA01160064A13700322054B1A60704700BFA2
S21444BCB02218402021184020581B4020201840209D
S21444BCC0541C4020044B054A1B781370013B012B3F
S21444BCD001D8FFF7DBBF70471C1E402022184020C7
S21444BCE0FE28D4BF01300020704770B50022FF23E1
S21444BCF0064ED4B2551C8C4202D3D843C0B270BD53
S21444BD00025D53402A46F35CF3E700BF687B460077
S21444BD100721013008B5FFF7E8FFC0B208BDB0F50B
S21444BD20447F38B5144617D1244D204695F8F4324E
S21444BD30FF2B14BF01330023DBB285F8F432537073
S21444BD401F4A1370FFF7E4FF1E4BC0B285F8F50296
S21444BD5020701870012038BD402818D0B0F5547FA4
S21444BD60F8D1164D204695F8F032FF2B14BF013318
S21444BD700023DAB285F8F0226270134A1360FFF7A4
S21444BD80C7FFC0B2114B85F8F102207014E00B4D8A
S21444BD90204695F8E832FF2B14BF01330023DAB26D
S21444BDA085F8E82262700A4A1360FFF7B1FF094B30
S21444BDB0C0B285F8E90220701860CBE7C083402003
S21444BDC03719402036194020301940202C1940207D
S21444BDD0BC194020B8194020402838B5144616D11E
S21444BDE0254D204695F82033FF2B14BF01330023FE
S21444BDF0DAB285F820236270204A1360FFF788FF82
S21444BE001F4BC0B285F821032070186005E0B0F5DA
S21444BE10547F04D0B0F5447F17D0012038BD164D6A
S21444BE20204695F82833FF2B14BF01330023DAB29B
S21444BE3085F828236270134A1360FFF769FFC0B27F
S21444BE40114B85F829032070DFE70B4D204695F803
S21444BE502C33FF2B14BF01330023DBB285F82C337D
S21444BE6053700A4A1370FFF753FF094BC0B285F864
S21444BE702D0320701870D0E7C08340201819402046
S21444BE8014194020C0184020BC184020C718402031
S21444BE90C6184020402838B5144617D1254D2046AC
S21444BEA095F82033FF2B14BF01330023DAB285F80C
S21444BEB05C236270204A1360FFF72AFF1F4BC0B210
S21444BEC085F85D0320701860012038BDB0F5547FB6
S21444BED018D0B0F5447FF7D1164D204695F8683310
S21444BEE0FF2B14BF01330023DBB285F8683353704D
S21444BEF0134A1370FFF70CFFC0B2124B85F8690360
S21444BF00207014E00B4D204695F86433FF2B14BF85
S21444BF1001330023DBB285F8643353700A4A137046
S21444BF20FFF7F6FE094BC0B285F86503207018701B
S21444BF30CAE700BFC0834020A8184020A418402069
S21444BF409C1840209B184020981840209718402062
S21444BF50402838B5144616D1254D204695F86C33FE
S21444BF60FF2B14BF01330023DAB285F86C236270CA
S21444BF70204A1360FFF7CCFE1F4BC0B285F86D0312
S21444BF802070186005E0B0F5547F04D0B0F5447FC7
S21444BF9017D0012038BD164D204695F87833FF2B30
S21444BFA014BF01330023DAB285F878236270134A4B
S21444BFB01360FFF7ADFEC0B2114B85F879032070CD
S21444BFC0DFE70B4D204695F87433FF2B14BF01333F
S21444BFD00023DBB285F8743353700A4A1370FFF7B4
S21444BFE097FE094BC0B285F8750320701870D0E7E9
S21444BFF0C0834020901840208C1840207C18402055
S21444C000781840208318402082184020502870B565
S21444C0100546144616D18C4A92F8AC31FF2B14BF11
S21444C02001330023D9B282F8AC11884A21711360D7
S21444C03040F285339D4200F0DD80162D00F0F080FE
S21444C040012070BD642826D065283BD032284FD0C6
S21444C050702863D0712877D0332800F08C806A2803
S21444C06000F09F80B0F5617FE2D1774D204695F889
S21444C070F832FF2B14BF01330023DBB285F8F832C5
S21444C0805370734A1370FFF743FEC0B2714B85F882
S21444C090F90220706DE06C4E204696F8B032FF2BC5
S21444C0A014BF01330023DBB286F8B03253706A4AB9
S21444C0B01370FFF72DFE694BC0B286F8B4022070A9
S21444C0C01870B5E7604E204696F81833FF2B14BF19
S21444C0D001330023DBB286F818335370604A13707A
S21444C0E0FFF716FEC0B25F4B86F81C032070E7E7E6
S21444C0F0554E204696F8C832FF2B14BF0133002312
S21444C100DBB286F8C8325370574A1370FFF700FE06
S21444C110C0B2564B86F8C9022070D1E74A4E204634
S21444C12096F8BC32FF2B14BF01330023DBB286F8EB
S21444C130BC3253704E4A1370FFF7EAFDC0B24D4B03
S21444C14086F8BD022070BBE73F4D204695F80C3379
S21444C150FF2B14BF01330023DBB285F80C33537036
S21444C160454A1370FFF7D4FD444BC0B285F80D031F
S21444C1702070187064E7344D204695F83033FF2B12
S21444C18014BF01330023DBB285F8303353703C4A86
S21444C1901370FFF7BDFDC0B23A4B85F831032070EB
S21444C1A0E7E7294D2046D5F8E032D5F8E022C3F338
S21444C1B0C733FF2B14BF01330023DBB263F3D632FD
S21444C1C0C5F8E0226370D5F8E0322F4AC3F3C7338C
S21444C1D01360FFF79DFDB5F8E232C0B22B4A60F318
S21444C1E0CE13A5F8E2322070B5F8E232C3F3C71393
S21444C1F0136025E7144D2046254A95F84833FF2B0F
S21444C20014BF01330023DBB285F8483363701370E0
S21444C210FFF77EFDC0B21F4B85F849032070A8E7A0
S21444C2200949B1F89422C2F34313013303F00F03D0
S21444C23063F34812A1F894226370B1F89432164A14
S21444C240C3F34313D4E700BFC0834020281C4020D8
S21444C2502819402027194020781940207919402071
S21444C2600C1940200D194020C2194020C119402005
S21444C2705919402058194020E9184020E818402011
S21444C2801E1940201D1940206C1940206819402072
S21444C290B5184020B4184020C01A40200F28D4BFF8
S21444C2A001300020704770B50022FF23074ED4B2F9
S21444C2B0551C8C4205D3DB4383EA131303F00F006B
S21444C2C070BD025D53402A46F35CF0E7687C460046
S21444C2D00721013008B5FFF7E6FFC0B208BDB0F548
S21444C2E0AE6F70B5054614461AD1C04D204695F833
S21444C2F009221309013363F3071203F00F0385F889
S21444C3000922BB4A1360FFF7E3FF95F80A3260F34D
S21444C310030300F00F0085F80A32B64B1860C0E0FD
S21444C320B0F5B06F1DD0B0F5B26F35D1AF4D2046E5
S21444C33095F81A2202F00F03013363F3030203F065
S21444C3400F0385F81A22AC4A1360FFF7C1FF95F82D
S21444C3501A3260F3071300F00F0085F81A32A74B21
S21444C360DCE7A24D2046B5F81022C2F3831301330E
S21444C37063F3891203F00F03A5F81022A04A136052
S21444C380FFF7A6FF95F8113260F3850300F00F001F
S21444C39085F811329B4BC1E740F29553984222D020
S21444C3A040F28553984258D050287CD0512835D1F5
S21444C3B08E4D204695F8342202F00F03013363F382
S21444C3C0030203F00F0385F834228F4A1360FFF705
S21444C3D07FFF95F8343260F3071300F00F0085F8BA
S21444C3E034328A4B9AE7814E204696F81F22C2F38F
S21444C3F08303013303F00F0363F3850286F81F2299
S21444C400834A1370FFF764FF96F8203200F00F005B
S21444C41060F3030386F820327E4B1870602D5DD09F
S21444C420612D35D1714D204695F8442202F00F0314
S21444C430013363F3030203F00F0385F84422764A7C
S21444C4401360FFF745FF95F8443260F3071300F096
S21444C4500F0085F84432714B60E7644E2046D6F8A8
S21444C4602422C2F38333013363F3913203F00F0380
S21444C470C6F824226A4A1360FFF72AFF96F8263243
S21444C48060F3850300F00F0086F82632654B18608B
S21444C490132D3ED0142D57D0152D70D0162D00F0E8
S21444C4A08980012070BD514D204695F82C2202F01B
S21444C4B00F03013363F3030203F00F0385F82C22C2
S21444C4C0594A1360FFF704FF95F82C3260F30713BC
S21444C4D000F00F0085F82C32544B1FE7434D20469E
S21444C4E095F83C2202F00F03013363F3030203F092
S21444C4F00F0385F83C224E4A1360FFF7E9FE95F891
S21444C5003C3260F3071300F00F0085F83C32494B89
S21444C51004E7364D2046B5F84E22C2F38313013362
S21444C52063F3891203F00F03A5F84E22424A1360C0
S21444C530FFF7CEFE95F84F3260F3850300F00F0008
S21444C54085F84F323D4BE9E6284D204695F856226D
S21444C55002F00F03013363F3030203F00F0385F87D
S21444C5605622374A1360FFF7B3FE95F8563260F307
S21444C570071300F00F0085F85632324BCEE61B4DBB
S21444C580204695F85E2202F00F03013363F303025C
S21444C59003F00F0385F85E222B4A1360FFF798FEDC
S21444C5A095F85E3260F3071300F00F0085F85E32AC
S21444C5B0264BB3E60D4D2046B5F89422C2F34313FA
S21444C5C0013363F3481203F00F03A5F89422204A7C
S21444C5D01360FFF77DFE95F8953260F3440300F050
S21444C5E00F0085F895321B4B98E600BFC083402069
S21444C5F00C1A4020081A40202C1E4020281E40209A
S21444C600E41D4020E01D4020A01A40209C1A4020F3
S21444C610D7194020D6194020801A40207C1A402042
S21444C620E0194020DC194020B01A4020AC1A4020C3
S21444C630901A40208C1A4020001B4020FC1A4020B0
S21444C640E01A4020DC1A4020C81A4020C41A402071
S21444C650C01A4020BC1A40200D4B0E490E4810B557
S21444C6601C680E4B1A78A2421A460BD10B8801332B
S21444C6709BB2312B0B8008D932230B8001230370E5
S21444C680147010BD00230B80F9E70023F7E700BFC2
S21444C690541D4020941740207C1740208417402087
S21444C6A00D4B0E490E4810B51C680E4B1A78A24224
S21444C6B01A460BD10B8801339BB2312B0B8008D919
S21444C6C032230B8001230370147010BD00230B80AB
S21444C6D0F9E70023F7E700BFB01D4020921740203B
S21444C6E07B174020831740200D4B0E490E4810B54B
S21444C6F01C680E4B1A78A2421A460BD10B8801339B
S21444C7009BB2312B0B8008D932230B800123037054
S21444C710147010BD00230B80F9E70023F7E700BF31
S21444C720A01D4020901740207A17402082174020B2
S21444C7300D4B0E490E4810B51C680E4B1A78A24293
S21444C7401A460BD10B8801339BB2312B0B8008D988
S21444C75032230B8001230370147010BD00230B801A
S21444C760F9E70023F7E700BF841D40208E174020DA
S21444C77079174020811740200D4B0E490E4810B5BE
S21444C7801C780E4B1A78A2421A460BD10B880133FA
S21444C7909BB2312B0B8008D932230B8001230370C4
S21444C7A0147010BD00230B80F9E70023F7E700BFA1
S21444C7B00C1D40208C174020241C4020801740200D
S21444C7C00D4B0E490E4810B51C780E4B1A78A242F3
S21444C7D01A460BD10B8801339BB2312B0B8008D9F8
S21444C7E032230B8001230370147010BD00230B808A
S21444C7F0F9E70023F7E700BF981C40208A1740203B
S21444C800231C40207F1740200D4B0E490E4810B580
S21444C8101C680E4B1A78A2421A460BD10B88013379
S21444C8209BB2312B0B8008D932230B800123037033
S21444C830147010BD00230B80F9E70023F7E700BF10
S21444C840501D402088174020221C40207E17402040
S21444C8500D4B0E490E4810B51C680E4B1A78A24272
S21444C8601A460BD10B8801339BB2312B0B8008D967
S21444C87032230B8001230370147010BD00230B80F9
S21444C880F9E70023F7E700BFCC1C4020861740207A
S21444C890211C40207D1740201D4B1B78012B30D196
S21444C8A01C4B1B78003B18BF01231B4A13701B4BC1
S21444C8B01B78012B27D1174B1B78003B18BF01234D
S21444C8C0174A1370174B1B78012B1ED1114B1B783C
S21444C8D0003B18BF0123144A1370144B1B78012BDA
S21444C8E00CD0134B1B78012B08D0124B1B78012B12
S21444C8F004D0114B1B785A1E534253410F4A1370AF
S21444C90070470023D1E70023DAE70023E3E700BFBC
S21444C9104E1F4020A4174020261C40204D1F402078
S21444C920251C40204C1F4020201C40207C174020C3
S21444C9307B1740207A1740207917402078174020EC
S21444C9400B4B1B68012B09D10A4A11680A4A106826
S21444C95088420ABF094A116013607047022B06D109
S21444C960074B1B68012B02BF044B00221A6070471A
S21444C970541C4020581F4020781F4020701F4020E1
S21444C980601F402038B53E4B1A783E4B1B78134305
S21444C9903ED13D4B1B78013B18BF01233B4A1370E5
S21444C9A03B4B1A683B4B1B6813433B4B14BF01225B
S21444C9B000221A70394B1A78394B1B781343394B7B
S21444C9C014BF012200221A70374B384A1B78013BA9
S21444C9D018BF01231370364B364A1B78003B18BFEA
S21444C9E001231370344B354A1B78003B18BF012390
S21444C9F01370334B1C788CB9324D2B78012B09D1EC
S21444CA00314B1C70314B1C70BDE83840FFF71AB9E7
S21444CA100123C3E7022B23D12C7038BD012CFCD153
S21444CA20284B1B78012B09D1294A1360264A1370D8
S21444CA30FFF7ECF8BDE83840FDF712B8022B03D1F7
S21444CA40BDE83840FDF790B8032BE6D1FEF7C8FFA3
S21444CA50FFF738F9FFF726F8BDE83840FFF79CB8EB
S21444CA60032B02D1FFF706F9D6E7002BD5D1194A96
S21444CA7001211160184A1360BDE83840FDF704B937
S21444CA80DE1D4020DD1D4020141E4020631840203B
S21444CA90881E4020841E402060184020CD1D402023
S21444CAA0CC1D402061184020151E402062184020AE
S21444CAB0161E40205F184020201E40205E1840204E
S21444CAC06518402064184020281B402072184020D7
S21444CAD04C1B4020601B4020581C40207047704729
S21444CAE030B53D4C85B03D48237801A90193019B60
S21444CAF01B020193019A637813440193019B1B0222
S21444CB000193019AA37813440193019B1B0201935A
S21444CB10019AE3781344019323790293029B1B0200
S21444CB200293029A637913440293029B1B02029374
S21444CB30029AA37913440293029B1B020293029A1D
S21444CB40E37913440293237A0193019B1B020193D6
S21444CB50019A637A13440193019B1B020193019A41
S21444CB60A37A13440193019B1B020193019AE37A2F
S21444CB7013440193237B0293029B1B020293029A63
S21444CB80637B13440293029B1B020293029AA37B89
S21444CB9013440293029B1B020293029AE37B1344C0
S21444CBA0029342F21273019342F21373029300F01B
S21444CBB0B0FB04F1100004F1080104F11802082344
S21444CBC014F8015B013B00F8015B11F8015B02F8C5
S21444CBD0015BF5D105B030BDE41042208080800072
S21444CBE00C4A0823002102F1280030B402F108055B
S21444CBF002F12004013B02F8011B05F8011B13F067
S21444CC00FF0304F8011B00F8011BF3D130BCFFF707
S21444CC1067BF00BFE41042204F4BF0B51B688BB093
S21444CC2002934E4B1A6803925A6804929B68059383
S21444CC3042F21273029A9A4200F08980484800F001
S21444CC4013FBFFF7CDFF002346480AAA50F82310EB
S21444CC5002EB83020133082B42F8201CF5D1002353
S21444CC6040480AAA50F8231002EB83020133082BEB
S21444CC7042F8201CF5D102990025039A049B059896
S21444CC80394C00903948264600F0EEFA029B384864
S21444CC901B0E2370029B1B0C6370029B1B0AA37023
S21444CCA0029BE370039B1B0E2371039B1B0C637157
S21444CCB0039B1B0AA371039BE371049B1B0E237205
S21444CCC0049B1B0C6372049B1B0AA372049BE372B3
S21444CCD0059B1B0E2373059B1B0C6373059B1B0A4A
S21444CCE0A373059BE37300F0B6FA013516F8010BFF
S21444CCF000F0DAFA082DF8D11E4D002600F0CBFAE3
S21444CD001D482F4600F0A7FA013617F8010B00F02D
S21444CD10CBFA082EF8D100F0BEFA184B002203F1E5
S21444CD20080703F1100003F118019446013214F881
S21444CD30016B15F801EB082A03F8016B07F801EBC1
S21444CD4000F8016B01F801CBF0D10BB0F0BD0C48F4
S21444CD5000F08AFA77E700BF8080800084808000F5
S21444CD60CA82460010808000E4104220EE824600CC
S21444CD700B834600EC10422015834600F4104220F4
S21444CD80E0824600194A08211948F0B592F8A531C0
S21444CD9000F1100C00F1080500F11807012B9CBFA8
S21444CDA0002382F8D431002310F8014B01391CF8D3
S21444CDB0016B17F801EBB4422E7818BF013344EAEE
S21444CDC0060418BFDBB2764505F8014B1CBF013399
S21444CDD0DBB211F0FF01E7D133B1B2F8BE301BB974
S21444CDE0BDE8F040FFF77CBEF0BD00BF20114220F6
S21444CDF0E41042201FB5144B01A953F820305A1EA4
S21444CE00073312F8010F9A4201F8010BF9D19DF845
S21444CE1004300024502B8DF80C4007D0432B0CD004
S21444CE20422B0DD0552B08BF4FF440040DF105009E
S21444CE3000F04CFA204404B010BD4FF48004F5E7EB
S21444CE404FF40004F2E700BFFC2040202DE9F04FE9
S21444CE505C4D8DB082462B6805F1080806AC09A9DE
S21444CE6063F07C4340462E46A9462B604246082340
S21444CE7016F8017B013B04F8017B9BB210F8017B5A
S21444CE8001F8017B002BF3D1BAF10A0F0BD14146CE
S21444CE904C4C0823FF20013B04F8010B01F8010B1E
S21444CEA09BB2002BF7D1484BC8240021013C03F821
S21444CEB0011BA4B2002CF9D126464449DFF808B138
S21444CEC004F1080380279BB200932B781F4203D1BA
S21444CED098F800301F4248D051F824300DF10C0C1D
S21444CEE0581E073310F801EF98420CF801EBF9D1BD
S21444CEF04FF000038DF814309DF80C30502B59D069
S21444CF00432B59D0422B5AD0552B34D14FF440039F
S21444CF100DF10D00019300F0D9F9019B95F800C07E
S21444CF20184498F800302A4A3B404FEA102E2749C6
S21444CF3018BF082317EA0C0F4FEA104C18BF43F0EB
S21444CF4001030BF806C006F1010C1FFA8CFC0BF823
S21444CF500CE006F1020C1FFA8CFC0BF80C00F01CDB
S21444CF60043680B2B6B20BF800300134009B7F081A
S21444CF70A4B2A342A9D1013508F1010895429FD134
S21444CF80BAF10A0F0FD19DF81A30BDF8182089F867
S21444CF900230A9F800209DF82630BDF8242089F8F0
S21444CFA00A30A9F80820084B002230469A550DB09E
S21444CFB0BDE8F08F0023ABE74FF48003A8E74FF4B7
S21444CFC00003A5E7E410422032224020FC20402003
S21444CFD0EC104220F0B50D4C0822002004F1080560
S21444CFE014F8016B082380210E4202D12F7839426F
S21444CFF001D0013080B2013B49089BB2002BF3D1EB
S21444D000013A013592B2002AEAD1F0BDE41042203A
S21444D0102DE9F04FDFF8B480002685B08346A8F1AA
S21444D020080A3446284B022E4FF080094FF000027F
S21444D03034BF082703272744BFB29AF8001019EADA
S21444D040010F04D198F8001019EA010F2DD053F8B7
S21444D050241001AD481E073110F801CF814205F86F
S21444D06001CBF9D19DF804108DF80C20502914D02A
S21444D070432914D0422915D055291CD14FF44005D4
S21444D0800DF1050000F022F905440F4B00225D45E2
S21444D0900BD1E0B205B0BDE8F08F0025F0E74FF4C1
S21444D0A08005EDE74FF40005EAE701344FEA5909F5
S21444D0B0A4B2A742C1D1013608F101080AF1010A17
S21444D0C0082EB0D1FF20E5E7FC204020EC1042209B
S21444D0D02DE9FF4700240746204EA146022C4FF078
S21444D0E0000834BF4FF0080A4FF0030A336801A91A
S21444D0F05A1E073312F8010F9A4201F8010BF9D170
S21444D1009DF804308DF80C90502B0DD0432B15D041
S21444D110422B16D0552B17D001340436082CDDD1BB
S21444D120FF2004B0BDE8F08700250DF1050000F0AF
S21444D130CDF80544BD420AD1E0B2F2E74FF480058B
S21444D140F3E74FF40005F0E74FF44005EDE708F148
S21444D15001081FFA88F39A45C8D8DDE7FC2040202A
S21444D1602DE9F04FDFF8C490002585B08346A9F139
S21444D17008082C462B4A022D4FF0800A4FF0000137
S21444D18034BF082703272744BFB298F800001AEA9A
S21444D190000F04D199F800001AEA000F32D052F872
S21444D1A024000DF1040C461E073016F801EFB04279
S21444D1B00CF801EBF9D19DF804008DF80C105028BA
S21444D1C018D0432818D0422819D0552820D14FF4D7
S21444D1D040060DF1050000F079F80644124B002194
S21444D1E05E45104A0ED15955E0B21D44297205B029
S21444D1F0BDE8F08F0026ECE74FF48006E9E74FF4ED
S21444D2000006E6E701344FEA5A0AA4B2A742BCD164
S21444D210013509F1010908F10108082DABD1FF20B9
S21444D220E5E700BFFC204020E4104220EC104220FA
S21444D2307047092894BF30303730C0B2704707B5BE
S21444D24001220DF107018DF80700002013F0C8FBFA
S21444D25003B05DF804FB10B5441E14F8010F00B982
S21444D26010BDFFF7ECFFF8E70FB400B5C3B044AA0F
S21444D27002A852F8041B019204F066FC002302A89C
S21444D2808DF805318DF80631FFF7E5FF43B05DF8BC
S21444D29004EB04B070470D2008B5FFF7D0FF0A2012
S21444D2A0BDE80840FFF7CBBF10B504460009FFF7BA
S21444D2B0C0FFFFF7C4FF04F00F00FFF7BAFFFFF705
S21444D2C0BEFF2C20BDE81040FFF7B9BF002330B5A1
S21444D2D01A46441E184614F8011F392908D82F291F
S21444D2E00AD95D1C01F00F0303EB00102B4606E041
S21444D2F0A1F14105052D06D900B943B108220132F2
S21444D300072AE8D930BD5D1CA1F13703ECE71D467A
S21444D310EAE7002070470000034A92F89E30013343
S21444D32082F89E30704700BF2011422010B52A4C28
S21444D33094F89A30642B94BF0133002384F89A30CF
S21444D34094F8C63043B1013BDBB284F8C6301BB90F
S21444D35084F8C53084F88A3194F8C73053B1013B19
S21444D360DBB284F8C7302BB994F88A21032A08BF65
S21444D37084F88A31B4F8E4315BB1013B9BB2A4F83B
S21444D380E43133B9012284F8CF3184F8C13184F8CA
S21444D390A52194F8C231013384F8C231FFF7F2FC78
S21444D3A094F8A13123B1002084F8A10101F01FFCB8
S21444D3B0B4F8BE3073B1013B9BB2A4F8BE304BB94F
S21444D3C084F88A3184F8C53084F8A33184F8C131AE
S21444D3D084F8DC3110BD00BF20114220034A92F885
S21444D3E09830013382F89830704700BF20114220AD
S21444D3F070470323002010B5064CA4F8EC3104F122
S21444D40054020823E16CF5F7C5FA002384F89530F6
S21444D41010BD00BF20114220024B0022C3E9152252
S21444D420704700BF2011422030B5224B0022012411
S21444D4304FF4FB604FF4FA61082583F8A541A3F83E
S21444D4409820A3F8B420C3F8D420A3F8CA20A3F89D
S21444D450CC2083F88121A3F8822183F88C2183F899
S21444D4609C21C3F8A02183F8D62183F8DB2183F8D6
S21444D470DC21A3F8E42183F8EA21A3F8C220C3F808
S21444D480C420D864196083F89450A3F8C621C3F81E
S21444D490D02183F8D421C3E972424FF40C14C3E973
S21444D4A02E22C3E96122C3F8C04183F8C421C3E9EC
S21444D4B02B1030BD20114220144B002293F88D11BE
S21444D4C083F88A21E1B90322A3F8861183F854200D
S21444D4D093F8882142F0400283F8552093F89C2123
S21444D4E0012A01BF7F2283F85520002283F89C211D
S21444D4F0B3F8862152BAA3F8562000229A6570479C
S21444D50046F60362A3F85420E8E700BF2011422001
S21444D510054B3022A3F854200A2283F856200D22C5
S21444D52083F8C720704700BF20114220034B0122D6
S21444D53083F8C5200B2283F8C6207047201142206A
S21444D54008B5FFF783FC0330284B81B2284AC0B2A3
S21444D55007291DD85921C3F8982183F8540083F825
S21444D560551093F89E1183F85610FF2183F85710F0
S21444D570117883F85810517883F859109178D278F6
S21444D58083F85A1083F85B200422A3F8CA2008BD07
S21444D590A3F8CC10090AC3F8982141F0100183F887
S21444D5A0550083F85410592183F8561093F89E1169
S21444D5B083F85710FF2183F85810117883F85910D0
S21444D5C05178927883F85A1083F85B200322A3F8A4
S21444D5D0CA20012283F8C520022283F88A21212208
S21444D5E083F88C21222283F88821D0E72011422018
S21444D5F032224020024B002283F85420704700BF5A
S21444D6002011422038B5CB1C40F6FF749BB2A3428F
S21444D61028BF2346174C1D0A84F855306223A4F8C5
S21444D620CC1045F0100584F8580084F85630030AA8
S21444D63084F85450022163F00F03C4F8982184F808
S21444D64057300123A4F8CA301378A4F8CA1084F8D3
S21444D6505930537884F85A300323A4F8CA30937860
S21444D66084F85B30FFF762FF212384F88A1184F83C
S21444D6708C3138BD20114220F0B5C84C87B094F8A0
S21444D680C2310133DAB21B064ABF002384F8C221F2
S21444D69084F8C231B4F8C63113B1013BA4F8C6319C
S21444D6A094F8A03123B1002384F8A031FFF798FA08
S21444D6B094F88A51012D40F0288194F888312E2B15
S21444D6C03DD146F60362A4F854206289A4F8562055
S21444D6D094F88D210D2A0BD1002384F88A31012336
S21444D6E084F8953040F2F513A4F8BE3007B0F0BD88
S21444D6F00E2AF4D194F88911A9480491A9490391B2
S21444D700B4F8CA10CDE9012194F8C5202946009200
S21444D710B4F88421FFF7A8FD94F88931012B03D18E
S21444D720002001F064FAD7E7022B03D1002001F071
S21444D73079FAD1E7FF2BCFD184F8CB51CCE7222B13
S21444D740CAD1B4F88431B3F5A06F6BD1964D00229C
S21444D750964915F8010B134601321F2892B204D994
S21444D760322A01F8010BF4D11346E2182C213A2050
S21444D77082F8E4105A1C422114FA82F282F8E41029
S21444D7809A1C4F2114FA82F282F8E410DA1C14FA36
S21444D79082F282F8E4101A1D542114FA82F282F8B6
S21444D7A0E4105A1D562114FA82F282F8E410991DA8
S21444D7B0DA1D14FA81F192B281F8E4007C490878C3
S21444D7C042281FD022444E2182F8E41003F1080276
S21444D7D0302114FA82F282F8E41003F10A01093384
S21444D7E0202289B214FA83F383F8E42063180022D3
S21444D7F001314FF4A06083F8E42089B26B4AFFF706
S21444D80001FF6CE70B466B4D1878114601321F2812
S21444D81092B2EBD901332144AB4281F8E400F3D110
S21444D8201146E3E7644EB4F8862106EB4316B4F893
S21444D83086C14FEA122E3789D0B29CFA9CFCF26815
S21444D840FB1C99B2DBB207292FD984F85530C1F3B3
S21444D8500321622384F857E041F0100184F858000D
S21444D86084F85630002384F854100221A4F8CA30B1
S21444D870C4F89821A4F8CC701378A4F8CA5084F855
S21444D88059305378A4F8CA1084F85A30937884F8F8
S21444D8905B300323A4F8CA30FFF748FE322384F8EB
S21444D8A08A1184F8C630212374E0622184F8543007
S21444D8B0A4F856C0013384F855100021C4F89821C2
S21444D8C0DBB2A4F8CA10A4F8CC701078A4F8CA50F6
S21444D8D084F85800507884F859000220A4F8CA0006
S21444D8E0907884F85A000320A4F8CA00D27884F8C2
S21444D8F05B200422A4F8CA20DAB2082A3FF4ECAE2D
S21444D900E218013382F85410F6E7022D7FF4EEAEA7
S21444D91094F8C530002B7FF4E9AE94F88831222B76
S21444D9207FF4DDAE94F8C430012B06D9023BDBB25B
S21444D93084F8C430002B7FF4D9AE94F8C330072162
S21444D94094F88C212E27B4F8CC50D4F89861134818
S21444D95084F8C43084F85420B4F8CA30013901300D
S21444D960AB4238BF16F803C003F101032CBF80F85E
S21444D970547080F854C09BB211F0FF01A4F8CA302A
S21444D980EAD19D4202F10103DBB298BF84F88A11C2
S21444D9902F2B88D884F88C31A1E600BF2011422072
S21444D9A00E864600B812422000014400041242206B
S21444D9B02010400039104000687D4600FFF75CBEEA
S21444D9C038B51B4C6389A4F89E31FFF713FE94F8D0
S21444D9D09E5105F0F703022B05D10123002584F858
S21444D9E09D31284638BD012D0FD145F6061384F8DF
S21444D9F05650A4F8543094F89F3184F85730FFF7C3
S21444DA00E9FA40BAA4F85800EBE7032D12BF47F6EC
S21444DA10027345F6021384F856504FF001051BBFB7
S21444DA20A4F854301223A4F8543084F85630D8E777
S21444DA302011422008B5FFF7DDFD0B4B4CF2025295
S21444DA40A3F854209A7A012A83F8562004D1002257
S21444DA5083F8D421012008BD022A01D10122F7E728
S21444DA607F2283F85520F5E720114220064B47F6DF
S21444DA700372A3F85420012283F8560083F8571003
S21444DA8083F89C21704700BF20114220074B93F82F
S21444DA90D621132A09D093F8A521032A1FBF7F2233
S21444DAA083F8D621012283F89C2170472011422016
S21444DAB0002310B56B4C84F8D63194F8CE30222B24
S21444DAC007D194F8D531032B09D0132384F8D631E3
S21444DAD005E0202B14D194F8D531022BF5D894F8D0
S21444DAE0D63163B147F6037284F857300123A4F85D
S21444DAF0542094F8CE2084F89C3184F8562010BDE7
S21444DB00102B0BD194F8D531022BDED1A37A03F037
S21444DB107F03013B022BE2D91223D7E7852B12D190
S21444DB20A37A013B012B84BF122384F8D63194F8A0
S21444DB30D531022B02D0132384F8D63194F8D6017B
S21444DB40FFF7A4FFCBE7272B05D194F8D53103F094
S21444DB50FB03022BB8E7192B18D194F8D531012BC7
S21444DB60B3D0A27A0A2AF4D0032AF2D0022AAAD040
S21444DB70042A08D1062BA8D1A37B012BAFD0FF2BB8
S21444DB80ADD03123A2E7012AC6D19CE7282B1DD16C
S21444DB9094F8D511A27A032902F07F0305D0002B0E
S21444DBA0C9D0032BC7D0022902D0591E0129C2D995
S21444DBB012F07C0F01D01223BEE7E27A013A022A21
S21444DBC0BCD90BB1032BB9D13123B5E7142B1CD1E7
S21444DBD094F8D531042B7FF478AFE07AA37A00EB3F
S21444DBE00323207B00EB03206FF07F439842C4F866
S21444DBF0D0013FF474AF1C4B98423FF470AFFFF72C
S21444DC0067FAFF287FF46BAFBBE73E2B11D194F83D
S21444DC10D531022B7FF459AFA37A13F07F0F4FF41C
S21444DC20FA7318BF1222A4F8E43118BF84F8D62138
S21444DC3055E7312B09D194F8D531062B3FF645AF3D
S21444DC40A37A013B022B9CD849E72E2B05D194F8A6
S21444DC50D531022B7FF639AF41E70F2B3FF63FAF66
S21444DC60112333E720114220FF0040004FF2871370
S21444DC709842134B0ED10A290AD1002283F8D621A2
S21444DC8093F8D621003A18BF012283F8DB21704767
S21444DC901322F3E74FF28B12904201D10429EBE7AB
S21444DCA04FF29512904201D10329E5E74FF29312C1
S21444DCB09042F9D04FF28C129042DED10729DBE72E
S21444DCC0201142200B4B024693F90A00997A002809
S21444DCD0B3BF01F07F02012083F855200020B8BF6F
S21444DCE09A724FF00102A8BF83F8540083F8A52126
S21444DCF0704700BF20114220274B014610B593F9C8
S21444DD000A009A7A0028BBBF02F07F020020012056
S21444DD109A729A7A541E022C31D8062483F85510E7
S21444DD20022A4FF0000183F854404FF4997483F864
S21444DD305620A3F858404FF0F40483F8571083F85D
S21444DD405A404FF4FA7483F8A521A3F8E44112D15B
S21444DD50124A1278422A06D102F5800202F6DF728F
S21444DD6012784F2A03D0012283F89C2103E0012233
S21444DD70084683F8CA21002283F8CF2110BD47F60F
S21444DD800372A3F8542093F8CE2083F85620122228
S21444DD9083F85720E7E700BF2011422020104000B8
S21444DDA010B5214CA37AE07A00EB032080B2B0F59C
S21444DDB0754FA4F886010BD14FF4A063A4F88431C0
S21444DDC00123002084F88A31222384F8883111E024
S21444DDD0B0F5704F12D300F0A9FD4FF6FF7398428A
S21444DDE009D10223012084F85430637A43F0400377
S21444DDF084F8553010BDA4F88401E1E740F2DF739F
S21444DE00D4F8E001C01A47F60373A4F8543018BF98
S21444DE10012094F8CE3084F85630312384F85730B5
S21444DE20012384F89C31E5E7201142202DE9F04196
S21444DE304E4C2E23A27AE07A84F88831130900EBFC
S21444DE400220217B0E2B84F88D3180B284F8891110
S21444DE50A4F886010DD10123002084F88A3194F871
S21444DE60DB31012B71D1424A626584F89C31BDE8AE
S21444DE70F081B0F5704F13D300F0C3FD0F23024674
S21444DE80A4F8840184F88D314FF6FF73984204D089
S21444DE90384E06EB4013D96921B9032384F8DB31A5
S21444DEA00120DCE794F8CF11012901D00223F5E7DD
S21444DEB0002084F89C0194F8DB010028F0D19B688C
S21444DEC094F8D5010333DBB2984207D013232A488B
S21444DED084F8DB1184F8D631FFF7C6F9B4F88431F8
S21444DEE00027DFF89C80042506EB4313A4F8CA7089
S21444DEF0DA689B68C4F89421A4F8CC30B4F8CA30E5
S21444DF0018F8011BD4F89421D154B4F8CA30B4F8A4
S21444DF10CC2001339BB29A42A4F8CA30C0D9002020
S21444DF20FFF7CAFA94F89C3184F8DB7143B9B4F825
S21444DF30843106EB4313DB69012B08BF84F8A13117
S21444DF40013D15F0FF05D9D1AAE7022B03D10B4BAF
S21444DF506365012389E7032B01BF03F1445303F5AB
S21444DF60391303F57C53636581E700BF20114220D3
S21444DF70037F2E13687D46005F864600037F2E335C
S21444DF802C114220204B014630B593F90A009A7A68
S21444DF900028BBBF02F07F02002001209A72DA7A82
S21444DFA002F0FD04012C22D19A7A02F0FD05012DDF
S21444DFB011D183F8DC5193F8A521012A4FF00202CF
S21444DFC083F854201AD87F225A7222229A72002248
S21444DFD083F8DC2130BD12B983F8DC21EBE7022A52
S21444DFE006BF002083F8DC4183F89C41E3E7022A1D
S21444DFF01FBF7F225A7212229A72DCE79A7A83F8FB
S21444E000551083F85620E5E72011422070477047A4
S21444E0107047704750B123230549013B00284FEA17
S21444E02040009BB2B8BF4840002BF6D1704700BFB3
S21444E03069696C6CF8B56C4B064693F8A5211C468A
S21444E040012A0BD847F60372A3F854205A7A83F869
S21444E05056207F2283F8572001253DE0997A01F027
S21444E060FB05012D4AD1062384F8550084F8561042
S21444E07084F8543094F8CF31012B2FD101292DD177
S21444E0800023A4F8A631A4F8A83194F8A66101297F
S21444E09094F8A72194F8A83118BF022184F8582090
S21444E0A002EB062294F8A90184F8593003EB0223C4
S21444E0B084F85A0000EB032084F85760FFF7AAFF61
S21444E0C0030E84F8A631030C40BA84F8A731012322
S21444E0D0A4F8A80184F8C1312846F8BD94F8C231A2
S21444E0E003F1110284F8A63184F8A72103F1220231
S21444E0F0343384F8A82184F8A931C6E7022DABD17D
S21444E10093F8C121012A4FF0000210D083F8C121B0
S21444E11047F603720125A3F8542093F8CE2083F8DB
S21444E1209C5183F85620242283F85720D4E783F85A
S21444E130C121DA7A93F8A6319A420AD1227B94F81E
S21444E140A7319A4205D1B4F8A821B4F80D309A42C2
S21444E1501DD047F603730629A4F8543094F8CE30FD
S21444E16084F856304FF0350384F857304FF00103A7
S21444E17084F89C317FF470AF1C4B1B78422B08D03C
S21444E18001231B4884F89C31FFF76EF801E006290A
S21444E190F2D094F89C51002D7FF45EAFA37A022708
S21444E1A084F8556084F8563084F85470FFF721F9A3
S21444E1B0A37A062B0ED101230E4884F8CF7184F837
S21444E1C0CA31FFF748F80B48FFF745F80948FFF708
S21444E1D042F881E794F8A531023B012B9CBF01230A
S21444E1E084F8CF3178E700BF201142202010400049
S21444E1F073864600D1864600114B002293F89C1144
S21444E20083F8D621012904BF7F2183F89C2193F803
S21444E210CE2008BF83F85510312A0DD193F8D51176
S21444E220062903D9132283F8D62103E0997A0139C3
S21444E2300229F8D801207047342AFBD11222F2E78B
S21444E2402011422070B5674C0025637A264694F820
S21444E250DD2184F8CE30237A84F89C519A4284F89F
S21444E260D53101D800200FE0013B062BFAD8FFF742
S21444E2701FFC94F89C31012B0FD1D4F8E02140F2D6
S21444E280DF739A4201D0012070BD94F8D631113B19
S21444E290012BF8D884F89C51E4E7627A94F8CE309F
S21444E2A0102A43F0400003D1BDE87040FFF724BD78
S21444E2B0202A03D1BDE87040FFF704BD852A03D168
S21444E2C0BDE87040FFF7B6BB2A2B0AD1E37A84F840
S21444E2D0C33146F60223A4F85430A37A84F8563061
S21444E2E0D1E7222B04D16220BDE87040FFF758BD29
S21444E2F02E2B04D16E20BDE87040FFF797BD282B27
S21444E30004D16820BDE87040FFF73CBE2F2B0ED1E9
S21444E31046F60673344AA4F854300623013B12F8F2
S21444E320011B13F0FF0382F84B10F7D1ABE7142B15
S21444E33015D1FFF75FF9D4F8D0016FF07F439842C8
S21444E34002D02A4B984207D1012386F8A03145F2E1
S21444E3500143A6F8543096E7FEF702FFF7E7272B6B
S21444E36004D16720BDE87040FFF764BE192B03D183
S21444E370BDE87040FFF724BB312B0BD11C4A072362
S21444E380013B12F8011B13F0FF0382F8DA10F7D1B1
S21444E390712079E7112B0FD145F20213A4F85430BB
S21444E3A0A37A84F85630FFF724F81248FEF753FF52
S21444E3B01148FEF750FF66E73E2B0FD194F90A103A
S21444E3C0A37A0029FFF64EAF022142F0400284F8B9
S21444E3D0563084F8541084F8552054E7FEF79CFFD2
S21444E3E040E700BF201142202A114220FF0040008F
S21444E3F0291142207D8646009286460038B5424C16
S21444E4000F2384F88D312546237A217B03F00F02AF
S21444E410637AE07A03EB022304F1E40201EB002082
S21444E420C4F8942142F2030280B2A4F8CC30A4F893
S21444E4308A2194F8CE202F2A23D1033B2E22A4F8F7
S21444E4407A019BB284F8882104F22F12A4F886013C
S21444E450A4F8CC3084F87931A37BC4F8942184F8AA
S21444E46031310423627BA4F8CA30E37B84F87C21F0
S21444E47084F82F1184F8302184F83231FFF748F8B5
S21444E48014E0A4F8860100F051FA4FF6FF73984260
S21444E4900ED147F603723123A5F8542095F8CE20C2
S21444E4A085F8D63185F8562085F85730012038BD92
S21444E4B0164B03EB4013DA69002AEAD02E22A4F85E
S21444E4C0840184F88821032284F88A21DA689B68C8
S21444E4D0C4F89421A4F8CC300123A4F8CA30637B52
S21444E4E01370B4F8CA30D4F89421591CA4F8CA104E
S21444E4F0A17BD154B4F8CA30D4F89421591CA4F85A
S21444E500CA10E17BD154B9E720114220687D460009
S21444E51008B51A4B0022197A83F88D2101F00F00B2
S21444E520597AA3F8842101EB00219A7AC82983F802
S21444E53088211A7B88BFC82183F8E520A3F8CC102D
S21444E540D97A02EB01205A7B83F8E41083F8E6205C
S21444E5509A7BA3F8860142F2030083F8E720DA7B2D
S21444E560A3F88A0183F8E82005220548A3F8CA20C0
S21444E570C3F89401FEF7CCFF012008BD20114220C9
S21444E58032224020184B0022987A83F8D62183F80A
S21444E5909C21A0F12E0283F8CE00D1B208291DD8C2
S21444E5A040F24912CA40D24312F0010216D12E2834
S21444E5B083F8DB2114D193F8A521012A02D993F8D4
S21444E5C0CF216AB97E2283F8D62102F17E2202F553
S21444E5D0381285325A65012283F89C2101207047FF
S21444E5E00020FFF70BBF00BF20114220002340F25B
S21444E5F0F51210B5884C84F8983084F89C31A4F809
S21444E600BE204FF4FA72C4E915332368A4F8E42113
S21444E610B3F5FA6F17D1431E04F10802073013F816
S21444E620011F984202F8011BF9D14FF4FA63C4F86B
S21444E630E031227A12F0F0032BD1FFF703FE0028D4
S21444E64040F08B804CE040F2DF72934220D1037856
S21444E65013F0F00F1CD14278A2F11003DBB2182B52
S21444E66011D9852A01D03E2A12D140F2DF736B4A73
S21444E670C4F8E031431E073013F8011F834202F802
S21444E680011BF9D1D5E7664A22FA03F3DB07ECD43B
S21444E69010BD102B02D1FFF775FFD0E7202B40F0BA
S21444E6A08F8094F8CE302E3BD9B206295CD84923C5
S21444E6B0CB40DB4313F0010356D194F88A11032967
S21444E6C00ED194F8DD11072910D8B4F8CA300139B0
S21444E6D01944B4F8CC30994202D2002384F88A31E3
S21444E6E0002384F89C3184F89830D1E794F88B1151
S21444E6F0914205D14B4884F88A31FEF7ACFDEFE7EA
S21444E70084F88B210D2284F8C72094F8DB2132B993
S21444E710E218D4F89411507AB4F8CA208854B4F85D
S21444E720CA20B4F8CC10013292B29142A4F8CA205E
S21444E73042D894F8DB31012B1AD147F60372A4F879
S21444E740542094F8CE2084F85620132284F8572078
S21444E75084F89C31002384F8DB3194F89C31012BF7
S21444E76004BF7F2384F85530012384F89530B7E7F7
S21444E770022B0CD147F60373A4F8543094F8CE30E9
S21444E78084F85630332384F857300123E0E70020DA
S21444E790FEF792FEB4F88421234B94F89C1103EBC5
S21444E7A042132248DA69012A08BF84F8A12194F862
S21444E7B0A131FEF759FDCDE70133072BA5D18FE7ED
S21444E7C0302B8DD194F8DD31022B86D9312A03D1F2
S21444E7D00B2384F8C63083E794F8C5305BB9322AF5
S21444E7E009D146F20323A4F85430B4F886315BBA10
S21444E7F0A4F856304CE7A37A0021312A03F10303E8
S21444E80084F8C51084F8C610DBB284F8C33084F8A4
S21444E810C4303FF662AF63E72011422028114220FD
S21444E82013020401A2864600687D4600BA86460066
S21444E8300A4810B5FEF718FD72B64FF00053084963
S21444E8401022084C0848C3E90012FEF70DFDFBF7FA
S21444E85000F92046FEF708FDFBE700BFCC864600DD
S21444E8607154CA3DF3864600D986460038B52C4BCB
S21444E87093F8C8211C4632B9FEF7D6FD2948BDE8B0
S21444E8803840FEF7E8BC93F89820002A3FD0002290
S21444E89093F89D1183F8982081B193F89E0183F8EC
S21444E8A09D21FEF74DFE012384F8953040F2F51382
S21444E8B0A4F8BE30BDE83840FEF79BBD93F89550AB
S21444E8C0002DF3D1184A13780133DBB2022B01D85A
S21444E8D0137038BD1570FEF7CFFE94F8993094F84F
S21444E8E0C22101330132DBB284F8C221042B84F8FE
S21444E8F099300CD984F89950FEF718FDB4F89C303A
S21444E900C72B96BF0133A4F89C50A4F89C3094F8C7
S21444E910CA2194F8CB311343DBD0FFF789FF00BFFD
S21444E9202011422002874600F82140204FF2280357
S21444E930984218D84FF20F03984259D9A0F5704020
S21444E940113817280DD8DFE800F056292B2D2F3123
S21444E95031333537393B3D3F4143454547494B4D78
S21444E9604F51042070474FF29313984245D00CD829
S21444E9704FF28713984242D04FF288124FF6FF73F5
S21444E980904214BF1846012070474FF295124FF636
S21444E990FF73904214BF1846022070470620704703
S21444E9A00720704708207047092070470A207047A0
S21444E9B00B2070470C2070470D2070470E20704780
S21444E9C00F20704710207047112070471220704760
S21444E9D01320704714207047152070471620704740
S21444E9E01720704718207047192070471A20704720
S21444E9F04FF6FF707047052070470320704700208D
S21444EA007047FFF793BF1C280146F0B585B037D84A
S21444EA103F4B420103EB40169C584FF6FF739C4213
S21444EA202ED0F369012B2BD1756804F50004B36826
S21444EA30AD082246009337482B46FEF715FCD6E928
S21444EA4003639A1E012A1DD8002315E036F82310C6
S21444EA50023389B2029102990904029150880299BC
S21444EA6001440291918889B2039103990904039160
S21444EA70D188039A0A4403929D4206EB8302E5D862
S21444EA8005B0F0BD043B012B3FD90027BD4206EB41
S21444EA908701F5D916F82730204602370834DBB20A
S21444EAA00293029B1B0602934A78029B03EB0243A3
S21444EAB002938A78029B03EB02230293CB78029A52
S21444EAC0134402930B79DBB20393039B1B06039315
S21444EAD04A79039B03EB024303938A79039B03EB34
S21444EAE002230393CB7902A9039A13440393FEF7B4
S21444EAF010FCCBE756F82310023302915268039277
S21444EB009D4206EB8302F5D8BAE70023F8E700BF38
S21444EB10687D46000D8746001C28014630B403D95C
S21444EB202C4830BCFEF7A0BB42012B4B03EB4010F5
S21444EB309B584FF6FF7293421FD0C269012A1CD1DC
S21444EB400169072919D0826803F50003C468881E42
S21444EB50012814D852080234002191420DD253F8A9
S21444EB60040B050C24F8025C4D1C954205D2023178
S21444EB7080B28A4224F8040BEFD830BC704704397C
S21444EB80012925D822F0030222449442F5D053F8B2
S21444EB90041B44F8041BF8E75858050E25704D1C12
S21444EBA0AA42EAD9C0F3074565708D1CAA42E4D947
S21444EBB0C0F30725A570CD1CAA42DED90431C0B2E5
S21444EBC004348A4204F8010CD7D99142E4D3D4E7FA
S21444EBD00021FAE72E874600687D460010B50024DB
S21444EBE0A0B20134FFF798FF1D2CF9D110BD1FB514
S21444EBF00024A0B20134FFF706FF1D2CF9D1074BC1
S21444EC0002A902934FF47C730393054B0193019836
S21444EC10FEF77FFB002004B010BD00BF55EFCDAB20
S21444EC201000800008B508B9FFF7D8FF002008BDDB
S21444EC30124B00B51B688BB00293114B1A680392B3
S21444EC405A6804929B6805930299039A049B059814
S21444EC5000900C48FEF708FB039BB3F57C7F06D177
S21444EC600948FEF701FB01200BB05DF804FB07489A
S21444EC70FEF7FAFA4FF0FF30F6E700BF10008000C8
S21444EC80140080003E87460056874600618746004B
S21444EC9008B5FFF7CDFF012805D1FFF79FFFBDE874
S21444ECA00840FDF7B9BFFFF7C3FF0128F5D00020A1
S21444ECB0FFF79DFFFFF7BCFFF1E700BF10F8012BFD
S21444ECC011F8013B012A28BF9A42F7D0D01A704760
S21444ECD0034613F8012B002AFBD1181A0138704753
S21444ECE001F0FF01102A2BDB10F0070F08D010F8B4
S21444ECF0013B013A8B422DD010F0070F42B3F6D1B8
S21444ED00F0B441EA012141EA014122F007047FF0D0
S21444ED1000070023F0E80256083C85EA010586EA27
S21444ED20010685FA47F5A3FA87F586FA47F6A5FA63
S21444ED3087F68EB9EED1F0BC01F0FF0102F007026F
S21444ED4032B110F8013B013A83EA010313B1F8D11A
S21444ED500020704701387047002D06BF35460338FB
S21444ED60073815F0010F07D1013015F4807F02BF34
S21444ED70013015F4C03F0130F0BC0138704700BF85
S21444ED8081F0004102E000BF83F0004330B54FEA13
S21444ED9041044FEA430594EA050F08BF90EA020F80
S21444EDA01FBF54EA000C55EA020C7FEA645C7FEA13
S21444EDB0655C00F0E2804FEA5454D4EB5555B8BF36
S21444EDC06D420CDD2C4480EA020281EA030382EAA7
S21444EDD0000083EA010180EA020281EA0303362D39
S21444EDE088BF30BD11F0004F4FEA01314FF4801C0C
S21444EDF04CEA113102D0404261EB410113F0004F1E
S21444EE004FEA03334CEA133302D0524263EB4303D4
S21444EE1094EA050F00F0A780A4F10104D5F1200E72
S21444EE200DDB02FA0EFC22FA05F2801841F10001CD
S21444EE3003FA0EF2801843FA05F359410EE0A5F1A1
S21444EE4020050EF1200E012A03FA0EFC28BF4CF0D2
S21444EE50020C43FA05F3C01851EBE37101F0004588
S21444EE6007D54FF0000EDCF1000C7EEB00006EEB95
S21444EE700101B1F5801F1BD3B1F5001F0CD349081F
S21444EE805FEA30004FEA3C0C04F101044FEA445276
S21444EE9012F5800F80F09A80BCF1004F08BF5FEAFD
S21444EEA0500C50F1000041EB045141EA050130BDDD
S21444EEB05FEA4C0C404141EB0101013C28BFB1F5EF
S21444EEC0801FE9D291F0000F04BF01460020B1FA3A
S21444EED081F308BF2033A3F10B03B3F120020CDA0D
S21444EEE00C3208DD02F1140CC2F10C0201FA0CF0EB
S21444EEF021FA02F10CE002F11402D8BFC2F1200C50
S21444EF0001FA02F120FA0CFCDCBF41EA0C01904005
S21444EF10E41AA2BF01EB0451294330BD6FEA04044E
S21444EF201F3C1CDA0C340EDC04F11404C4F1200239
S21444EF3020FA04F001FA02F340EA030021FA04F34B
S21444EF4045EA030130BDC4F10C04C4F1200220FAA2
S21444EF5002F001FA04F340EA0300294630BD21FAE0
S21444EF6004F0294630BD94F0000F83F4801306BFA6
S21444EF7081F480110134013D4EE77FEA645C18BF9A
S21444EF807FEA655C29D094EA050F08BF90EA020F31
S21444EF9005D054EA000C04BF1946104630BD91EA29
S21444EFA0030F1EBF0021002030BD5FEA545C05D12C
S21444EFB04000494128BF41F0004130BD14F580046B
S21444EFC03CBF01F5801130BD01F0004545F0FE41DF
S21444EFD041F470014FF0000030BD7FEA645C1ABF14
S21444EFE0194610467FEA655C1CBF0B46024650EA4B
S21444EFF0013406BF52EA033591EA030F41F4002177
S21444F00030BD00BF90F0000F04BF0021704730B5FC
S21444F0104FF4806404F132044FF000054FF00001D1
S21444F02050E700BF90F0000F04BF0021704730B592
S21444F0304FF4806404F1320410F0004548BF404267
S21444F0404FF000013EE700BF42004FEAE2014FEABC
S21444F05031014FEA02701FBF12F07F4393F07F4F97
S21444F06081F06051704732F07F4208BF704793F09A
S21444F0707F4F04BF41F40021704730B54FF46074AD
S21444F08001F0004521F000411CE700BF50EA0102B0
S21444F09008BF704730B54FF000050AE050EA010259
S21444F0A008BF704730B511F0004502D5404261EBC9
S21444F0B041014FF4806404F132045FEA915C3FF40A
S21444F0C0D8AE4FF003025FEADC0C18BF03325FEAA7
S21444F0D0DC0C18BF033202EBDC02C2F1200300FA58
S21444F0E003FC20FA02F001FA03FE40EA0E0021FA7D
S21444F0F002F11444BDE600BF70B54FF0FF0C4CF46B
S21444F100E06C1CEA11541DBF1CEA135594EA0C0F1C
S21444F11095EA0C0F00F0DEF82C4481EA030621EA57
S21444F1204C5123EA4C5350EA013518BF52EA033592
S21444F13041F4801143F4801338D0A0FB02CE4FF044
S21444F1400005E1FB02E506F00042E0FB03E54FF074
S21444F1500006E1FB03569CF0000F18BF4EF0010E6C
S21444F160A4F1FF04B6F5007F64F5407404D25FEA68
S21444F1704E0E6D4146EB060642EAC62141EA55511B
S21444F1804FEAC52040EA5E504FEACE2EB4F1FD0C5D
S21444F19088BFBCF5E06F1ED8BEF1004F08BF5FEADB
S21444F1A0500E50F1000041EB045170BD06F000468D
S21444F1B046EA010140EA020081EA0301B4EB5C043A
S21444F1C0C2BFD4EB0C0541EA045170BD41F4801132
S21444F1D04FF0000E013C00F3AB8014F1360FDEBF57
S21444F1E0002001F0004170BDC4F10004203C35DA33
S21444F1F00C341BDC04F11404C4F1200500FA05F3B6
S21444F20020FA04F001FA05F240EA020001F0004256
S21444F21021F0004110EBD37021FA04F642EB0601CC
S21444F2205EEA430E08BF20EAD37070BDC4F10C04F6
S21444F230C4F1200500FA04F320FA05F001FA04F2BA
S21444F24040EA020001F0004110EBD37041F10001A6
S21444F2505EEA430E08BF20EAD37070BDC4F12005B1
S21444F26000FA05F24EEA020E20FA04F301FA05F219
S21444F27043EA020321FA04F001F0004121FA04F2C1
S21444F28020EA020000EBD3705EEA430E08BF20EA91
S21444F290D37070BD94F0000F0FD101F000464000CB
S21444F2A041EB010111F4801F08BF013CF7D041EA4D
S21444F2B0060195F0000F18BF704703F00046520051
S21444F2C043EB030313F4801F08BF013DF7D043EA22
S21444F2D00603704794EA0C0F0CEA135518BF95EAD8
S21444F2E00C0F0CD050EA410618BF52EA4306D1D15F
S21444F2F081EA030101F000414FF0000070BD50EA7E
S21444F300410606BF1046194652EA430619D094EA07
S21444F3100C0F02D150EA013613D195EA0C0F05D1F1
S21444F32052EA03361CBF104619460AD181EA030145
S21444F33001F0004141F0FE4141F470014FF00000FD
S21444F34070BD41F0FE4141F4780170BD70B54FF098
S21444F350FF0C4CF4E06C1CEA11541DBF1CEA135518
S21444F36094EA0C0F95EA0C0F00F0A7F8A4EB0504FA
S21444F37081EA030E52EA03354FEA013100F08880F1
S21444F3804FEA03334FF0805545EA131343EA1263BA
S21444F3904FEA022245EA111545EA10654FEA00266F
S21444F3A00EF000419D4208BF964244F1FD0404F528
S21444F3B0407402D25B084FEA3202B61A65EB030584
S21444F3C05B084FEA32024FF480104FF4002CB6EB41
S21444F3D0020E75EB030E22BFB61A754640EA0C00C1
S21444F3E05B084FEA3202B6EB020E75EB030E22BF01
S21444F3F0B61A754640EA5C005B084FEA3202B6EB42
S21444F400020E75EB030E22BFB61A754640EA9C0000
S21444F4105B084FEA3202B6EB020E75EB030E22BFD0
S21444F420B61A754640EADC0055EA060E18D04FEA8E
S21444F430051545EA16754FEA06164FEAC30343EA2E
S21444F44052734FEAC2025FEA1C1CC0D111F4801FFB
S21444F4500BD141EA00014FF000004FF0004CB6E7F4
S21444F46011F4801F04BF01430020B4F1FD0C88BF93
S21444F470BCF5E06F3FF6AFAEB5EB030C04BFB6EB9E
S21444F480020C5FEA500C50F1000041EB045170BD91
S21444F4900EF0004E4EEA113114EB5C04C2BFD4EBBE
S21444F4A00C0541EA045170BD41F480114FF0000E42
S21444F4B0013C90E645EA060E8DE60CEA135594EABE
S21444F4C00C0F08BF95EA0C0F3FF43BAF94EA0C0FC1
S21444F4D00AD150EA01347FF434AF95EA0C0F7FF436
S21444F4E025AF104619462CE795EA0C0F06D152EA8A
S21444F4F003353FF4FDAE1046194622E750EA41066E
S21444F50018BF52EA43067FF4C5AE50EA41047FF47E
S21444F5100DAF52EA43057FF4EBAE12E74FF0FF3CE3
S21444F52006E000BF4FF0010C02E000BF4FF0010CB4
S21444F5304DF804CD4FEA410C7FEA6C5C4FEA430C2D
S21444F54018BF7FEA6C5C1BD001B050EA410C0CBF7C
S21444F55052EA430C91EA030F02BF90EA020F0020DE
S21444F560704710F1000F91EA030F58BF994208BF45
S21444F57090422CBFD8176FEAE37040F00100704702
S21444F5804FEA410C7FEA6C5C02D150EA013C07D159
S21444F5904FEA430C7FEA6C5CD6D152EA033CD3D0A4
S21444F5A05DF8040B704700BF8446104662468C469E
S21444F5B01946634600E000BF01B5FFF7B7FF0028D1
S21444F5C048BF10F1000F01BD4DF808EDFFF7F4FFFA
S21444F5D00CBF012000205DF808FB00BF4DF808ED85
S21444F5E0FFF7EAFF34BF012000205DF808FB00BFA8
S21444F5F04DF808EDFFF7E0FF94BF012000205DF8CA
S21444F60008FB00BF4DF808EDFFF7CEFF94BF01207E
S21444F61000205DF808FB00BF4DF808EDFFF7C4FF77
S21444F62034BF012000205DF808FB00BF4FEA410CC0
S21444F6307FEA6C5C02D150EA013C0AD14FEA430CA3
S21444F6407FEA6C5C02D152EA033C02D14FF00000E0
S21444F65070474FF0010070474FEA410212F500121E
S21444F66015D211D56FF47873B3EB625212D94FEAC0
S21444F670C12343F0004343EA505311F0004F23FAAA
S21444F68002F018BF404270474FF00000704750EAFF
S21444F690013005D111F0004008BF6FF000407047BC
S21444F6A04FF00000704700BF4A0011D212F5001216
S21444F6B011D20DD56FF47873B3EB62520ED44FEA81
S21444F6C0C12343F0004343EA505323FA02F0704701
S21444F6D04FF00000704750EA013002D14FF0FF303F
S21444F6E070474FF0000070474FEA4102B2F1E043E2
S21444F6F024BFB3F5001CDCF1FE5C0DD901F0004CD0
S21444F7004FEAC0024CEA5070B2F1004F40EB83001F
S21444F71008BF20F00100704711F0804F21D113F14B
S21444F7203872BCBF01F00040704741F480114FEA84
S21444F7305252C2F11802C2F1200C10FA0CF320FA0D
S21444F74002F018BF40F001004FEAC1234FEAD3232A
S21444F75003FA0CFC40EA0C0023FA02F34FEA430394
S21444F760CCE77FEA625307D150EA01331EBF4FF01D
S21444F770FE4040F44000704701F0004040F0FE4038
S21444F78040F40000704700BF80F0004002E000BF35
S21444F79081F0004142001FBF5FEA410392EA030F33
S21444F7A07FEA226C7FEA236C6AD04FEA1262D2EB7D
S21444F7B01363C1BFD218414048404140B8BF5B4282
S21444F7C0192B88BF704710F0004F40F4000020F01B
S21444F7D07F4018BF404211F0004F41F4000121F031
S21444F7E07F4118BF494292EA030F3FD0A2F101027B
S21444F7F041FA03FC10EB0C00C3F1200301FA03F1B9
S21444F80000F0004302D5494260EB4000B0F5000FDB
S21444F81013D3B0F1807F06D340084FEA310102F19A
S21444F8200102FE2A51D2B1F1004F40EBC25008BF4C
S21444F83020F0010040EA03007047490040EB000016
S21444F840013A28BFB0F5000FEDD2B0FA80FCACF117
S21444F850080CB2EB0C0200FA0CF0AABF00EBC25044
S21444F86052421843BCBFD0401843704792F0000F32
S21444F87081F4000106BF80F400000132013BB5E785
S21444F8804FEA41037FEA226C18BF7FEA236C21D0FB
S21444F89092EA030F04D092F0000F08BF0846704760
S21444F8A090EA010F1CBF0020704712F07F4F04D12E
S21444F8B0400028BF40F00040704712F100723CBF41
S21444F8C000F50000704700F0004343F0FE4040F46B
S21444F8D0000070477FEA226216BF08467FEA236329
S21444F8E00146420206BF5FEA412390EA010F40F414
S21444F8F0800070474FF0000304E000BF10F0004360
S21444F90048BF40425FEA000C08BF704743F0964346
S21444F91001464FF000001CE050EA010208BF704761
S21444F9204FF000030AE000BF50EA010208BF7047E8
S21444F93011F0004302D5404261EB41015FEA010CFD
S21444F94002BF84460146002043F0B64308BFA3F1F5
S21444F9508053A3F50003BCFA8CF2083AA3EBC253D7
S21444F96010DB01FA02FC634400FA02FCC2F12002F6
S21444F970BCF1004F20FA02F243EB020008BF20F02D
S21444F9800100704702F1200201FA02FCC2F1200293
S21444F99050EA4C0021FA02F243EB020008BF20EA88
S21444F9A0DC7070474FF0FF0C1CEAD0521EBF1CEAB6
S21444F9B0D15392EA0C0F93EA0C0F6FD01A4480EAA4
S21444F9C0010C400218BF5FEA41211ED04FF000638D
S21444F9D043EA501043EA5111A0FB01310CF00040B9
S21444F9E0B1F5000F3EBF490041EAD3715B0040EADF
S21444F9F0010062F17F02FD2A1DD8B3F1004F40EBAF
S21444FA00C25008BF20F00100704790F0000F0CF081
S21444FA10004C08BF49024CEA502040EA51207F3A45
S21444FA20C2BFD2F1FF0340EAC250704740F4000020
S21444FA304FF00003013A5DDC12F1190FDCBF00F011
S21444FA4000407047C2F10002410021FA02F1C2F1BF
S21444FA50200200FA02FC5FEA310040F1000053EA5B
S21444FA604C0308BF20EADC70704792F0000F00F0A9
S21444FA70004C02BF400010F4000F013AF9D040EAAF
S21444FA800C0093F0000F01F0004C02BF490011F443
S21444FA90000F013BF9D041EA0C018FE70CEAD15341
S21444FAA092EA0C0F18BF93EA0C0F0AD030F0004CC1
S21444FAB018BF31F0004CD8D180EA010000F0004075
S21444FAC0704790F0000F17BF90F0004F084691F033
S21444FAD0000F91F0004F14D092EA0C0F01D142026D
S21444FAE00FD193EA0C0F03D14B0218BF084608D136
S21444FAF080EA010000F0004040F0FE4040F4000080
S21444FB00704740F0FE4040F4400070474FF0FF0C12
S21444FB101CEAD0521EBF1CEAD15392EA0C0F93EA59
S21444FB200C0F69D0A2EB030280EA010C49024FEAAB
S21444FB30402037D04FF0805343EA111143EA101364
S21444FB400CF000408B4238BF5B0042F17D024FF41C
S21444FB50000C8B4224BF5B1A40EA0C00B3EB510FF7
S21444FB6024BFA3EB510340EA5C00B3EB910F24BFE0
S21444FB70A3EB910340EA9C00B3EBD10F24BFA3EB65
S21444FB80D10340EADC001B0118BF5FEA1C1CE0D12D
S21444FB90FD2A3FF650AF8B4240EBC25008BF20F0E0
S21444FBA0010070470CF0004C4CEA50207F32C2BF34
S21444FBB0D2F1FF0340EAC250704740F400004FF0D1
S21444FBC00003013A37E792F0000F00F0004C02BF02
S21444FBD0400010F4000F013AF9D040EA0C0093F0CC
S21444FBE0000F01F0004C02BF490011F4000F013B26
S21444FBF0F9D041EA0C0195E70CEAD15392EA0C0F8E
S21444FC0008D142027FF47DAF93EA0C0F7FF470AFC5
S21444FC10084676E793EA0C0F04D14B023FF44CAF08
S21444FC2008466EE730F0004C18BF31F0004CCAD19D
S21444FC3030F000427FF45CAF31F000437FF43CAFD9
S21444FC405FE700BF4FF0FF3C06E000BF4FF0010CFB
S21444FC5002E000BF4FF0010C4DF804CD4FEA4002DD
S21444FC604FEA41037FEA226C18BF7FEA236C11D027
S21444FC7001B052EA530C18BF90EA010F58BFB2EBDA
S21444FC80030088BFC81738BF6FEAE17018BF40F05A
S21444FC90010070477FEA226C02D15FEA402C05D10E
S21444FCA07FEA236CE4D15FEA412CE1D05DF8040B93
S21444FCB0704700BF844608466146FFE70FB5FFF726
S21444FCC0C9FF002848BF10F1000F0FBD4DF808EDDE
S21444FCD0FFF7F4FF0CBF012000205DF808FB00BFCF
S21444FCE04DF808EDFFF7EAFF34BF012000205DF829
S21444FCF008FB00BF4DF808EDFFF7E0FF94BF012076
S21444FD0000205DF808FB00BF4DF808EDFFF7D2FF72
S21444FD1094BF012000205DF808FB00BF4DF808EDB5
S21444FD20FFF7C8FF34BF012000205DF808FB00BF82
S21444FD3042000ED2B2F1FE4F0BD34FF09E03B3EB0C
S21444FD40126209D44FEA002343F0004323FA02F038
S21444FD5070474FF00000704712F1610F01D1420224
S21444FD6002D14FF0FF3070474FF00000704700BF9D
S21444FD7053B94AB9002908BF00281CBF4FF0FF31C9
S21444FD804FF0FF3000F0A6B9ADF1080C6DE904CE93
S21444FD9000F03EF8DDF804E0DDE9022304B07047E5
S21444FDA038B505460C462846214600220023FFF770
S21444FDB015FC28B928462146BDE8384000F00AB864
S21444FDC0284604F1004100F005F8404261EB410149
S21444FDD038BD00BFD0B50C4B002206460F46FFF791
S21444FDE08BF9FFF761FC0446FFF70CF9074B00223A
S21444FDF0FFF782F902460B4630463946FEF7C4FF03
S21444FE00FFF752FC2146D0BD0000F03D0000F04113
S21444FE102DE9F047089D0E4604468C46002B40F0DC
S21444FE2081808A42174645D9B2FA82F24AB1C2F173
S21444FE30200106FA02F320FA01F1974041EA030C46
S21444FE4094404FEA174E230CBCFBFEF6B9B20EFBA9
S21444FE5016CC43EA0C4306FB01F0984209D9FB183A
S21444FE6006F1FF3C80F01581984240F21281023E32
S21444FE703B441B1AA4B2B3FBFEF00EFB103344EA19
S21444FE80034400FB01F1A14209D93C1900F1FF33B8
S21444FE9080F00181A14240F2FE8002383C44641A5C
S21444FEA040EA064000211DB1D4400023C5E9004382
S21444FEB0BDE8F08702B9FFDEB2FA82F2002A4FD1DB
S21444FEC0CB1B4FEA174E1FFA87F80121B3FBFEFC03
S21444FED0260C0EFB1C3346EA034608FB0CF3B342DF
S21444FEE007D9BE190CF1FF3002D2B34200F2EB80C0
S21444FEF08446F61AA3B2B6FBFEF00EFB106643EA3F
S21444FF00064408FB00F8A04507D93C1900F1FF3326
S21444FF1002D2A04500F2D2801846A4EB080440EA78
S21444FF200C40C0E78B4208D9002D00F0AF8000217A
S21444FF30C5E900060846BDE8F087B3FA83F1002910
S21444FF4049D1B34202D3824200F2BB80841A66EBA4
S21444FF50030301209C46002DAAD0C5E9004CA7E720
S21444FF60C2F120039740D8409140DE404FEA174EF6
S21444FF7008434FEA104CB6FBFEF11FFA87F80EFB17
S21444FF8011664CEA064601FB08F3B34204FA02F44F
S21444FF9009D9BE1901F1FF3C80F08E80B34240F28D
S21444FFA08B8002393E44F31A86B2B3FBFEF00EFB56
S21444FFB0103346EA034600FB08F3B34207D9BE199A
S21444FFC000F1FF3C74D2B34272D902383E44F31A6D
S21444FFD040EA01417AE7C1F1200703FA01F422FA24
S21444FFE007F31C4320FA07F906FA01F34FEA144CC8
S21444FFF0FE4049EA03094FEA1943B6FBFCFE1FFAE2
S21445000084F80CFB1E6643EA06460EFB08FAB24524
S21445001002FA01F200FA01F308D9A6190EF1FF30EB
S21445002048D2B24546D9AEF1020E2644A6EB0A069C
S2144500301FFA89F9B6FBFCF00CFB106649EA064642
S21445004000FB08F8B04507D9A61900F1FF3C2DD2AC
S214450050B0452BD90238264440EA0E40A6EB0806A2
S214450060A0FB02894E45C446CE4618D315D075B377
S214450070B3EB0C0266EB0E0606FA07F722FA01F317
S214450080CE401F43C5E90076002111E7294628469C
S2144500900EE76646EDE6184601E74345E7D2B8EB78
S2144500A0020C69EB04040138A646E0E76046D3E750
S2144500B060468CE78646B9E7614674E702383C44B5
S2144500C02BE7084647E7ACF1020C3E4411E72946C4
S2144500D0EEE600BF704700BF2DE9F04788B0002B1D
S2144500E01F461446B8BF03F10043129A109DDDF82B
S2144500F04CA0B6BF1F4600232D231370149B23F038
S2144501002008B8F1460F05D0B8F1450F00D10135A6
S214450110022300E0032307AA049206AACDE902A219
S214450120CDE9003522463B4601F0A6FDB8F1470F1E
S214450130064602D1119BDB0722D5B8F1460F06EBE2
S214450140050910D13378302B0AD1002200232046EA
S2144501503946FFF739FA18B9C5F10105CAF800500E
S214450160DAF8003099440022002320463946FFF746
S2144501702BFA08B1CDF81C903022079B4B4507D388
S214450180079B159A9B1B3046136008B0BDE8F08761
S214450190591C07911A70F0E7F7B503460029B8BF12
S2144501A0494203F8022BB4BF2D222B22092942705F
S2144501B02ADD0DF10704A4460A27A6460A4691FB02
S2144501C0F7F607FB16153035632A04F1FF340EF8AB
S2144501D0015C3146F1DC3031AEF1020504F8011C14
S2144501E0441C294661450AD30DF10902A2EB0E02CD
S2144501F0654588BF00221344181A03B0F0BD11F8B0
S214450200012B04F8012FEDE7302330318370C170A0
S214450210031DF1E72DE9F04F91B00C46DDF86880F7
S21445022016461F46054602F04DFE036809931846D6
S214450230FEF74EFD00230E93D8F800300A9007339C
S21445024023F0070303F1080294F81890D4F800B099
S214450250C8F80020D3E90023C4E91223D4E9128A5A
S2144502602AF000430B930B999C4B4FF0FF324046C8
S214450270FFF7DCF970BB994B0B994FF0FF324046C0
S214450280FFF7B6F930BB0022002340465146FFF73C
S214450290A5F910B12D2384F84330914B9148B9F117
S2144502A0470F94BF98468046032323612BF00403EB
S2144502B023604FF0000A009733460FAA214628468A
S2144502C000F0D2F9013040F08F804FF0FF3011B08A
S2144502D0BDE8F08F4246534640465146FFF7A6F9DD
S2144502E040B1BAF1000FBCBF2D2384F843307E4899
S2144502F07E4BD4E763685A1C09F0DF0142D10623DA
S2144503006360002206920EAACDE904920DAA4BF42C
S214450310806303920DF13302CDE9013223606368B1
S21445032000934246534628460B91FFF7D5FE0B9958
S214450330472980460D9908D1C81C02DB6368994257
S21445034040DDA9F102095FFA89F9B9F1650F1FD8B1
S21445035001394A4604F150000D91FFF71DFF0E9AEC
S2144503601318012A8246236102DC2268D20701D58A
S214450370013323619DF83330002B9CD02D2384F820
S214450380433098E74729BCD1002BBAD10123B7E7BC
S214450390B9F1660F18D1002963680BDD216113B9E1
S2144503A02268D00702D501330B442361A1654FF07F
S2144503B0000ADFE713B92268D20701D50233F4E70E
S2144503C00123F2E74FF067090E9B994205DB236848
S2144503D02161D807EAD54B1CE7E70029D4BFC1F110
S2144503E0020201221344E0E723685A0507D423692D
S2144503F0424631462846B84701302BD165E7B9F124
S214450400650F40F2DC80D4E9120100220023FFF795
S214450410DBF8002833D0364A012331462846B8470C
S21445042001303FF452AFDDE90D239A4202DB2368E3
S214450430D8070FD5DDE9092331462846B8470130A8
S2144504403FF443AF4FF0000804F11A090E9B013BF9
S214450450434509DC23689B0700F10181E0680F9B53
S2144504609842B8BF184632E701234A4631462846E1
S214450470B84701303FF429AF08F10108E6E70D9B80
S214450480002B37DC1A4A012331462846B847013047
S2144504903FF41BAFDDE90D23134302D12368D9078B
S2144504A0D8D5DDE9092331462846B84701303FF41B
S2144504B00CAF4FF0000904F11A0A0D9B5B424B4501
S2144504C001DC0E9B94E70123524631462846B84741
S2144504D001303FF4FAAE09F10109EEE7FFFFEF7F81
S2144504E06E874600728746007A87460076874600BE
S2144504F07E8746000E9AA36D9A42A8BF1A46002AE2
S214450500914637DC4FF0000B29EAE97904F11A02E7
S214450510D4F858A0AAEB09035B4533DCDDE90D2387
S2144505209A423BDB2368DA0738D40E9A0D99A2EB3C
S2144505300A03A2EB01099945A8BF9946B9F1000FF0
S21445054034DC4FF0000829EAE97904F11A0ADDE9B6
S2144505500D239B1AA3EB090343457FF77BAF012386
S214450560524631462846B84701303FF4AEAE08F10C
S2144505700108ECE71346314642462846B84701305F
S214450580C0D1A2E60123314628460B92B847013032
S2144505903FF49BAE0B9A0BF1010BB9E7DDE9092356
S2144505A031462846B8470130BFD18EE64B4608EB64
S2144505B00A0231462846B8470130C2D185E60E9A2A
S2144505C0012A01DCDB0737D501234246314628465A
S2144505D0B84701303FF479AEDDE909233146284670
S2144505E0B84701303FF471AED4E91201002200232A
S2144505F0FEF7EAFFD8B90E9B08F10102013B3146EA
S2144506002846B84701300ED15FE601234A463146B3
S2144506102846B84701303FF458AE08F101080E9B0E
S214450620013B4345F1DC534604F15002E1E64FF009
S214450630000804F11A09F2E701234246DFE70123E1
S2144506404A4631462846B84701303FF43EAE08F1A3
S2144506500108E3680F995B1A4345F0DCFEE64FF068
S214450660000804F11909F4E72DE9F04716469946BE
S2144506708A680B69DDF820809342B8BF134633601D
S21445068091F8432007460C460AB101333360236888
S214450690990642BF336802333360256815F0060570
S2144506A006D104F1190AE36832689B1AAB4226DC88
S2144506B094F84320131E226818BF012392062BD4B4
S2144506C004F1430249463846C04701301ED02368E8
S2144506D0E568326803F00603042B08BFAD1AA36825
S2144506E022690CBF25EAE57500259342C4BF9B1ACF
S2144506F0ED1800261A34B5421AD1002008E0012329
S214450700524649463846C047013003D14FF0FF3080
S214450710BDE8F0870135C6E7E1185A1C302081F858
S2144507204300224494F8451082F843100233C7E745
S2144507300123224649463846C0470130E6D00136B1
S214450740D9E700002DE9FF470C469146277E0C99D0
S214450750782F80469A4604F1430207D8622F0AD876
S214450760002F00F0D880582F00F0A38004F14206F1
S21445077084F842703AE0A7F16303152BF6D801A03A
S21445078050F823F0DD074500F10745006D074500A5
S2144507906D0745006D0745006D074500F1074500A7
S2144507A06D0745006D0745006D0745006D0745001B
S2144507B0FD08450021084500DF0845006D07450052
S2144507C06D0745001F0945006D0745002108450092
S2144507D06D0745006D074500E70845000B681A1D7F
S2144507E01B680A6004F1420684F842300123A3E000
S2144507F0256808682E0600F104030AD505680B60CF
S214450800002D03DA2D236D4284F843305E480A23D3
S21445081019E015F0400F05680B6018BF2DB2EFE7DD
S2144508200B682568181D0860280601D51D6802E076
S2144508306906FBD51D8854486F2F0CBF08230A232D
S214450840002184F843106668A660002EA2BF216882
S21445085021F0040121600DB9002E4DD01646B5FB9A
S214450860F3F103FB1157C75D06F8017D2F46BB42E2
S2144508700D46F4D9082B0BD12368DF0708D5236925
S21445088061689942DEBF302306F8013C06F1FF3623
S214450890921B2261CDF800A04B4603AA214640464E
S2144508A0FFF7E2FE01304CD14FF0FF3004B0BDE813
S2144508B0F087354884F8457023680E681F0656F855
S2144508C0045B0E6014D5D90744BF43F0200323606C
S2144508D01DB9236823F0200323601023B0E723685F
S2144508E043F0200323607823284884F84530E3E71F
S2144508F05E0648BFADB2E6E71646BBE70B68266818
S21445090060691D1D0D6035061B6801D5186002E03F
S2144509107106FBD51880002323611646BAE70B6897
S2144509201A1D0A601E68626800213046FEF7D8F92F
S21445093008B1801B606063682361002384F84330F8
S214450940A8E72369324649464046D0470130ABD0F2
S21445095023689B0713D4E068039B9842B8BF1846A4
S214450960A4E70123324649464046D04701309BD04E
S2144509700135E36803995B1AAB42F2DCEBE70025E9
S21445098004F11906F5E700BF8087460091874600C3
S2144509902DE9F04F87B0174603938B685A1EB2F57C
S2144509A0AE7F83BF6FF4AE755B190293002386BF97
S2144509B040F25D138B6002930B688B46002543F42B
S2144509C0F0634BF81C3BCDE9045580460C465E4625
S2144509D0AA46A9460195A26852B13B681B784E2B9C
S2144509E064D8402B3CD8A3F12B01C8B20E283AD97F
S2144509F0B9F1000F03D0236823F4807323600AF10E
S214450A00FF3ABAF1010F00F213815E4500F2058107
S214450A100125284607B0BDE8F08FA3F161020D2AEF
S214450A20E6D801A151F822F0670B4500F1094500CB
S214450A30F1094500F1094500C70B45009F0B4500E8
S214450A40F1094500F1094500750B4500F1094500DA
S214450A50F1094500F1094500F10945002D0B450012
S214450A60A3F14102DBE70E29C2D801A050F821F0D8
S214450A701F0B4500F10945001F0B4500B30B45000C
S214450A80F1094500CD0A4500090B4500090B45000F
S214450A90090B4500090B4500090B4500090B4500A8
S214450AA0090B4500090B4500090B45006E2B09D877
S214450AB0602BB2D8542B77D0592B99D1072D97D187
S214450AC0082529E0742B6FD0792BF6E72168C805F1
S214450AD01AD5029B21F08001216009F101091BB15D
S214450AE0013B01320293A260A368013BA3602369E0
S214450AF0013323617B68013B002B7B6040F3848098
S214450B003B6801333B6066E71AEB050F7FF470AF31
S214450B10226822F4C072226006F8013BE4E72268A8
S214450B2010067FF565AF22F08002F4E7BAF1000FB4
S214450B300ED1B9F1000F0ED1226802F4E061B1F58D
S214450B40E06F08D122F4F06222604FF0010AE3E735
S214450B50BAF1020F55D0012D02D0042D7FF448AFCF
S214450B600135EDB2D8E7BAF1010F7FF441AF4FF04A
S214450B70020AD1E77DB9B9F1000F7FF43CAF226890
S214450B8002F4E061B1F5E06F7FF439AF22F4F0622C
S214450B9022600125C0E7032DE2D0052DDEE7022DB4
S214450BA07FF426AF0325B7E7062D7FF421AF07254B
S214450BB0B2E7226891057FF51BAF22F420722260CA
S214450BC0CDF80490A8E7226802F4A061B1F5806FDD
S214450BD006D050057FF50CAFB9F1000F3FF40FAFC7
S214450BE0910558BF019922F4F06258BFA9EB01015F
S214450BF042F4C07258BFCDE9041622604FF0000992
S214450C008AE74FF0030A87E7D4F8803139464046ED
S214450C10984700283FF4DFAEEAE6D4F87C3116F86C
S214450C20011D3A46404698472369013B2361ECE659
S214450C306B1E062B25D8022D36D85E457FF6E8AEC8
S214450C40D4F87C3116F8011D3A4640469847236944
S214450C50013B2361F1E70298D4F87C3110F8011D79
S214450C6002903A46404698472369013B23610AF17C
S214450C70FF3A5FFA8AFABAF1020FECD1033DEDB2BC
S214450C80761B2368DA052FD55B0510D55E457FF6BE
S214450C90BFAED4F87C3116F8011D3A464046984713
S214450CA02369013B2361F1E7AA460296DFE716F87A
S214450CB0011C2369652903F1FF3306F1FF352361DE
S214450CC00CD045290AD0D4F87C313A464046984758
S214450CD0236916F8021C013BB51E2361D4F87C3106
S214450CE03A46404698472E46256815F0100559D190
S214450CF03570236803F4C063B3F5806F1CD1019B40
S214450D004B45A3EB090224D100225946404600F044
S214450D1083FED4F800C0039B1CF0020F1B680646F2
S214450D200F4621D003991A1D0A601B68C3E9006760
S214450D30E3680133E3606CE6049B002BE4D0059939
S214450D400A232A460131404600F0E6FE049B059EEE
S214450D50C21A04F26F139E4228BF04F5B7761249AD
S214450D60304600F029F8CFE71CF0040F03F1040ED7
S214450D7003D00399C1F800E0D7E7039AC2F800E02C
S214450D80D3F8008002460B46FEF750FC28B10748CC
S214450D9000F00EF8C8F80000CAE730463946FEF7B8
S214450DA0A3FCF7E7002534E6A28746008C8246007A
S214450DB0004870470000C07F0EB400B59AB01BAB24
S214450DC0019005906FF00041094806910391094945
S214450DD053F8042B04910068009301A902F0E4FD42
S214450DE0019B00221A701AB05DF804EB03B07047F9
S214450DF00C2340200802FFFF2DE9F0410F469046A0
S214450E0002F084FB04460D46B8F1000F11D0C7F337
S214450E100A53C3F16B03002B0BDD1B0503F17F550E
S214450E20002405F5401522462B46FEF765F904468F
S214450E300D4620462946BDE8F0810000000000002A
S214450E402DE9F04FA1B09B4600231C939E4B17926D
S214450E501F68824638460E46FDF73AFF4FF00008B3
S214450E6004464FF000091B961B9B1A782B2A4CD03C
S214450E703AD80D2A33D8082A33D8002A3DD000233D
S214450E800C931B9D2B78302B40F0A9806B7803F094
S214450E90DF03582B66D10C9B01931CAB00938B4A02
S214450EA0CDF808B01DAB1BA9504601F01FFD10F04C
S214450EB00706044605D0062E29D1013500231B9585
S214450EC00C93179B002B40F08E850C9BD3B1424666
S214450ED009F100431046194621B0BDE8F08F202A97
S214450EE0CDD101331B93BFE72D2AC8D101220C92E1
S214450EF05A1C1B925B78002BC3D1179B1B96002B65
S214450F0040F06F8542464B46E4E70022EFE71C9AE1
S214450F103AB135211EA802F0F0FB1C99504602F066
S214450F2031F8013E042E06D8DFE806F00A0314170A
S214450F300A00DDE91E892107C3D549F00049C0E707
S214450F40DDE91E831D9A23F4801302F2334243EAF9
S214450F500259F0E7DFF87891EDE76FF000494FF07A
S214450F60FF38E8E71B9B5A1C1B925B78302BF9D061
S214450F70002BA6D0012307931B9B08930023CDE99E
S214450F8005339B460A221B980578A5F13003D9B24E
S214450F90092926D92246394602F01CFE002832D0B9
S214450FA000202B465C4604900246652B01D0452B17
S214450FB013D11CB9079B03439FD000241B9E731C6B
S214450FC01B9373782B2B78D02D2B7BD00027A3F142
S214450FD03001092940F282801B9600259EE00023B9
S214450FE0C9E7BBF1080FD5BF0699059902FB013342
S214450FF002FB013300F10100D4BF069305930BF1C4
S214451000010B1B90BFE71B9B1A191B921B5DBBF17F
S214451010000F36D004905C46A3F13002092A12D957
S2144510200122C2E71B9B5A1C1B925B780130302B72
S214451030F8D0A3F13102082A00F2DA841B9A04900C
S214451040002008920446303B00F1010213D0049973
S21445105011440491224605190A21954213D12218B6
S214451060082A04F1010404441BDC06990A2202FB03
S2144510700133069300221B9B591C1B915B78104637
S214451080CAE75846D3E7082A04DC069F4F43069727
S2144510900132E2E7571C102FDEBF059F4F430597E9
S2144510A0F6E7102CDFBF05990A2202FB01330593AC
S2144510B0E0E70023049301227CE70027B31C1B933B
S2144510C0B37884E70127F9E708894600A8874600EC
S2144510D00000F07F1B9B591C1B915B78302BF9D089
S2144510E0A3F1310108293FF678AFA3F1300C1B9BDD
S2144510F009934FF00A0E1B9B591C1B915B78A3F175
S2144511003005092D35D9099D491B082944F61F6523
S21445111002DC6545A8BF654607B16D42002C4CD13B
S214451120079901437FF4CDAE002A7FF4E6AE692BDE
S21445113026D023DC492B23D04E2B7FF4DEAE9C49AC
S2144511401BA801F00FFE00283FF4D7AE1B9B1B786B
S214451150282B2CD197491EAA1BA801F017FE052857
S21445116025D11F9BDDF8788043F0FF4949F4E00917
S214451170A7E60EFB0C3CACF1300CBCE76E2BDCE76F
S2144511808D491BA801F0EEFD00283FF4B6AE1B9B2B
S2144511908A49013B1BA81B9301F0E4FD10B91B9B34
S2144511A001331B93DFF824924FF0000889E6844804
S2144511B002F00AFD8046894683E6049B0698EB1AAC
S2144511C0BBF1000F08BFA346102C07932646A8BFC1
S2144511D01026FDF717FF092C8046894613DD794B07
S2144511E003EBC60353E91223FDF786FF80460598B1
S2144511F08946FDF707FF02460B4640464946FDF73A
S214451200C5FD804689460F2C36DC079B002B3FF4F0
S21445121058AE22DD162B09DC6A4C04EBC304D4E930
S214451220000142464B46FDF767FFC3E7079AC4F100
S2144512302503934220DB634DC4F10F0405EBC4013F
S21445124042464B46D1E90001FDF756FF079B1C1B5E
S21445125005EBC405D5E90023E5E7079B16330BDB0D
S214451260049B584A5D1B02EBC505D5E9002340465D
S2144512704946FEF76BF89DE7079BA61B1E44002EC6
S21445128071DD16F00F030AD04E4901EBC301424605
S2144512904B46D1E90001FDF72FFF8046894636F0DB
S2144512A00F0650D0B6F59A7F27DD4FF0000BCDF8E8
S2144512B010B0CDF820B0CDF818B02223DFF80C9149
S2144512C0CAF800304FF00008089B002B3FF4F9ADF4
S2144512D01C99504601F056FE0699504601F052FEBE
S2144512E00499504601F04EFE0899504601F04AFED4
S2144512F05946504601F046FEE3E500233611404682
S21445130049461F46012E21DC0BB1804689462E4BA9
S214451310A9F1547903EBC70742464B46D7E9000186
S214451320FDF7EAFE294B0A460B4029498B42804683
S214451330BBD8A1F580118B4286BFDFF898904FF059
S214451340FF3802F15479002305937EE0F20707D56E
S2144513501D4B03EBC703D3E90023FDF7CDFE012361
S21445136001377610CEE7EED0764216F00F020AD059
S214451370144B03EBC20340464946D3E90023FDF729
S214451380E5FF804689463611DDD01F2E24DD4FF019
S214451390000BCDF810B0CDF820B0CDF818B022230C
S2144513A04FF000084FF00009CAF800308CE700BF40
S2144513B07B874600BC87460073874600FC88460008
S2144513C08C82460048894600208946000000F07F0A
S2144513D00000A07CFFFFEF7F16F0100318BF6A23BE
S2144513E0B34F0593404649460023F20704D5D7E94F
S2144513F00023FDF781FE0123761007F10807F4D197
S2144514000BB180468946059BBBB1C9F30A53C3F168
S2144514106B03002B494610DD1F2B40F32881342BE8
S214451420DEBF203B4FF0FF3202FA03F34FF00008D1
S214451430CCBF4FF05C7903EA010900220023404601
S2144514404946FEF7C1F80028A1D1069B00930899A6
S21445145023465A46504601F0EAFD089000283FF4D8
S21445146024AF049B5D1B079B002BB4BF2B46002374
S2144514700E93079B4FF0000B23EAE3731693CDF8C4
S21445148010B0089B5046596801F048FD0690002864
S2144514903FF413AF089B1A69023203F10C01920020
S2144514A00C3001F02DFD1EAB01931DAB009342465B
S2144514B04B465046CDE90A8902F0A2F81C90002812
S2144514C03FF4FBAE0121504601F03DFE0490034635
S2144514D000283FF4F2AE1D9D1E9A002DABBF0E9B15
S2144514E0169B169C0E9EACBFEE185C1B059BED1A14
S2144514F01544704B013D9D42C2F1360280F2C980CB
S2144515005B1B1F2BA2EB03024FF0010700F3B680CF
S21445151007FA03F30F930025B718059BBE421444FC
S2144515201C443346A8BF3B46A342A8BF2346002BD0
S214451530C2BFFF1AE41AF61A0E9B002B17DD049954
S2144515401A46504601F0A4FE049000283FF4B5AE76
S21445155001461C9A504601F0FFFD099000283FF4CD
S214451560ACAE1C99504601F00DFD099B1C93002F0F
S21445157000F39380079B002B08DD169A0699504684
S21445158001F086FE069000283FF497AE002C08DD55
S21445159006992246504601F0C9FE069000283FF4BB
S2144515A08CAE002E08DD04993246504601F0BEFE4C
S2144515B0049000283FF481AE069A1C99504601F0E7
S2144515C02FFF834600283FF478AE0024C36804996D
S2144515D0C4600D9301F009FFA04271DA0D9B53EAF2
S2144515E0080340F09780C9F31303002B40F0928020
S2144515F029F000431B0D1B05B3F1D66F40F28A80D8
S214451600DBF8143023B9DBF81030012B40F3828029
S21445161059460122504601F089FE0499834601F059
S214451620E4FE002876DD0599234A4B46002900F05E
S214451630928002EA0901B1F1D66F00F38C80B1F1D0
S2144516405C7F7FF7ACAE1D4A0023CDE91432404699
S214451650DDE914234946FDF74FFD0B46034308BF16
S21445166022238046894608BFCAF8003030E64FF048
S214451670FF3202FA03F303EA0808DEE6C5F17F45C2
S21445168005F57F0505F57B45E23507FA05F50F9720
S21445169042E7012300250F933EE71C993A465046FC
S2144516A001F044FE1C9000287FF464AF05E600BFB9
S2144516B0D087460002FCFFFF0000F07F000050394F
S2144516C0CDF8249066D10D9AC9F313035AB39C4AB4
S2144516D093422CD1059B404603B39A4A4B461A4043
S2144516E0B2F1D46F4FF0FF311BD8120DC2F16B0328
S2144516F001FA03F398421AD1934B099A9A4202D1BA
S21445170001303FF4DAAD8F4B099A1A4002F580193D
S2144517104FF00008059B002B95D1D9E54FF0FF33D8
S214451720E8E70B46E6E753EA08033FF47CAFE5B146
S214451730099B1D42EED00D9B059A40464946C3B1CE
S214451740FFF75AFB02460B46DDE90A01FDF71EFB8D
S21445175080468946DEE71340A3F580136FEA1359A2
S2144517606FEA09594FF0FF38D4E70F9B13EA080F85
S214451770E0E7FFF741FB02460B46DDE90A01FDF7C8
S21445178003FB0022002380468946FDF71DFF0028FF
S214451790C0D004E60499584601F081FF00224FF078
S2144517A0804306460F46FDF723FF002875D00D9B60
S2144517B0002B47D0654F0026644D099B23F0004318
S2144517C01B0D1B050F930F9A614B9A4240F0C8803C
S2144517D0DDE90A23CDE91423099BA3F15479404654
S2144517E0494601F093FE02460B4630463946FDF71C
S2144517F083FC42464B46FDF7C9FA0B465149554AC6
S2144518001940914280465ED90B9B02F15472934231
S21445181003D10A9B01333FF450ADDFF82C914FF0CE
S214451820FF381C99504601F0ADFB0699504601F02D
S214451830A9FB0499504601F0A5FB5946504601F0D0
S214451840A1FB1EE6B8F1000F19D1099BC3F313039C
S214451850E3B93E4B002230463946FDF7BFFEC8B9D0
S2144518603D4B002230463946FDF746FC04460D46BC
S21445187005F1004318941993DDE918679DE7B8F11B
S214451880010F03D1099B002B3FF489AD334F00264A
S214451890002491E70D9C304DEAE72F4B0022304659
S2144518A03946FDF729FC0D9B04460D4633B901F133
S2144518B0004310901193DDE910677EE702460B461C
S2144518C0CDE91023F7E703F15479059B002BA8D102
S2144518D029F000430F9A1B0D1B059A42A1D12046BD
S2144518E02946FEF75DFAFDF7D9FB02460B4620462C
S2144518F02946FDF749FA0D9AC9F3130343EA080347
S214451900134304460D4666D009A3D3E90023FDF7E5
S21445191065FE00287FF4DCAC07A3D3E90023204608
S2144519202946FDF779FE00283FF47BAFD0E400BF9B
S2144519309535A094FFFFDF3F35E5AF350000E03F26
S214451940FFFF0F000000F07FFFFFEF7F0000F03F36
S2144519500000E07FFFFF9F7C0000E03F0000F0BFF7
S214451960059B13B30F9BB3F1D46F1ED826A3D3E9BB
S214451970002320462946FDF73BFE90B129462046E2
S214451980FDF792FE012838BF0120FDF73BFB0D9B76
S21445199004460D46D3B901F1004312901393DDE991
S2144519A012670F9A07F1D6639F1ADDE90A0101F01F
S2144519B0ADFD02460B4630463946FDF79DFBDDE953
S2144519C00A23FDF7E3F9804689467EE702460B463D
S2144519D0CDE91223E3E70EA3D3E90023FDF7FEFD89
S2144519E0A1E700230C93179A1B9B1360FFF76DBA6C
S2144519F0652B3FF45EAB452B3FF45BAB0122FFF70F
S214451A008FBB00BFAFF300800000C0FFFFFFDF4184
S214451A109535A094FFFFCF3F014BFFF711BA00BFA6
S214451A20742340202DE9F0473A4E86468C4660465C
S214451A301CF8014BA55D15F00805F8D12D2C33D1C2
S214451A409CF800404FF0010800F1020C002B5CD0DA
S214451A50102B0CD1302C0AD19CF8000000F0DF008A
S214451A6058284DD19CF8014010230CF1020C08F182
S214451A700047013F0026B7FBF3F9304603FB197ACA
S214451A80A4F13005092D18D82C46A34224DD751C33
S214451A9007D081451DD301D1A2451ADB00FB034083
S214451AA001261CF8014BEBE72B2C08BF9CF80040A1
S214451AB0A84608BF00F1020CC8E7A4F14105192D58
S214451AC001D8373CE1E7A4F16105192D04D8573C08
S214451AD0DBE74FF0FF36E4E7731C06D12223CEF84A
S214451AE00030384642B9BDE8F087B8F1000F00D05F
S214451AF04042002AF7D00EB10CF1FF311160F2E7F3
S214451B003024002BB3D10823B1E7302CA4D00A23C8
S214451B10ADE700BFF9874600FFF784BF00B59BB029
S214451B20019105916FF00041069103910549049195
S214451B3001A901F039FF019B00221A701BB05DF820
S214451B4004FB00BF0802FFFF13460A46014602484B
S214451B500068FFF7E3BF00BF0C2340202DE9F74F91
S214451B6003690C69A3420746C0F28180013C01F136
S214451B70140800F1140505EB8403019358F8243046
S214451B8055F8242001339A424FEA840B08EB840922
S214451B90B2FBF3F631D34FF0000E4046AC46F24664
S214451BA050F8042B93B206FB03E34FEA134E9BB261
S214451BB0AAEB0303120CDCF800A006FB02E213FABC
S214451BC08AF34FEA124E1FFA82FADCF80020CAEB77
S214451BD0124202EB23429BB243EA024381454CF84C
S214451BE0043B4FEA224ADBD255F80B302BB9019B12
S214451BF0043B9D421A462ED33C61384601F0F5FB20
S214451C00002824DB013628464FF0000C58F8042BF4
S214451C10D0F800E093B2ACEB0303120C13FA8EF344
S214451C20C2EB1E4202EB23429BB243EA0243C14546
S214451C3040F8043B4FEA224CE8D255F8242005EB01
S214451C40840322B9043B9D421A460AD33C6130467A
S214451C5003B0BDE8F08F1268043B002ACCD1013CA6
S214451C60C7E71268043B002AF0D1013CEBE70020A9
S214451C70EEE70000000000002DE9F04F446A99B0F9
S214451C8016461F46CDE90467DDF8948005463CB9FF
S214451C90102001F01BF9C0E9014468620460C46085
S214451CA06B6A196851B15A684A60012393408B6044
S214451CB0284601F067F96B6A00221A603B1EB9BFD9
S214451CC023F0004305930023C8F80030DDF8149050
S214451CD0A74BBCBF0122C8F8002033EA090319D137
S214451CE0249A42F20F731360C9F31303334300F08B
S214451CF06D85269B53B99F4B23E09F4B0393083333
S214451D00269A1360039819B0BDE8F08F994B039354
S214451D100333F5E7DDE90434CDE90C34DDE90C01A0
S214451D2000220023FDF750FC804660B1249A01232B
S214451D301360269B002B00F04685904B269A136031
S214451D40013B0393DEE716AB019317AB009328469A
S214451D50DDE90C2301F054FCC9F30A548346002CF4
S214451D607ED00D9BCDF84C80C3F31303DDE90C0103
S214451D7043F07F5141F44011A4F2FF34804B0022DA
S214451D80FDF702F874A3D3E90023FDF7B5F974A36C
S214451D90D3E90023FCF7FAFF064620460F46FDF733
S214451DA041F971A3D3E90023FDF7A6F902460B4690
S214451DB030463946FCF7EAFF06460F46FDF74CFC2B
S214451DC000228246002330463946FDF707FC48B1D7
S214451DD05046FDF727F932463B46FDF7F5FB08B971
S214451DE00AF1FF3ABAF1160F57D8664B03EBCA030A
S214451DF0D3E90023DDE90C01FDF7F0FB00284ED0C2
S214451E000AF1FF3A00230F93169B1C1B631E09938A
S214451E1045BFC4F101030693002300234CBF099335
S214451E200693BAF1000F3CDB099BCDF838A0534426
S214451E30099300230A93229B092B00F2B580052BB4
S214451E40C4BF043B2293229BA3F10203CCBF0024CC
S214451E500124032B00F2B480DFE803F02D987AA422
S214451E60DDE916431C4404F23243202BC3BFC3F1BD
S214451E70400304F2124009FA03F3C3F12003C6BF38
S214451E8026FA00F0184306FA03F0FDF7BBF80123DF
S214451E90A1F1F871013C139370E70123B3E70F9066
S214451EA0B2E7069BA3EB0A030693CAF100030A931F
S214451EB000230E93BFE700230B93239B002B00F3D1
S214451EC082804FF00109CDF820904B46CDF88C9096
S214451ED06E6A00227260042202F11400984271680C
S214451EE077D9284601F01AF86B6A30601B68039369
S214451EF0089B0E2B00F2EE80002C00F0EB80BAF12A
S214451F00000F7ADD1F4A0AF00F0302EBC303D3E93D
S214451F1000341AF4807FCDE910344FEA2A145CD099
S214451F20194BDDE90C01D3E90823FDF70FFACDE996
S214451F30040104F00F040327134E002C4FD1DDE9AE
S214451F401023DDE90401FDF701FACDE904016EE051
S214451F500123B1E7AFF3008061436F63A787D23FA4
S214451F60B3C8608B288AC63FFB799F501344D33F3E
S214451F700000F07F02894600F98846007F874600C4
S214451F800000F83F488946002089460000230B9309
S214451F90239B0AEB030909F10103012B0893B8BFFC
S214451FA0012395E70123F2E70124002322930B94AE
S214451FB04FF0FF390022CDF820901223239287E771
S214451FC001230B93F4E7DDF88C90CDF820904B4633
S214451FD07EE70131716052007EE70227ACE7E107F4
S214451FE008D5DDE91001D6E90023FDF785F8CDE9EA
S214451FF010010137641008369FE700F0A580CAF146
S2144520000004A44BA44E04F00F0203EBC203D3E92D
S2144520100023DDE90C01FDF76FF8CDE90401241135
S21445202000230227002C40F08480002B8DD10F9B87
S214452030002B00F08B80DDE90434CDE91034DDE972
S2144520401001964B0022FDF7C9FA00287ED0089B62
S214452050002B7BD0B9F1000F38DDDDE91001904B40
S2144520600022FDF749F8CDE904010AF1FF380137AA
S2144520704C463846FCF7D6FFDDE90423FDF73CF829
S214452080884B0022FCF782FEA1F15076CDE910017F
S2144520901196002C5DD1DDE90401834B0022FCF747
S2144520A073FE02460B46CDE90423109A3346FDF7E8
S2144520B0B3FA002840F09782DDE90401109A06F14C
S2144520C00043FDF78BFA002840F08B82DDE90C349F
S2144520D0CDE90434179B002BC0F25181BAF10E0F9F
S2144520E000F34D816B4B03EBCA03D3E90034CDE9CE
S2144520F00634239B002B80F2DB80089B002B00F3E5
S214452100D78040F06D82684B0022DDE90601FCF77A
S214452110F3FFDDE90423FDF775FA089C26460028FB
S21445212040F04382039F312307F8013B0AF1010A39
S2144521303FE2E20705D5D6E90023FCF7DDFF013788
S2144521400123641008366DE7022770E7089CD046E1
S2144521508FE703994F4B214412910B9903EBC40328
S214452160DDE9106753E90223002946D04F49002090
S214452170FDF7ECF83B463246FCF706FECDE9100186
S214452180039FDDE90401FDF767FA0446FCF74AFFBD
S21445219002460B46DDE90401FCF7F6FD30340246FF
S2144521A00B46CDE9042307F8014BDDE91023FDF77F
S2144521B015FA002865D1DDE9042338490020FCF7E7
S2144521C0E3FDDDE91023FDF709FA002840F0B68067
S2144521D0129B9F423FF47AAFDDE91001304B002257
S2144521E0FCF78AFF2E4BCDE910010022DDE90401FC
S2144521F0FCF782FFCDE90401C3E730463946FCF7D4
S2144522007BFFCDE91001129B039C1493DDE9040185
S214452210FDF722FA1590FCF705FF02460B46DDE969
S2144522200401FCF7B1FD159B303304F8013B129BC6
S2144522309C4206460F464FF0000224D11B4BDDE973
S2144522401001FCF7A3FD02460B4630463946FDF71E
S214452250E3F9002871D1DDE9102314490020FCF785
S21445226093FD02460B4630463946FDF7B7F900283A
S2144522703FF42CAF149F7B1E149317F8013C302B6C
S214452280F8D0C24649E0064BFCF736FFCDE90401D7
S214452290BCE700BF48894600208946000000F03F5D
S2144522A00000244000001C40000014400000E03FB1
S2144522B0DDE90489039FDDE9062340464946FDF7E7
S2144522C045F8FDF7C9F90446FCF7ACFEDDE90623FB
S2144522D0FCF712FF04F130060B46024649464046D7
S2144522E0FCF752FD07F8016B039E089BBE1BB342E5
S2144522F038D102460B46FCF749FDDDE90623804604
S2144523008946FDF789F958BBDDE906234046494627
S214452310FDF75AF908B1E10722D42846594600F098
S21445232031FE00233B70249B0AF101001860269B72
S214452330002B3FF4E7AC1F60E4E427463B461F46C8
S21445234013F8012D392A07D1039A9A42F7D10399F2
S214452350302208F101080A701A7801321A7090E79F
S214452360D046EBE7A14B0022FCF7C6FE0022002331
S21445237080468946FDF728F900289CD0CDE70B9A7C
S214452380002A00F0CD80229A012A00F3AF80139AE6
S214452390002A00F0A78003F233430A9C069F069A5C
S2144523A01A440692099A01211A442846099200F0D1
S2144523B0CAFE0646002F0CDD099B002B09DDBB42F5
S2144523C0069AA8BF3B46D21A0692099AFF1AD31A0E
S2144523D009930A9BF3B10B9B002B00F0A580002CBC
S2144523E010DD31462246284600F052FF5A46014641
S2144523F00646284600F0B0FE59468046284600F078
S214452400C1FDC3460A9B1A1B04D05946284600F010
S2144524103FFF83460121284600F095FE0E9B002B84
S214452420044640F383801A460146284600F030FFAE
S214452430229B012B04467CDD4FF00008236904EB04
S2144524408303186900F031FEC0F12000099B18444B
S21445245010F01F0000F08E80C0F12003042B40F3DF
S2144524608780C0F11C00069B03440693099B0344E2
S21445247007440993069B002B05DD59461A46284610
S21445248000F054FF8346099B002B05DD21461A467E
S214452490284600F04BFF04460F9B002B6CD0214688
S2144524A0584600F0A2FF002866DA002359460A225D
S2144524B0284600F07EFD0B9B0AF1FF3A8346002B2B
S2144524C000F08B81314600230A22284600F071FD34
S2144524D0B9F1000F064600F39180229B022B40F38C
S2144524E08D8051E0169BC3F1360356E7089B5C1E6C
S2144524F00A9BA342BFBF0A9B0A94E21A0E9BB6BF2D
S2144525009B181C1B0E93089BB8BF0024002BB9BF15
S214452510069B089A069F089BBCBF9F1A00233EE76A
S2144525200A9C069F0B9E45E70A9A6EE7229B012B5F
S21445253019DC049BBBB9059BC3F313039BB9059BE9
S21445254023F000431B0D1B0583B1069B0133069301
S214452550099B013309934FF001080E9B002B7FF42E
S2144525606DAF012072E74FF00008F6E79846F4E7AE
S21445257080D018461C3076E7089B002B38DC229B1B
S214452580022B35DDDDF82090B9F1000F0DD121463F
S2144525904B460522284600F00CFD014604465846A3
S2144525A000F023FF00283FF7BDAD239B039F6FEA4E
S2144525B0030A4FF000082146284600F0E3FC002EAB
S2144525C03FF4ABAEB8F1000F05D0B04503D0414659
S2144525D0284600F0D7FC3146284600F0D3FC9CE65A
S2144525E000242646E1E7C24626469BE500002440F1
S2144525F00B9BDDF82090002B00F0F680002F05DDC4
S21445260031463A46284600F091FE0646B8F1000F98
S21445261055D07168284600F081FC3269023207467B
S214452620920006F10C010C3000F06AFC0122394696
S214452630284600F07BFE039B01330893039B4B44DF
S2144526400A93049B03F00103B04609930646089B8C
S2144526502146013B58460493FFF780FA034630333C
S2144526600690414658460B9300F0BFFE32468146DB
S2144526702146284600F0D4FEC2680B9B074602BB9F
S2144526800146584600F0B1FE0B9B024639462846A1
S214452690CDE90B3200F076FC229B0C9A089F43EA64
S2144526A00201099B0B430B9B0DD1392B29D0B9F160
S2144526B0000F01DD069B3133049A13707BE73046E5
S2144526C0B9E70122E2E7B9F1000F06DB229941EAB4
S2144526D00909099959EA010120D1002AECDD594634
S2144526E001222846089300F021FE2146834600F045
S2144526F07CFE0028089B02DCDED1DA07DCD5392BC8
S214452700D8D1049A392313703B461F46013B17F828
S214452710012C392A50D001321A704CE7002A03DDC5
S214452720392BEED00133C7E7089A0A9902F8013CDF
S2144527308A422AD0594600230A22284600F039FC08
S214452740B04583464FF000034FF00A0241462846FF
S21445275007D100F02EFC80460646089B01330893B9
S21445276075E700F026FC3146804600230A222846B7
S21445277000F01FFC0646F0E7B9F1000F039ACCBF00
S2144527804F46012717444FF0000859460122284670
S214452790089300F0CBFD2146834600F026FE002830
S2144527A0B2DC02D1089BDB07AED43B461F4613F886
S2144527B0012D302AFAD0FEE6039A9A42A5D10AF1AF
S2144527C0010A312379E7134BFFF7BBBA269B002B4B
S2144527D07FF493AA104BFFF7B4BAB9F1000F03DCA8
S2144527E0229B022B3FF7D0AE039F21465846FFF764
S2144527F0B5F900F1300307F8013B039ABA1A91453B
S214452800BADD594600230A22284600F0D2FB834605
S214452810EBE700BF7E874600F98846000369B3EBC1
S214452820611F2DE9F0434FEA611200F1140445DDBE
S21445283011F01F0104EB830604EB82050CD100F171
S21445284010072946B14234D39B1A9B00EA1E96428E
S21445285038BF0023234415E054F82270C1F1200800
